:020000041000EA
:1000000000B5324B212058609868022188439860DF
:10001000D860186158612E4B002199600221596106
:100020000121F02299502B49196001219960352056
:1000300000F044F80222904214D00621196600F024
:1000400034F8196E01211966002018661A6600F04E
:100050002CF8196E196E196E052000F02FF8012189
:100060000842F9D1002199601B49196000215960AB
:100070001A491B48016001219960EB211966A021F2
:10008000196600F012F800219960164914480160C1
:100090000121996001BC002800D000471248134993
:1000A000086003C880F30888084703B5996A0420EC
:1000B0000142FBD001200142F8D103BD02B5186610
:1000C0001866FFF7F2FF186E186E02BD00000240BE
:1000D000000000180000070000035F00212200005C
:1000E000F4000018222000A00001001008ED00E03C
:1000F00000000000000000000000000074B24E7A12
:1001000000000420E3010010C3010010E903001007
:10011000C1010010C1010010C1010010C101001097
:10012000C1010010C1010010C10100104503001001
:10013000C1010010C1010010C9030010D503001057
:10014000CD010010CD010010CD010010CD01001037
:10015000CD010010CD010010CD010010CD01001027
:10016000CD010010CD010010CD010010CD01001017
:10017000CD010010CD010010CD010010CD01001007
:10018000CD010010CD010010CD010010CD010010F7
:10019000CD010010CD010010CD010010CD010010E7
:1001A000CD010010CD010010CD010010CD010010D7
:1001B000CD010010CD010010CD010010CD010010C7
:1001C00000BE00BE00BE00BE00BE00BE00F03FF894
:1001D000103800BE00202049086006C881F3088856
:1001E00010471E48006800282DD10CA40ECC002911
:1001F00002D000F010F8F9E719491A4A002000E08F
:1002000001C19142FCD1184988471849884700BE6E
:10021000FDE701C901C29A42FBD370475C5B021043
:10022000C000002014100020BC6A0210000004204E
:1002300000000420BC6A02100010042000100420FA
:100240000000000070470A4813F092FE0047EFF3E9
:100250000580C0B27047000008ED00E0000000D04B
:100260002010002084AB0020CD020010B11F01102F
:1002700057560000F8B5C046F8BC08BC9E4670470B
:10028000F8B5C04610B5064C2378002B07D1054BB6
:10029000002B02D0044800E000BF0123237010BDF2
:1002A000B09500200000000084020010044B10B53F
:1002B000002B03D00349044800E000BF10BDC04636
:1002C00000000000B495002084020010164B002BA3
:1002D00000D1144B9D46402292029A1A9246002168
:1002E0008B460F461348144A121A17F0ADF90F4BFC
:1002F000002B00D098470E4B002B00D098470020D1
:10030000002104000D000D48002802D00C4811F017
:1003100052FE16F01BFD200029000EF0BBF911F073
:1003200047FEC04600000800000004200000000056
:10033000F5E500102010002084AB0020B71F01104D
:10034000000000007046C0082CD3EFF309808169DB
:1003500002390978002929D101B50FC8B8470CBC6A
:1003600003C29E461E4B06CB91421ED0083B1A602C
:10037000002909D0EFF3098020388863F0C0444693
:100380004D4656465F46F0C0906B1030F0C8A04610
:10039000A946B246BB4680F309882038F0C802203F
:1003A000C0430047EFF30880D1E770470D4A136858
:1003B0009942FAD801B5890053589C460FC8E047C6
:1003C0000CBC10609E46704701B50DF0EFFB03BCFE
:1003D0008E46C7E701B50DF0A7FB03BC8E46C1E70B
:1003E0003C0400200C340210102304E0202302E01F
:1003F000302300E040239C46F0B404AE7546E80884
:1004000001D3EFF309860E4F0FCE0FC70FBC0FC7F6
:100410004046494652465B460FC71DCE3100A60AEC
:1004200000D304316E0900D248311FC7EFF30980B1
:100430006946EFF3148663C76046014911F05EF91F
:1004400070A7002001480421014B18473006002006
:10045000813F011002B4714649084900095649001C
:100460008E4402BC7047C04602B471464908490038
:10047000095C49008E4402BC7047C0460022430814
:100480008B4274D303098B425FD3030A8B4244D35C
:10049000030B8B4228D3030C8B420DD3FF2209029E
:1004A00012BA030C8B4202D31212090265D0030B5D
:1004B0008B4219D300E0090AC30B8B4201D3CB0353
:1004C000C01A5241830B8B4201D38B03C01A524195
:1004D000430B8B4201D34B03C01A5241030B8B4297
:1004E00001D30B03C01A5241C30A8B4201D3CB0282
:1004F000C01A5241830A8B4201D38B02C01A524167
:10050000430A8B4201D34B02C01A5241030A8B4269
:1005100001D30B02C01A5241CDD2C3098B4201D381
:10052000CB01C01A524183098B4201D38B01C01AFF
:10053000524143098B4201D34B01C01A5241030976
:100540008B4201D30B01C01A5241C3088B4201D325
:10055000CB00C01A524183088B4201D38B00C01AD2
:10056000524143088B4201D34B00C01A5241411AF9
:1005700000D20146524110467047FFE701B5002006
:1005800000F0F0F802BDC0460029F7D076E77047CA
:1005900003460B437FD4002243088B4274D30309E4
:1005A0008B425FD3030A8B4244D3030B8B4228D385
:1005B000030C8B420DD3FF22090212BA030C8B42AB
:1005C00002D31212090265D0030B8B4219D300E04B
:1005D000090AC30B8B4201D3CB03C01A5241830BD0
:1005E0008B4201D38B03C01A5241430B8B4201D380
:1005F0004B03C01A5241030B8B4201D30B03C01AA9
:100600005241C30A8B4201D3CB02C01A5241830A22
:100610008B4201D38B02C01A5241430A8B4201D351
:100620004B02C01A5241030A8B4201D30B02C01A7B
:100630005241CDD2C3098B4201D3CB01C01A5241E2
:1006400083098B4201D38B01C01A524143098B426B
:1006500001D34B01C01A524103098B4201D30B0154
:10066000C01A5241C3088B4201D3CB00C01A524179
:1006700083088B4201D38B00C01A524143088B423E
:1006800001D34B00C01A5241411A00D201465241D7
:10069000104670475DE0CA0F00D04942031000D3F6
:1006A0004042534000229C4603098B422DD3030A4B
:1006B0008B4212D3FC22890112BA030A8B420CD35B
:1006C000890192118B4208D3890192118B4204D384
:1006D00089013AD0921100E08909C3098B4201D304
:1006E000CB01C01A524183098B4201D38B01C01A3E
:1006F000524143098B4201D34B01C01A52410309B5
:100700008B4201D30B01C01A5241C3088B4201D363
:10071000CB00C01A524183088B4201D38B00C01A10
:100720005241D9D243088B4201D34B00C01A5241E7
:10073000411A00D20146634652415B10104601D374
:100740004042002B00D54942704763465B1000D3FE
:10075000404201B5002000F005F802BD0029F8D0A4
:1007600016E770477047C046D0400B1CD1409C46EE
:10077000203AD3401843524263469340184370478F
:100780009140031C90409C46203A934019435242AA
:100790006346D340194370478446101C62468C461A
:1007A000191C634600E0C0461FB501F095FF002804
:1007B00001D40021C8421FBD10B501F0EDFE40423A
:1007C000013010BD10B501F087FF002801DB0020CB
:1007D00010BD012010BDC04610B501F07DFF0028FE
:1007E00001DD002010BD012010BDC04610B501F094
:1007F0000FFF002801DC002010BD012010BDC04605
:1008000010B501F005FF002801DA002010BD01201D
:1008100010BDC0468446081C6146FFE71FB500F0C6
:10082000D7FC002801D40021C8421FBD10B500F03C
:1008300059FC4042013010BD10B500F0C9FC002841
:1008400001DB002010BD012010BDC04610B500F036
:10085000BFFC002801DD002010BD012010BDC046F6
:1008600010B500F067FC002801DC002010BD01205D
:1008700010BDC04610B500F05DFC002801DA002074
:1008800010BD012010BDC0461C2101231B0498424D
:1008900001D3000C10391B0A984201D3000A083911
:1008A0001B09984201D30009043902A2105C4018C8
:1008B0007047C0460403020201010101000000006C
:1008C00000000000002B15D1002A13D1002906DBFF
:1008D00001DC002806D00020C043410802E080214E
:1008E0000906002007B4024801A14018029003BD88
:1008F00075FEFFFF03B4684601B5029800F02AF9BF
:10090000019B9E4602B00CBC7047C046002B11D123
:10091000002A0FD1002900D1002802D00021C943AC
:10092000081C07B4024802A14018029003BDC0464B
:1009300035FEFFFF03B4684601B5029800F048F8A1
:10094000019B9E4602B00CBC7047C046F0B5CE4637
:10095000474615042D0C2E0080B50704140C3F0CDF
:100960009946030C7E435D43674363437F19340C10
:10097000E4199C46A54203D980235B029846C444EF
:100980004B4643435143250C36046544360C24043E
:10099000A4195B19591820000CBC90469946F0BD6B
:1009A0009E2110B5C905041CFFF764FF002803D180
:1009B000201C00F069FF10BD9E21201CC90500F01D
:1009C00089FD00F061FF80231B069C466044F2E72E
:1009D000F0B54F464646D646C0B5040082B00D007D
:1009E000914698468B422FD82CD04146484602F07B
:1009F00029FE29000600200002F024FE331A9C463E
:100A0000203B9A4600D576E04B46524693401F0065
:100A10004B46624693401E00AF4228D825D053462D
:100A2000A41BBD41002B00DA7BE0002200230092D2
:100A30000193012352469340019301236246934060
:100A4000009318E08242D0D9002200230092019343
:100A50000A9B002B01D01C605D600098019902B0D8
:100A60001CBC90469946A246F0BDA342D7D90022AD
:100A70000023009201936346002BE9D0FB079846C0
:100A8000414672080A437B0866460EE0AB4201D13C
:100A9000A2420CD8A41A9D41012024196D410021C5
:100AA000013E24184D41002E06D0AB42EED9013E46
:100AB00024196D41002EF8D1009801995346001970
:100AC0006941002B23DB2B005246D3402A006446A9
:100AD000E2401C0053461500002B2DDB2600574634
:100AE000BE40330026006746BE403200801A99415E
:100AF00000900191ACE7624620239B1A4A46DA40F7
:100B00006146130042468A4017001F4380E7624651
:100B100020239B1A2A0066469A402300F340134381
:100B2000D4E76246202300219B1A00220091019203
:100B30000122DA40019280E72023624626009B1AB8
:100B4000DE402F00B0466646B74046463B00334382
:100B5000C8E7C046F0B583B016001F0000900191B1
:100B600002F07CFD04000D0002000B003000390093
:100B7000FFF7ECFE009A019B121A8B4108992000A6
:100B80000A604B60290003B0F0BDC046F8B5474687
:100B9000CE4643025B0A4400C20F9C464800DD007B
:100BA0004B02240E5B0A000E80B598462600914643
:100BB000C90FDB00271A8A4229D0002F15DD002833
:100BC0004AD1002B00D095E0ED08FF2C00D188E041
:100BD0006B025B0AE6B25B02F605580A3043D207A5
:100BE00010430CBC90469946F8BD002F00D087E01A
:100BF000601CC0B2012800DCB6E0EE1A720100D51C
:100C0000C5E0002E3DD1002200260023E3E7002F9F
:100C100000DC96E000285DD0FF2C60D08022D2045A
:100C200013431B2F00DDECE02022D21B1800934061
:100C3000F8405A1E93410343ED186B017BD50134F4
:100C4000FF2C00D1B7E0012207262A406B089A4DFD
:100C50001D4015432E4029E0FF2CB5D08022D20440
:100C600013431B2F00DDB2E02022D21B190093405A
:100C7000F9405A1E93410B43ED1A6B015BD5AD0150
:100C8000AE093000FFF700FE05388640844265DC7F
:100C9000041B330020200134E340041BA640751ED2
:100CA000AE41334307261D0000241E4001224B465F
:100CB0001A40002E04D00F232B40042B00D0043503
:100CC0006B0100D480E70134E6B2FF2C2FD1FF2660
:100CD000002380E7002B52D1FF2C00D074E70A00DC
:100CE000ED08002DF3D08023DB032B435B025B0A6E
:100CF000FF2670E7013F002FBED0FF2CB1D163E784
:100D0000002C47D0FF2869D08024E4047A42254390
:100D10001B2A00DDC5E02C002026D440B21A9540E5
:100D20006A1E954125435D1B04008946A5E7AB017A
:100D30005B0A50E7002401224B461A406B07BAD1E8
:100D400042E7002F3BD10134E0B201284ADDFF2CFD
:100D5000BDD00726ED186D082E40A7E70723574D95
:100D6000241A35401E40A1E7002C1BD1002D6ED166
:100D7000002B00D19AE00A001D003C0024E7013F4F
:100D8000002F00D158E7FF2C00D04AE7A7E75E1BF1
:100D9000894676E7002D1CD10A00FF281FD00400E9
:100DA0001D0011E7002D5DD1002B17D180230022FB
:100DB000DB03FF260FE70A00FF2600230BE7002CCA
:100DC00021D1002D66D1FF28E9D11D0087E701233D
:100DD00052E77A1CA7D0FA43FF2899D10A001D00D8
:100DE000FF24F1E6002E21D1002D4FD0002B4CD056
:100DF000ED186B019ED5314B07362E4001241D4066
:100E000054E7012318E7FF28DFD08024E4047F4261
:100E100025431B2F4DDC2026F61B2C00B540FC4043
:100E20006A1E95412543ED18040006E7002DCCD03D
:100E3000002B00D153E780216046C903084203D04C
:100E40004046084200D11D000121114047E7002B18
:100E500000D1B9E6EA1A500125D507265D1B2E40C0
:100E6000894623E7FF24002B00D1ADE680226046AF
:100E7000D203104204D04046104201D11D008946E1
:100E800001224B46FF241A409EE62B00DD080A0093
:100E900000249DE67A1CC6D0FF43FF28B9D11D006F
:100EA0001DE701253FE7151E00D044E7002200237F
:100EB00091E60125B7E7C046FFFFFF7DFFFFFFFB7F
:100EC000F8B557464E464546DE464402E0B5460074
:100ED0008846640A360EC70F002E63D0FF2E24D03A
:100EE0008023E400DB041C43002399469B467F3E9D
:100EF000434642465D02D20F5B006D0A1B0E9046D0
:100F0000924665D0FF2B55D080220021ED00D204FF
:100F10007F3B1543F61A43464A467B400F2A00D9C9
:100F20008DE06D48920082589746002C54D10823DA
:100F30009946063BFF269B46DAE7002553460229E1
:100F40001BD0032900D1BFE0012928D030007F3019
:100F5000002820DD6A0704D00F222A40042A00D08E
:100F600004352A0103D530005C4A80301540FE2844
:100F700003DCAC01640AC2B201E0FF220024640277
:100F8000D205600ADB07104318433CBC90469946E3
:100F9000A246AB46F8BD0122101A1B287CDD0022B8
:100FA0000024ECE7002C1DD104239946033B0026C6
:100FB0009B469DE7FF3E002D20D1022143464A4635
:100FC0007B400A430F2AD8D845489200825897465A
:100FD000002D19D10121F1E70C239946093BFF2689
:100FE0009B4685E72000FFF74FFC7626431F9C4079
:100FF00000237642361A99469B4679E74A460323F0
:101000001A439146032186E72800FFF73DFC431F62
:1010100036189D40763600217DE780240023E403C6
:10102000FF22ACE700258023DB031C4228D01D42B1
:1010300026D12B435C02640A4346FF229FE76201EC
:101040006C01A24224D21B210025013E0127100081
:101050006D005200002801DB944201D8121B3D4371
:1010600001390029F3D11400621E944125436DE734
:10107000BA46594625005346022900D061E77CE76D
:101080008023DB031C436402640A3B00FF2276E7F3
:10109000121B1A210125D9E79E362A00B5402C00E3
:1010A000C240651EAC411443620704D00F222240A7
:1010B000042A00D00434620103D4A401640A00228B
:1010C0005DE7012200245AE78024E4032C436402F4
:1010D000640AFF2253E7C04694C80110FFFFFFF7E0
:1010E000D4C8011070B542004E024C0045026D0A92
:1010F000120EC30F760A240EC90FFF2A0FD0FF2C41
:1011000011D00120A24200D070BDB542FCD18B426B
:101110000DD0002AF8D12800451EA841F4E701208F
:10112000002DF1D1EBE70120002EEDD1E9E7002001
:10113000EAE7C04670B54A004E02450244006D0A17
:10114000240EC30F760A120EC90FFF2C15D0FF2AEA
:101150000ED0002C15D1002A01D1002E1CD0002D5C
:1011600014D08B4227D00220013B1840013870BDBB
:10117000002EEED002204042F9E7002DFAD1FF2ADE
:101180000ED0002A0ED1002EEDD00BE00123013944
:10119000994308000130EAE70020002DE7D0E2E79C
:1011A000002EE7D18B42DED1944205DD0221581E8C
:1011B00008400138DBE70024A24204DCB542D2D863
:1011C0000020B542D3D2581E012398430130CEE708
:1011D00030B5420044024D02C30F4800640A120EAB
:1011E0006D0A000EC90FFF2A12D0FF280CD0002A6A
:1011F00012D1002819D1002D17D1002C2BD002209C
:10120000013B1840013826E0002DF0D0022022E0FA
:10121000002CFBD1FF281FD000281FD1002D1DD18D
:101220000220013B1840013815E0002C0ED08B4203
:10123000E5D10022904204DCAC42E0D80020AC4270
:1012400009D2581E01239843013004E001230139DB
:1012500099430800013030BD002DD7D18B42CED14B
:101260008242E7DD0221581E08400138F3E7C046FC
:10127000F0B54E4657464546DE46E0B543025B0AAA
:10128000450083B00F1C99462D0EC60F002D57D078
:10129000FF2D24D08020DB00C004184300238146AA
:1012A0009A469B467F3D7C027A00FB0F640A120E31
:1012B000984623D0FF2A4BD0E30080240020E4048A
:1012C0007F3A1C43AD186B1C474601935346774049
:1012D0003A000F2B48D87D499B00CB589F46002BE6
:1012E00000D085E008339A46063B9B467C027A0094
:1012F000FB0FFF25640A120E9846DBD1002C00D0AC
:1013000090E0524601231A4392460120DBE74C4607
:1013100058461700022824D0032800D1CFE000222D
:10132000002301284DD15802D205400AFF0710437F
:10133000384303B03CBC90469946A246AB46F0BD4C
:10134000002B5BD104239A46033B00259B46AAE76A
:10135000FF35002C60D1524602231A4392460220E8
:10136000B1E7FF220023DEE74B461B0C9C464B46B1
:101370002604360C180461463300220C6446000C27
:1013800043434E435043544380191A0C121896425B
:1013900003D9802149028C4664441B041B0C1004B1
:1013A000C01883015E1EB341800E1843130C1B1935
:1013B0009B0103431C00230179D5012362081C40D3
:1013C0001443019A7F32002A4DDD630704D00F23B6
:1013D0002340042B00D00434230103D53C4B019A55
:1013E0001C408032FE2ABCDCA3015B0AD2B29AE721
:1013F0000C239A46093BFF259B4654E71800FFF74C
:1014000043FA4A46431F76259A4000236D4291468F
:101410002D1A9A469B4646E7524603231A439246A4
:10142000032050E72000FFF72FFA431F2D1A9C409E
:10143000763D002047E780230027DB03FF2272E789
:10144000424666E74C463200584662E780234A46E9
:10145000DB031A4222D01C4220D123435B025B0AE9
:101460004746FF225FE701239A1A1B2A21DC23004B
:101470000199D3409E318C401A0023005C1EA34189
:1014800013435A0704D00F221A40042A00D0043311
:101490005A0111D49B015B0A002244E780234A468B
:1014A000DB0313435B025B0A3700FF223BE7019536
:1014B00087E70022002336E70122002333E7802359
:1014C000DB0323435B025B0AFF222CE714C90110F4
:1014D000FFFFFFF7F8B54746CE464400C20F80B580
:1014E00047024802400A8446664648007F0A240EA6
:1014F000F60025009046FB00000EC90FB146FF28FC
:1015000000D185E001267140261A914257D0002E65
:1015100043DD002800D07FE04946002900D1AAE041
:10152000013E002E00D0F7E05B1A5A0100D48BE098
:101530009B019C092000FFF7A7F9053884408542EC
:1015400000DDD3E0451B230020200135EB40451B87
:10155000AC40621E94412343072400251C40012215
:1015600041460A40002C04D00F211940042900D024
:101570000433590100D480E00135ECB2FF2D00D0D6
:10158000A3E0FF2400235B02E405580AD2072043AE
:1015900010430CBC90469946F8BD002E74D1601CD7
:1015A000C0B2012800DCA7E04A469C1A620100D5BF
:1015B000B6E0002CBED1002200240023E3E7002E79
:1015C00000DC85E0002846D0FF2C49D08022484628
:1015D000D2041043814601221B2E09DC20204C46F8
:1015E000801B84404A462000F240441EA041024332
:1015F0009B185A0128D50135FF2D00D1A8E0012202
:10160000072494491A405B080B4013431C40A6E78B
:10161000002E00D078E775E7FF2C54D08022494691
:10162000D2041143894601221B2E09DC20214846A1
:10163000891B88404A460100F240481E81410A4306
:101640009B1A5A0100D573E7012241460A40590707
:1016500000D089E711E04846002858D1FF2C0CD172
:10166000DB08002B00D18CE78020C00303435B0222
:101670005B0AFF2487E7FF2C25D0DB08FF2DF0D085
:101680005B025B0AECB27EE7002C4DD0FF2818D03D
:101690008024E404724223431B2A00DDC4E01C00C2
:1016A0002025D440AA1A93405A1E934123434A4608
:1016B0000500D31A884638E7721CF8D0F243FF2899
:1016C000EAD10A004B46FF25D7E79B015B0A5AE7A0
:1016D000002E41D1651CE9B2012945DDFF2D00D165
:1016E0004FE707244B445B081C4038E707225A4B5E
:1016F0002D1A2340144032E7002C1DD1002B7AD143
:101700004B46002B00D191E00A000025B5E7013ED1
:10171000002E19D14B446CE7FF2C84D1FF25ACE798
:101720004A468846D41A05E7002BC5D10A00FF288F
:10173000C8D005004B46A0E7002B49D14B46002BF3
:1017400077D00A00FF2598E7FF2C00D043E787E712
:101750000A00FF24002316E7002C15D1002B57D1D7
:10176000FF28E6D14B467BE7002C20D1002B57D039
:101770004946002953D04B445A0168D50724364ABC
:101780001C4001251340EAE6FF28EBD08022D2045A
:10179000764213431B2E53DC2025AD1B1A00AB40B1
:1017A000F2405C1EA34113434B44050021E7002B8C
:1017B000D8D04946002900D152E78021C9030F4201
:1017C00000D14DE76046084200D049E74B4647E765
:1017D0004846FF25002800D14FE78022D203174258
:1017E00004D06046104201D14B4688460122414652
:1017F000FF250A4041E7484600281FD01A1A500129
:1018000020D54A460724D31A1C4088460025A6E660
:10181000741CC9D0F643FF28BCD14B4620E799463B
:101820004B460025DB082BE7012340E7002200237D
:10183000A9E680230022DB03FF24A4E600251CE7A1
:101840000123B1E7002AF1D013000025FCE60025B2
:10185000FAE6C046FFFFFF7DFFFFFFFB42024B029F
:1018600040004900520A5B0A090E000EFF2806D00C
:101870000020FF2902D11800431E98417047FE380E
:10188000002AFBD1F4E7C04641024200C30F490AD7
:10189000120E00207E2A0DD99D2A0CD8802000042B
:1018A0000143952A0ADC9620821AD1404842002B37
:1018B00000D108007047034A9818FBE7963A914018
:1018C000F4E7C046FFFFFF7F70B500283DD0C31787
:1018D000C5185D40C40F2800FEF7D6FF9E22121ADD
:1018E000962A07DCD2B2082833DD08388540680222
:1018F000400A23E0992A0BDD052329001B1AD94051
:1019000003001B339D402B005D1EAB4119430D00AE
:10191000052801DD431F9D402B000F490B406E073A
:1019200009D00F263540042D05D004335D0102D5C2
:101930009F220B40121A9B01580AD2B24002D205D4
:10194000400AE4071043204370BD00240022002019
:10195000F4E76802400AF1E7FFFFFFFBF0B54F46EE
:101960004646D6460C000903C0B5490A470F5E003B
:1019700039431F03DB0F9C4665007B0A570F1F434B
:101980006D0DE40F760DA146C000B846D200AB1B2A
:1019900064457BD0002B5FDD002E00D0A4E03E002C
:1019A000164300D112E15E1E002E00D09EE1871A80
:1019B0004346B84280410125C91A4042091A0B0228
:1019C00000D431E149024E0A002E00D16EE1300010
:1019D000FEF75AFF0300083B1F2B00DD61E12022C8
:1019E0003900D21A9E40D1409F400E439D4200DDF7
:1019F00051E15D1B6B1C1F2B00DD7CE12021C91A0E
:101A00003D0030008F408840DD40791E8F4131001D
:101A100007222843D940002507433A40002A09D02D
:101A20000F233B40042B05D03B1DBB42BF417F42EF
:101A3000C9191F000B0200D426E26A1CC64B5505CB
:101A40006D0D9A4200D106E1C44AFF080A405307CF
:101A500052023B43120B8EE0002B00D0B8E06B1C0F
:101A60005B055B0D012B00DC30E1871A4346B84271
:101A7000B641CB1A76429E1B330200D54CE13B00A7
:101A80003343A1D100220024002570E0002B00DCAC
:101A9000E5E0002E00D183E0AF4EB54260D0802655
:101AA00036043743B846382B00DC3EE14346134347
:101AB0001F007A1E97413F18874280414042091813
:101AC0000B0200D4B0E0A44B01359D4200D1C3E02D
:101AD000A24A7B080A4001210F401F435108D30747
:101AE00007221F433A4099E79B4EB54238D08026E3
:101AF00036043743B846382B00DDDCE01F2B00DC12
:101B000030E11E004746203EF740BC46202B04D063
:101B10004026F31A46469E403243170063467A1E1B
:101B200097411F43CCE0002B00D104E2434613430E
:101B300000D159E14B07C00818438023C9081B0393
:101B4000194208D04546ED081D4204D14346D0084D
:101B5000590708432900420FC9007F4D1143C000B7
:101B60004B07CA087C49C00803438D4268D0120362
:101B70006D05120B6D0D002112031800130B0A0DD9
:101B800012051A43764B2D0513402B435B00E407E7
:101B90005B08234319001CBC90469946A246F0BD41
:101BA0003E00164312D05E1E002E00D000E18718C2
:101BB0008742804141444042091801250B0233D538
:101BC000022585E764463300414610001D00C7E743
:101BD000002D00D0DAE00C000443F3D05C1C00D1EF
:101BE0009FE15D4CA64200D12FE1DB43382B00DDA5
:101BF00066E11F2B00DD83E120240500E41A0F00BD
:101C0000DD40D940A0404346A7405B1A441EA04196
:101C100098462F433843171ABA42924143465242DC
:101C2000991A64463500CAE607223A40002A00D0D5
:101C3000F6E64B07CA084849FF083B438D4296D158
:101C40001900114300D19EE1802109030A431203C8
:101C5000120B414D8FE71500002200238BE7002B6C
:101C600000D0C7E06B1C5F057F0D012F00DCF1E0A9
:101C7000394DAB4200D1B9E085180A00854289414F
:101C80004244494251180722CF076D082F434908A3
:101C90003A401D00C2E607223049ED1A31403A4071
:101CA000BCE63E002838864000279FE63800FEF755
:101CB000EBFD20308EE6434613431F007A1E97410A
:101CC000C71BB84280414042091A78E60E003B002B
:101CD00006431343002D61D1002E00D0F4E0002B09
:101CE00000D11BE164463900100039E71A4FBB42AE
:101CF0007AD03300FFE630001F3DE840202B03D0B0
:101D00004021CB1A9E4037437B1E9F410722074349
:101D10003A400021002589E7171A4346BA42B641E6
:101D2000591A76428E1B64464EE61F2B00DDADE04D
:101D300020264746F61AB740B9461700B246DF409C
:101D40004E463E4337005646B240561EB2411743F8
:101D50004246DA408918AEE6FF070000FFFF7FFF2A
:101D6000FFFF0F8020264746F61AB740B9461700F6
:101D7000B246DF404E463E4337005646B240561EFE
:101D8000B24117434246DA40891A99E77F4CA6428E
:101D90005BD0802424045B42214327E7002E0CD132
:101DA000002B00D1CBE0644639001000774DD7E618
:101DB000764FBB4218D0330075E6002B14D04B078A
:101DC000C00818438023C9081B03194207D0FC0828
:101DD0001C4204D17907D0080843E14621004C4653
:101DE000420FC9001143C000684DB9E61D00002232
:101DF0000023C0E6002D5BD10D00054300D1E2E6D3
:101E00005D1C00D1B0E0614DAE421FD0DB43382BEA
:101E100071DC1F2B00DD96E020250F00ED1AAF408E
:101E2000B9460700AA46DF404D463D432F005546C0
:101E3000A840D940451EA84188440743BF1897428F
:101E400092415142414435003AE6644635004146EC
:101E5000100085E60B000343002D00D063E6002B45
:101E6000F5D04346134300D17AE687188742804174
:101E700007224144404209183A400B0200D4D5E6FB
:101E8000434B01351940C9E5380069E61E00474655
:101E9000203EF740BC46202B04D04026F31A46468D
:101EA0009E403243170063467A1E97411F4302E665
:101EB000364DAE42CAD080252D045B422943A6E7A9
:101EC0000843411E8841A6E6002B00D148E6871A48
:101ED0004346B842B641CB1A76429E1B33024BD5DD
:101EE000171A4346BA429241591A5242891A072296
:101EF00064463A4092E501430F00791E8F419DE709
:101F00001C000F00203CE740202B03D04024E31AA4
:101F100099400843411E884138437CE60022002452
:101F200025E6171A4346BA429241591A5242891A73
:101F30006446350043E541461000144D10E680220A
:101F40000024120380E61D000F00203DEF40BC4638
:101F5000202B03D04025EB1A994008430700634625
:101F6000781E87411F4369E7871897429B41414488
:101F70005B42C9183500A3E53B003343CED00722AE
:101F800031003A4052E600231A00F4E5FF07000052
:101F9000FFFF7FFFF0B55746DE464E464546E0B5AB
:101FA000834607000E03480085B092461C00360B9E
:101FB000400DCD0F002800D19DE0954B984239D0BF
:101FC0008023F6001B041E43924A7B0F334399463D
:101FD000944603006344009300230026FF0002930D
:101FE00023031B0B98466300E40F52465B0D0194DC
:101FF00000D1B3E086498B4200D19EE04246D10039
:10200000802212040A435146490F11438B468149ED
:1020100052468C4600996344CB1A0021D2000093AB
:102020002B0063409A460F2E00D905E17A4BB6008B
:102030009B599F465B463343994600D0B8E0022344
:102040000826002700900293CAE7CB463A0002997F
:102050000195019B9A46022927D0032900D180E2ED
:10206000012944D06D49009B8C4663441C00002C20
:1020700038DD530700D013E2D2085B46DB0109D5F7
:102080005946674B19408B468021C9008C46009BFE
:1020900063441C00634B9C4207DC5B4664055F079E
:1020A0005B0217431B0B620D02E000230027584A16
:1020B00000211B031C0B0B0D1B05234314055A4A5F
:1020C000380013401C4353466400DB0764081C437C
:1020D000210005B03CBC90469946A246AB46F0BDF7
:1020E0000122524201231B1B382B00DCADE10022F0
:1020F00000230027DCE75B46334399465ED0002E81
:1021000000D18AE13000FEF7BFFB03000B3B1C2B24
:1021100000DD7BE11D22D31A5A460100DA4008395E
:102120008E4013005F46334399468F403F4B002655
:102130001B1A00930023029352E7414653460B4378
:102140003B499B468C46009B634400935B46002BB7
:102150003BD1022300221E43022161E74346134381
:102160009B4637D04346002B00D162E14046FEF744
:102170008BFB03000B3B1C2B00DD53E102004146AF
:10218000083A914088461D21CB1A5146D9400B0090
:1021900041460B439B46534693401A00009B2549FA
:1021A0009C46604403008C4663440093002137E75B
:1021B0000323B14600900C26029311E700230093FD
:1021C00001330426002702930AE70323C3461E4374
:1021D000032125E701331E430022012120E70023CC
:1021E0009A46802300271B03094A61E7802349465A
:1021F0001B03194200D1E2E05946194200D0DEE04B
:102200000B431B0317001B0BA246014A50E7C046B5
:10221000FF07000001FCFFFF54C90110FF0300008D
:10222000FFFFFFFEFE070000FFFF0F800DFCFFFF1A
:1022300001F8FFFFF3030000D94500D9CBE000D13E
:10224000C6E03C0048460027009B013B00935B46EC
:10225000160E1B021E431302984633041B0C9946AC
:10226000310C0191FEF790F94A4642430B04210CD0
:10227000050019438A4207D98919013D8E4203D8C6
:102280008A4201D9851E8919881A0199FEF77CF9BD
:1022900009048C464A46210464464243090C030063
:1022A00021438A4204D98919013B8E4200D8F1E0CA
:1022B0002D041D43AB464346891A4246280C12049E
:1022C0001D0C5B46140C22001B041B0C5A43039488
:1022D0006B434443029568431B19150CEB189C4251
:1022E00003D980246402A44660441C0C15041B041A
:1022F0002D0C20185D19814277D373D00C1AA24A95
:102300007D1BAF42BF419446009B7F426344E01B6C
:102310001C00864200D1DBE00199FEF735F94A4600
:1023200042430B04290C070019438A4207D9891933
:10233000013F8E4203D88A4201D9871E8919881A23
:102340000199FEF721F909044A46894629044D46B8
:102350004243090C030029438A4207D98919013BEA
:102360008E4203D88A4201D9831E89193F04891AF3
:102370003A00039F1A43380013041B0C584381464C
:102380000298150C6F43434345434846000C84466E
:10239000DB1963449F4203D9802040028446654490
:1023A00048461F0C00041B04000C7D191818A94294
:1023B00000D284E000D17FE001231A4357E6802356
:1023C0004A461B0313431B031B0BAA466F4A6FE6C7
:1023D000BA4200D935E74B46DC0758087B081C4356
:1023E000FF0734E70024AF4289D247444745A44160
:1023F0005B466442A4196418013BA6421ED2A04267
:102400006DD800D1B6E0241A9B4678E703005A46FF
:10241000283B9A400027914688E65846FEF734FA52
:10242000203072E603005246283B9A409346002231
:10243000B4E65046FEF728FA20309AE6A642E2D1EA
:10244000B845DCD9341A9B4659E71F2B65DC504C44
:102450000099A4465C46614408008C40110082400B
:10246000D940501E82410C4314435A46DA401300AF
:10247000620709D00F222240042A05D02200141D31
:102480009442894149425B181A0262D50122002315
:1024900000270DE68A4200D80AE7831E891907E75C
:1024A0000F231340042B00D1E6E5171D97429241FC
:1024B00053429B44FA08E0E5002800D1D7E57118A3
:1024C000531EB14227D3A94215D358D01A0073E73F
:1024D000002B00DC04E6012300229B44CDE502230F
:1024E0004744474589415B429C46494289190C193A
:1024F000E344241A03E743465F0047459B41B8463F
:102500005B429E19023A8919A94200D054E740451E
:1025100000D051E7ABE51A00F6E71F215F464942BC
:102520000C1BE740202B07D01A49009B8C466344C4
:1025300018005B4683401A43501E82413A430727E6
:102540000023174009D00F21002311401400042953
:1025500095D122005F075B021B0BD20817430022B4
:10256000A6E5802359461B030B431B0317001B0BD7
:10257000064A9DE5BD42B2D89B460024BFE6804591
:10258000B9D31A00C3E7C046FF030000FF070000ED
:102590001E0400003E040000F0B54F464646D646F5
:1025A0008446C0B58046194E18030F034D00000B3A
:1025B0005C0082463F0B6D0DC90F9146640DDB0F29
:1025C0000120B5420AD0B44203D0A54201D15745FB
:1025D0000CD01CBC90469946A246F0BD66463E43D0
:1025E000F7D1AC42F5D154461443F2D10120C8458D
:1025F000EFD1994207D0002DEBD163461F4338003D
:10260000471EB841E5E70020E3E7C046FF070000AA
:10261000F0B54F464646D6464D00C0B50E03C90F2D
:102620008A462C491F035C008046360B6D0D91468F
:102630003F0B640DDB0F8D421ED08C4216D0002D57
:102640001ED130438446002C01D13A4323D0624648
:10265000002A1AD09A4529D0514602200139084053
:1026600001381CBC90469946A246F0BD3900114382
:10267000E5D002204042F4E73043FAD1AC420FD01B
:10268000002C0FD13A43E7D00CE00122013B9343E9
:1026900018000130E5E763460020002BE1D0DBE7BE
:1026A0003A43E6D19A45D7D1A542D5DCA54205DB10
:1026B000BE42D1D808D00020BE42D2D2504601231B
:1026C000013898430130CCE7C845C5D80020C8453B
:1026D000F4D3C6E7FF070000F0B54F464646D6469E
:1026E0004D00C0B50E03C90F8A462E491F035C007A
:1026F0008046360B6D0D91463F0B640DDB0F8D420E
:1027000018D08C4211D0002D18D130438446002CB3
:102710001ED13A431CD163460020002B30D05146D5
:1027200002200139084001382AE039001143EAD07B
:10273000022025E03043FBD1AC4226D0002C26D12C
:102740003A4324D15146022001390840013817E0AC
:102750006246002A0FD09A45E1D1A54205DBBE4270
:10276000DDD819D00020BE420AD2504601230138DC
:102770009843013004E00122013B934318000130EB
:102780001CBC90469946A246F0BD3A43D0D19A452A
:10279000C5D1A542C3DCE0E7C845C0D80020C84584
:1027A000E3D3EDE7FF070000F0B55746DE464E469F
:1027B0004546E0B5834606000F03480087B09246C1
:1027C0001D003F0B400DCC0F002800D16FE0DE4B09
:1027D000984238D08023FF001B041F43730F3B43F4
:1027E0000193DA4B0027994600239B46F60081446B
:1027F0002B0369001B0B52469846490DED0F00292B
:1028000000D185E0D04B994200D173E04346DA0015
:1028100080231B0413435246CC48520F8446134373
:10282000524600206144D200894421006940009151
:102830008C46012149448A460F2F00D990E0C449B3
:10284000BF00CF59BF465B463B43019300D06AE1CE
:1028500002230827002681469B46C9E732005846D6
:10286000019B61460091022800D175E0032800D148
:10287000FEE1012800D02CE10023002700260025DE
:102880003F032A0D3F0BB34812053A4302401B0594
:102890001343009A5B00D1075B080B43300019001B
:1028A00007B03CBC90469946A246AB46F0BD5B469D
:1028B0003B43019300D12FE1002F00D1A5E1380067
:1028C000FDF7E2FF03000B3B1C2B00DD96E11D2210
:1028D000D31A5A460100DA405E4608398F40130089
:1028E0008E403B4301939C4B00271B1A99460023C3
:1028F0009B467DE7414653460B4393498C46E14452
:10290000002B00D01AE102220220174300228CE79C
:10291000134300D10DE14346002B00D181E1404635
:10292000FDF7B2FF02000B3A1C2A00DD72E1010044
:10293000434608398B4098461D239A1A5346D34084
:102940001A004346134352468A404946081A8249B0
:1029500089468144002068E77B4B002700268EE7EC
:10296000140C1204120C1100370C3604350C794388
:1029700028008C462E006043604483465643210065
:10298000300C80465846794340440291844506D92C
:102990008846802149028C46E04441460291360433
:1029A000010C360C00048B4681191E0C1B041B0CF9
:1029B0000391190079438C46280075436544A84665
:1029C0005843050C45447743A94203D98021490265
:1029D0008C466744290C8C4639000004000C2D04F9
:1029E0002D186144AB4405915946049101990F0497
:1029F0003F0C080C390051434243904602008C467C
:102A0000090C8B4662437C4344445C44A04503D993
:102A10008021490288464244210C884661460904C7
:102A2000090C8C4639005943434370437E430F0CD5
:102A3000F6182404BE19644442448C46B34203D9B8
:102A400080235B0298464044029B61469846049B63
:102A5000370443449B46AB45AD416B420D04059999
:102A60002D0C8C467F196744FD18A8465D462D192C
:102A7000A542A44193466442A446C344DC448F4229
:102A8000BF4198459B4193459241A445A4415B4277
:102A90007F421F43360C52426442BF192243BF1883
:102AA000624638184302D20D039913436A020A435F
:102AB000501E82416146ED0D2A434E023243D90138
:102AC00000D4B3E00126500832400243DE0732430F
:102AD0005B08224C5444002C62DD510709D00F20C2
:102AE0001040042805D0101D9042924152429B187C
:102AF0000200D90104D580241948E400034054445D
:102B00001848844200DD27E75E075B02D2081F0BEE
:102B1000630516435B0DB2E6002399460133042793
:102B200000269B4664E60323019781460C279B46BB
:102B30005EE6012201201743002276E603230320EC
:102B40001F43434671E6C046FF07000001FCFFFF3C
:102B500094C90110FFFF0F800DFCFFFFFF03000071
:102B6000FFFFFFFEFE0700000023802700933F03C6
:102B70000026434B83E6019B3200A446584670E68C
:102B8000AC466EE6802701993F0339422DD03B4287
:102B90002BD11F433F033F0B00951600384B6EE6C9
:102BA00001252D1B382D00DD66E61F2D40DC354844
:102BB0001C005044160082408440EE40501E82416A
:102BC00034431443EB40620709D00F222240042A09
:102BD00005D02200141D9442804140421B181A0265
:102BE0003ED501230027002649E68027019B3F03AD
:102BF0001F433F033F0B0094214B40E603005A461E
:102C0000283B9A40002601926DE65846FDF73CFEAF
:102C1000203057E603005246283B9A40130000221A
:102C200093E65046FDF730FE20307BE6CA4650E77B
:102C30001F201E004042041BE640202D03D0124CF2
:102C40005444A3401A43501E8241324307260027B2
:102C5000164009D00F200023104014000428B9D1D9
:102C600022005E075B021F0BD2081643002306E614
:102C700080273F031F433F033F0B1600004BFEE539
:102C8000FF0700001E0400003E040000F8B5574690
:102C90004E464546DE460C000903E0B5490A460F9C
:102CA0005F0031431E03DB0F760A9B46530F33430D
:102CB000C84E6500C000E40FD2006D0DA2468146EB
:102CC0007F0D9C469046B74200D1B9E05B46012695
:102CD00073409B46EE1BA34500D183E0002E63DDCD
:102CE000002F00D0B1E06346134300D123E1731EEF
:102CF000002B00D0BAE1861A6346B042804101251C
:102D0000C91A4042091A0B0200D447E149024B0A92
:102D100098464346002B00D189E14046FDF7B4FDBB
:102D20000300083B1F2B00DD7CE120223000D21A7B
:102D30004146D040994002009E400A439D4200DD3A
:102D40006AE15D1B6B1C1F2B00DD94E1202110004C
:102D50003500C91A8E40DA408840DD40711E8E4130
:102D6000110007222843002506433240002A09D0DB
:102D70000F233340042B05D0331DB342B6417642B6
:102D800089191E000B0200D43DE26A1C914B5505C7
:102D90006D0D9A4200D119E18F4AF6080A40570793
:102DA00052023743120B9BE0002E00D0C5E06E1C90
:102DB0007605760D012E00DC48E16746861ACB1BAE
:102DC000B042BF417F42B8461F004346FF1A3B0056
:102DD000B8461B0200D55FE137439AD10022002498
:102DE000002579E0002E00DCFAE0002F00D18DE014
:102DF000784B9D4267D0802367461B041F43BC4627
:102E0000382E00DC52E1634613435A1E93411E18CC
:102E100086428041404209180B0200D4BEE06D4B4F
:102E200001359D4200D1D2E06B4A73080A4001216E
:102E30000E401E435108D30707221E43324095E738
:102E40001E00164300D045E740E7624B9D423AD052
:102E5000802367461B041F43BC46382E00DDEBE091
:102E60001F2E00DC3AE133006746203BDF403B0089
:102E7000202E05D04027BF1B6646BE4032439046F9
:102E80004646721E96413343DAE0002B00D114E22D
:102E90006346134300D168E180234E07C008C90888
:102EA0001B030643194208D06046C008184204D1EB
:102EB00063460100D2085E071643F3009946C90035
:102EC000720F444D11434B46DE08424B4F073743C8
:102ED000CA089D4200D16EE012036D05120B6D0D04
:102EE00000211203130B0A0D12051A433B4B2D054B
:102EF00013402B435B00E4075B08234338001900B1
:102F00003CBC90469946A246AB46F8BD6346134387
:102F100011D0731E002B00D007E186188642804135
:102F200061444042091801250B0237D502257BE791
:102F30003E00614691463500C5E75C46002D00D055
:102F4000E1E00B000343F3D0731C00D1ACE1214B53
:102F50009F4200D13AE1F343382B00DD6FE11F2B94
:102F600000DD8CE120250E00ED1AAE40B0460600D3
:102F7000AA46DE40454635432E005546D940A84076
:102F80006346451EA8415B1A9C463043161AB2425E
:102F9000924163465242991A3D00B4E607223240FC
:102FA000002A00D0E4E60B4BF6084F073743CA0867
:102FB0009D4200D090E73B00134300D1A6E180235F
:102FC0001B031A431203120B024D89E7150000225E
:102FD000002785E7FF070000FFFF7FFFFFFF0F804F
:102FE000002E00D0C7E06B1C5E05760D012E00DCC4
:102FF000F0E0C84DAB4200D1B9E085180A00854227
:1030000089416244494251180722CE076D082E4378
:10301000490832401D00A9E6BF49ED1A11400722B8
:103020003240A3E6320028388240002686E630008F
:10303000FDF72AFC203073E6634613435A1E934182
:10304000C61AB04280414042091A5CE60E0067464B
:1030500006431743002D5ED1002E00D0F3E0002F71
:1030600000D11EE15C46614691462CE7A94FBE4265
:103070007BD01E00F1E610001F3DE840202B03D05E
:103080004021CB1A9A401643731E9E4107220643E5
:1030900032400021002583E7161A6346B242804180
:1030A000591A40420B1A98465C4632E61F2E00DD44
:1030B000ABE02027BB1B9A4663465746BB40994668
:1030C00013004F46F3401F433B005746BA40571E7C
:1030D000BA4113436246F240891898E62027BB1B89
:1030E0009A4663465746BB40994613004F46F34005
:1030F0001F433B005746BA40571EBA41134362462E
:10310000F240891A9CE7834B9F425FD080252D04B3
:103110007342294320E7002E0CD1002F00D1D0E0CC
:103120005C46614691467B4DCDE67A4FBE421CD04F
:103130001E0065E6002F18D0C0084E070643802009
:10314000C9080003014208D06346DC08044204D1E8
:103150002100DA46D2085E071643F300994601249F
:103160005346C900720F11431C406A4DABE61D0067
:1031700000220027B4E6002D59D10B00034300D1F3
:10318000D6E6731C00D1B2E0624B9F421ED0F343DF
:10319000382B6FDC1F2B00DD97E020250E00ED1A89
:1031A000AE40B0460600AA46DE40454635432E00F6
:1031B0005546A840D940451EA8418C440643B61840
:1031C00096429241514261443D0025E63D006146F0
:1031D000914678E60B000343002D00D055E6002B06
:1031E000F5D06346134300D16DE6861886428041D0
:1031F00061444042091800220B0200D4D0E6464B3D
:1032000001351940B2E5B1465DE633006746203B23
:10321000DF403B00202E05D04027BF1B6646BE4046
:10322000324390464646721E96413343EFE5394B92
:103230009F42CBD080252D0473422943A8E7084341
:10324000411E8841A2E6002F00D13CE66346861A63
:10325000CF1AB0429B415B42FB1A98461B024ED5E7
:10326000161A6346B2429241591A5242891A5C4672
:1032700000227BE501430E00711E8E419FE71D0079
:103280000E00203DEE40B046202B04D04025EB1A26
:1032900099400843814648464346411E88411843A9
:1032A00074E60022002417E6161A6346B2429241E1
:1032B000591A5242891A3D0025E561469146154D3D
:1032C00001E680220024120379E61D000E00203D55
:1032D000EE40B046202B04D04025EB1A994008431D
:1032E00081464E464346711E8E411E4367E786184F
:1032F00096429B4161445B42C9183D008CE54746BC
:103300003743CED007224146324049E600273A00F3
:10331000E6E5C046FF070000FFFF7FFF70B50C4EDB
:103320000D031C0349005B002D0B490D240B5B0DA5
:10333000B14208D0064900208B4203D1144320003B
:10334000441EA04170BD05430120002DFAD1F1E7D4
:10335000FF07000030B5144D0A034B00120B5B0D44
:10336000C90F0024AB4211DD104CA34210DC8024B5
:10337000640322430E4CE41A1F2C0CDD0D48C31AC3
:10338000DA4013005C42002900D11C00200030BD4F
:10339000094BCC18FAE7094DE040AC4663449A402B
:1033A00013000343EEE7C046FE0300001D040000C7
:1033B0003304000013040000FFFFFF7FEDFBFFFF5D
:1033C00070B500282DD0C317C5185D40C40F280064
:1033D000FDF75AFA154B1B1A5B055B0D0A2815DD24
:1033E0000B38854000222D032D0B002110002D03EA
:1033F0000A0D2D0B12052A430D4D1B052A401343C0
:103400005B00E4075B082343190070BD020029003C
:10341000153291400A000B21081AC5402D032D0BCF
:10342000E3E70024002300250022DEE71E0400005D
:10343000FFFF0F8010B5041E25D0FDF725FA144BB1
:103440001B1A5B055B0D0A2812DD0B388440002235
:103450002403240B0021100024030A0D240B120561
:1034600022430C4C1B05224013435B00590810BD3E
:1034700002002100153291400A000B21081AC440B5
:103480002403240BE6E7002300240022E2E7C046E1
:103490001E040000FFFF0F804100090E4B1C70B599
:1034A000DBB24602750AC40F012B14DDE0239B003A
:1034B0006D07360BCB1800210A0D280012051C4D94
:1034C00032435B052A405B0813435B00E4075B085B
:1034D0002343190070BD002914D1002D1ED02800EF
:1034E000FDF7D2F90A281CDC0B232A001B1ADA404C
:1034F000030015339D400F4B12031B1A5B05160B7F
:103500005B0DD8E7002D06D0320B802636036D0701
:103510001643094BCFE7084B0026CCE700230026D3
:10352000C9E703002A000B3B9A400025E3E7C046A9
:10353000FFFF0F8089030000FF070000F0B54C007B
:10354000640D0B03621C5B0A460F5205C90F1E4334
:10355000C500520D012A29DD374BE718FE2F1CDC70
:10356000002F3BDD8001431E98410722F3006D0FC1
:1035700003432B431A40002A04D00F221A40042A86
:1035800000D004338022D2041A4024D00137FAB28A
:10359000FF2F02D09B01580A01E0FF2200204002C9
:1035A000D205400AC90710430843F0BD3543002C3B
:1035B00004D1002D0AD100220020F0E7002DECD02C
:1035C0008020C0033043FF22E9E7002400235B0290
:1035D000580AE2B2E3E7DB083C00F8E73B001733A8
:1035E000F3DB80231B0433431E26F61B1F2E14DD42
:1035F00002225242D71B1A00FA401700202E04D094
:103600000E4A94466444A3401D432B005D1EAB410B
:1036100007223B431A400027ADE7094A2800A218B9
:10362000954093406C1EA541F04007222B43034375
:103630001A4000279FE7C04680FCFFFFA2FCFFFF67
:1036400082FCFFFF10B5002903D1FDF71DF92030E2
:1036500002E0081CFDF718F910BDC046F0B54E4653
:103660005746DE464546E0B50F00002183B0060010
:103670008946002F06DA3900002746428F41012192
:1036800049428946002B07DA4946C943100089465A
:103690001900002342428B4134003D009246984677
:1036A000BB4269D866D041465046FFF7CBFF834600
:1036B00039003000FFF7C6FF5B461B1A9C46203BD3
:1036C0009B4600D575E05146584681400B00514657
:1036D000604681400A00BB4261D85ED034003D00A4
:1036E0005946A41A9D41002900DA7AE00021002001
:1036F00001260090019159468E40019661460126AF
:103700008E4061460096002950D0D90756085F08C0
:103710000E4363460EE0AF4201D1A6420CD8A41B73
:10372000BD41012124196D410022013B641855411E
:10373000002B06D0AF42EED9013B24196D41002B7E
:10374000F8D1009801995B4600196941002B3DDBD7
:103750002E00DE4063462C00DC405B46002B4BDB3A
:1037600034005D46AC4023006446A6403200801A17
:10377000994103E0B24296D9002000214B46002B2C
:1037800004D003000C0000215842A14103B03CBC0E
:1037900090469946A246AB46F0BDB1429ED9002163
:1037A00000200090019161460029AED10098019956
:1037B000E4E72023624651469B1AD94040460091D7
:1037C00061468840030000990B4380E7624620234E
:1037D0009B1A2A009A40260013006246D6401E43D8
:1037E000B8E7614620260127761A00200021F7401D
:1037F00000900191019781E76746202362463500DA
:10380000BC409B1ADD4023002B43ADE7024670B558
:103810000A4392072AD11E4DEE0104C808C9541B61
:103820009443344017D0D0B2D9B2401A2106014394
:1038300010D190B299B2401A210401430AD110026A
:103840001902000A090A401A2102014302D1100E8E
:10385000190E401A70BD9A42DFD010BA19BA8842C8
:1038600001D9012070BD0020C04370BD02780B78E3
:1038700001300131002A09D09A4207D102780B7831
:1038800001300131002A01D09A42EFD0D01A70BD28
:043890000101010130
:1038940070B5040010F0B4F9074BE6009B191A68E0
:1038A4005B6812184B41054D2000AD192A606B600E
:1038B40010F02EFA70BDC0462010002040100020E9
:1038C40070B5FFF7E5FFFE21074C89052068FDF779
:1038D4005BF90649051CFCF7CBFF002801D12560E4
:1038E40070BD00232360FBE7C4AA002000C0A847E2
:1038F400F0B589B01E000EAB170000229B5E059048
:1039040006910F981D490793FDF7E2FDFFF7C2FDED
:103914001B4A1C4BFEF746FF04000D0010F042FF4B
:10392400009001912000290010F0EAFF0290039119
:103934000798FDF7C7FF041C00980199FFF7FCFDE9
:10394400211CFDF793FC051C0598FDF7BBFF011C2A
:10395400281CFDF719F9386002980399FFF7ECFD6C
:10396400211CFDF783FC041C0698FDF7ABFF011C2A
:10397400201CFDF709F9306009B0F0BD0000B44225
:0839840011E7FAA146DF913FB3
:10398C00F0B589B0FFF782FD0022564BFEF706FF1B
:10399C000022554BFEF7F8FA0022534BFEF7F4FACF
:1039AC000022524B04000D00FEF7EEFAFFF7C0FDAB
:1039BC00290004902000FFF7BBFD4D4D0590002120
:1039CC00280005F099FB78234A4E4B4C1A0019003D
:1039DC0000962800019404F093F90421280004F0C7
:1039EC009EF8002332001900280004F093F80023FD
:1039FC000126069307933000FFF716FD0022394B82
:103A0C00FEF7CCFE0022394BFEF7BEFAFFF790FD15
:103A1C0078216E2306AA01900093080007ABFFF7EC
:103A2C0063FF80210798C905FDF7AAF8FDF726FF6B
:103A3C0007000698FDF722FF2D4D020031003B00D8
:103A4C002800013605F0C8FF0D2ED4D12B4B0026D3
:103A5C001B78012B01D1F8263602059B78210193A6
:103A6C0055230800009306AA07ABFFF73DFF079B01
:103A7C000296234A234E00930394069B0196111C35
:103A8C00280004F0BDFB1D4B00271B78022B01D135
:103A9C00F8273F02049B782101933C2306AA00934C
:103AAC00080007ABFFF720FF079B154A0394009310
:103ABC00111C069B28000297019604F0A1FB0194AF
:103ACC0078220024110028000094042304F018F933
:103ADC00902322005B002100280004F082FF09B033
:103AEC00F0BDC0460080764000004E4000002840EB
:103AFC0070A50020FFFF0000FFFFFF0054AB00206B
:083B0C000000F0420000C0407F
:103B140070B53C4D2B78BFF35B8F3B4CDB070DD46A
:103B240028000EF055FA002808D008F029FDFA23E1
:103B34009B00C018206028000EF06CFA08F020FDED
:103B44002368984209D908F01BFDFA239B00C0188A
:103B54002E4B20601868FFF717FF2D4C2378002B9D
:103B64001CD0062008F0AAFD00282DD1274D23786B
:103B74002868022B26D12749FDF706F828602E680D
:103B84002549301CFCF774FE002804D02249301C5F
:103B9400FDF79EFC28602868FFF7F6FE082008F071
:103BA4008DFD1E4E051E0BD13378002B08D02378D3
:103BB4000133DBB2032B23D82370642008F0F0FC1C
:103BC400357070BD1649D7E7072008F077FD002847
:103BD400E4D10E4D23782868022B0FD10D49FDF74F
:103BE40077FC28602E680021301CFCF723FE002897
:103BF400D1D00949301CFCF7C7FFCBE70849EEE7F1
:103C04002070DAE7289B002098A30020C4AA002093
:103C140054AB00200000614500C0A84744020020C6
:043C240000007042EA
:103C2800F02270B5124D1100280002F073FB114C00
:103C38002900200004F070FD0F49104A20000EF002
:103C4800B1F9E1200E4B00011B7858430D4B1A784F
:103C58003C235343C0180C4B1B78C018FDF730FEAB
:103C680000220A4B18600A4B1A705A6070BDC04691
:103C7800D4A9002070A500208992001040020020DD
:103C88004FAB002052AB002056AB0020C4AA002046
:043C9800CC950020A7
:103C9C00E12170B5314C4902200006F07BFF022176
:103CAC00062008F0A3FC0221072008F09FFC02214B
:103CBC00082008F09BFCFA20400008F06DFC284915
:103CCC00200008F02FFB274D2878032839D8FE2335
:103CDC0025499B05AB60C300C9180023234A0A6021
:103CEC004B60234969600FF0C1FF2878FFF7CCFDCA
:103CFC002049200008F0F7FA08F03EFC0A220100E7
:103D0C00200008F04DFB1C4C0021200002F0C4FCEC
:103D1C002000002102F048FCF8212000090203F0E9
:103D2C008BFEF122154C11000123200004F080FDC4
:103D3C001349200005F0C8FB124B1868FFF720FE52
:103D4C0070BD1149200008F0D2FA1049200008F08B
:103D5C00DFFA0F49200008F0DBFAD4E7E4990020E1
:103D6C00EAF30110CC950020201000203F420F00F8
:103D7C00C5380010F5F30110D4A9002070A500205F
:103D8C00D4C90110C4AA0020E2F3011016F40110EA
:043D9C002FF40110EF
:043DA0000020704748
:023DA400704766
:023DA600704764
:023DA800704762
:103DAA00030084331B78002B02D0C06F00B2704727
:043DBA00006DFBE7B6
:103DBE00020084321278031D002A02D0D86F00B29E
:063DCE007047406DFBE7A9
:103DD400F7B516002C4D2D4A8265C26510202A00C5
:103DE400EC680442FCD1D024802024064003A06166
:103DF400844607202F684740083007408020400150
:103E0400284307602A27AF60654601941A3FD468A7
:103E14003C42FCD1019C65610C0A94609160190AD2
:103E2400916093601023D1681942FCD1D023802182
:103E34002B241B064903996194601B3CD5682542D9
:103E4400FCD15961330A93609660089B1B0A936006
:103E5400089B93601023D1681942FCD1D0238021A0
:103E64001B06490399612C2393601C3BD1681942BA
:103E7400FCD10F231268934303608022D0235203A2
:103E84001B065A61F7BDC04600C00340FFFF000097
:0E3E940037B5057F04680095A46AA0473EBDBF
:103EA200F7B504000F0015001E00994201DD37002E
:103EB2000E00089B9D4202DD2B00089D089323689B
:103EC20020005B6B9847236801901B6B200098478A
:103ED200019BFC34BB4206DD002E04DBA84202DD5E
:103EE200089B002B0ADA0022A36D22626362A2629F
:103EF200E362236A2363636A6363F7BDFB43DB17F1
:103F02001F40019BB34201DC1E00013EEB43DB1765
:103F12001D40089B984201DC431E0893276265629C
:063F2200A662089BE4E723
:0E3F280037B5057F04680095A46AA0473EBD2A
:103F380030B515000A4B84101D400B405B1B6343D2
:103F4800FC24E40022402140891A48439B09054982
:103F5800000A5B1980180B402040184380B230BD1E
:083F68001FF800001FF8FFFF25
:103F700070B516000A4D0B4B2E400B409B1B841056
:103F80006343FC24E40022402140891A48439B09F2
:103F9000000A9B1980182B402040184380B270BD46
:083FA0001FF8FFFF1FF80000ED
:023FA800704760
:103FAC00030037B585331B78002B00D089E0040063
:103FBC00FF34647E002C00D183E0446F0919446EF9
:103FCC00A14200DA7DE0846F1219846EA24200DAFD
:103FDC0077E0C46EA14200DB73E0046FA24200DB09
:103FEC006FE00400F43425780834102D09D1E36C0B
:103FFC00F8305A43036851184900C85A40BA80B285
:10400C0020E0082D1FD1E06C4243206841188A5CE7
:10401C001800002A16D0C0212B4B490101935301E3
:10402C000B40E021500940031843C90093010B4099
:10403C00E0211843D3000B40DD390A4001A90343AA
:10404C00885C18433EBD042D12D1636D994238DA59
:10405C00E36C20695A436368521852109B5CCA0780
:10406C0003D41B115B00185AECE70F221340F9E73D
:10407C00C37F012B12D1A36D9B1A8AB2591EE36D1B
:10408C00F0305A4323685218D2109B5C072211401F
:10409C008B4000681B0612D54069B0E7022B06D195
:1040AC00636D591AA36D01399A1A013AE7E7032B8C
:1040BC00E5D1636D89B25B1A11005A1EDFE7806986
:1040CC009DE70248BEE7C046000B151FFFFF00002E
:1040DC00020070B5FF32527E0B00002A20D0020085
:1040EC000400F4321578FC34216B626B102D18D15E
:1040FC00E56CF8306A435118026849005BBA8B5280
:10410C00236BA26A01332363934209DD236AE26ABB
:10411C002363636B01336363934201DD636A6363FF
:10412C0070BD082D0FD11C26E06C1735424320685A
:10413C0041181812A8439D113540DB0628439B0FEC
:10414C0003438B54DCE7042D13D1E06C0B35424355
:10415C0060685218521082182B401078C90704D48A
:10416C001B01284018431070CAE7A843034313707F
:0A417C00C6E705682D69A847C2E7F1
:10418600020003000020FF32527E82420BD019004B
:104196001A00F431097884321278012904D982424E
:1041A6000CD0D86F00B27047D97FC90704D5002A52
:1041B600F7D1FC33986DF5E7002AF2D1FC33586D40
:0241C600F0E720
:1041C800020003000020FF32527E82420CD0190008
:1041D8001A00F431097884321278012905D982420B
:1041E8000DD00433D86F00B27047D97FC90704D502
:1041F800002AF6D1FC33586DF5E7002AF1D1FC33DB
:04420800986DF0E7D6
:10420C0030B50400FF34647E002C24D004008534C7
:10421C002478002C1FD1446F0919446EA1421ADB7B
:10422C00846F1219846EA24215DBC46EA14212DA9D
:10423C00046FA2420FDA0400F43425780834102DF0
:10424C000AD1E46CF8306243006851181A0A1B0258
:10425C00490013430B5230BD082D0FD1E06C1435BF
:10426C00424320681F244118180AA0439C092C4083
:10427C00DB0620439B0F03438B54ECE7042D13D137
:10428C000F20E56C64686A4352185210A218034060
:10429C001478C90704D41B0104401C431470DAE7DA
:1042AC00844323431370D6E7C07F012815D1606D7A
:1042BC00801A8AB2411EE06D4243206807245218CE
:1042CC00D2102140793482180C41002061B2105672
:1042DC00002B13D008431070BDE7022806D1606D87
:1042EC00411AA06D0139821A013AE4E70328E2D1A0
:1042FC00A06D89B2401A1100421EDCE78843EAE740
:10430C00F7B500910100FF31497E0400089D00299A
:10431C0000D184E001008531097800297FD1416FFB
:10432C0000984018616E884279DBE16E884276DA3B
:10433C00A76F216FD2198A4271DAA66EB24202DAE5
:10434C00921B9B183200D618B14200DA8B1A002B44
:10435C0065DD2100F4310978102910D1290A2D02CC
:10436C000D432100FC31C96CF8344A4312184E003D
:10437C005200013B53D321688D529219F9E7082959
:10438C0014D1E0261C27290A3140AE093E40ED0627
:10439C003143AD0F0D43D318FC349A423FD0E16C3E
:1043AC0026685143361875540132F6E7042926D194
:1043BC00D318C10712D4F0210F262D010D40FC3467
:1043CC009A422CD0E16C676851430918491079184E
:1043DC000F78013237402F430F70F1E70F26FC3472
:1043EC0035409A421BD0E16C67685143091849105B
:1043FC0079180F780132B7432F430F70F1E7D21BB6
:10440C00D3180193019B9A4209D0531C1E002368B8
:10441C0000991F6920002B00B8473200F2E7F7BD66
:10442C00F0B591B0039218AA167802000291853269
:10443C0017780400002F5FD17A32527E002A5BD0AD
:10444C001F2B59D90200B4321268002A00D0B0E0F8
:10445C00406FE26E121A91424EDAA16F226F039DE9
:10446C00521A954248DA06227243029D5219656E21
:10447C00281A824240DD0398F2001218A06E411AED
:10448C008A4239DD0522012E3AD1169917988142BC
:10449C0036D000215343A14A0EA89B185A5C0A54EB
:1044AC0001310529FAD10023039F43713B000833E6
:1044BC00049300230393029B039A991823681B69A6
:1044CC001D000EABD35C334218D0169B3A00200073
:1044DC00A847039B01330393052BECD1029B3A00B5
:1044EC00591D236820001D69179BA847049B760063
:1044FC000137F6B2BB42DCD111B0F0BD179BE5E73A
:10450C005A43029B089206930023059300230493BD
:10451C00059B052B05D0089A804BD318059A9B5CFC
:10452C000493012E22D1039D2B0008330793012302
:10453C00049A1A4209D0029B059A20009918236804
:10454C002A001B691F00169BB847049B01355B08AA
:10455C000493079BAB42EAD1059B01330593069B61
:10456C009B190693059B062BD0D1C5E70825039B09
:10457C0007930123049A1A4215D02368169A0192C4
:10458C0000965B6A079A1F00069933002000B84713
:10459C00049B013D5B080493079BEDB29B190793A9
:1045AC00002DE6D1D8E7169B179A9342F0D02368DA
:1045BC00E5E711898B429FD3508998429CD35B1AB3
:1045CC000C219BB24B435168656F5B1819790691AE
:1045DC000721595606988C467043029961440791FD
:1045EC004018616E491B884200DC85E7082103985E
:1045FC0059565D79059109183000684304914118AA
:10460C000891A06EA16F401A01000898884200DC46
:10461C0072E712681B880D920893012E2FD96346FE
:10462C001BB209936B461427DF5F7743039BFB1880
:10463C0000270593049B0B97EB180C93049B0C9A87
:10464C00934200D158E7002303936A460699127BE4
:10465C0091423BD9002F07D108990D9A8037525CB3
:10466C000B920A00013208920B9A3A400A9208D037
:10467C0001339BB2039A7F0801320392E5E7099755
:10468C00D3E7002BF6D02268012E0CD103980799A2
:10469C0009181698C91A0090126A20001500049A7D
:1046AC00A8470A9BE6E71800039D0999704349192E
:1046BC00C91A7143029B0096C918169B0193536A41
:1046CC00059A1D0003002000A847EAE7002B0CD038
:1046DC002268012E10D10698079909181698C91A44
:1046EC000090156A2000049AA847049B0133049398
:1046FC00059B9B190593A1E71800069D099970432A
:10470C004919C91A7143029B0096C918169B01934B
:10471C00556A0300059A2000A847E6E70A20021014
:10472C00F0B505001C002B00FF335B7E89B0080040
:10473C0016000E99002B65D02B0085331B78002BAF
:10474C0060D18A1AD317D2185A40231ADF17DB19F3
:10475C007B409C469A4205DC0F0021003C00370050
:10476C00060038008E4205DC2700040038000F00DC
:10477C0031003E00771A0697071BFB17FF185F40A6
:10478C000797771A7B10012703930597A04202DC49
:10479C0001204042059004910023624534DD049AC7
:1047AC00964225DB0398079A0133821A039212D59D
:1047BC000398069A821803922A68012B0FD1136969
:1047CC0028001F000A000F9B2100B847059BE41826
:1047DC00049B591C0023049A01320492DFE70F98C2
:1047EC000090D269280017000A002100B847EDE7B5
:1047FC00002B07D00F982A680090D6690A00210078
:10480C002800B04709B0F0BD049A964223DB039808
:10481C00079A0133821A039211D50398069A8218CB
:10482C0003922A68012B0ED1136928001F00220065
:10483C000F9BB847059BE418049B591C0023049A52
:10484C0001320492E0E70F980090126A28001700DA
:10485C002200B847EEE7002BD4D00F982A680090BE
:06486C00166A2200CCE7F1
:1048740001230D4A443010B5102103701300D06891
:104884000842FCD10422D968114201D09968FAE7A0
:1048940001221A62D02380221B0692035A61034824
:1048A40005F0FBFD10BDC04600C0034094A90020E4
:1048B400030010B545331B78002B06D103004433A5
:0C48C4001B78002B01D1FFF7D3FF10BDC3
:1048D000F7B51E0003000192FF335B7E0500002B3D
:1048E00053D0030085331B78002B4ED11300826F09
:1048F0009446826E63440093934246DB436FC26EDC
:10490000CC18944241DA0099006F81423DDA6F6E13
:10491000BC4202DAE41B36193C00A1198A4200DAD3
:10492000161B002E31DD2A00F4321278102A13D122
:104930002800089B089A1B0A110219433619FC30FB
:10494000F835B44221D0C36C009A53432A681B192E
:104950005B0099520134F4E7082A17D1089B1432FE
:10496000190AE0231940089BFC359B0913403200CB
:104970001943089B0098DB069B0F1943EB6C5843C7
:1049800004192868001912F05FFEF7BD042A2DD122
:10499000E2070AD5E11A2B68019A1F692800089BD3
:1049A000013EB847002EF0D00134A319DB070ED525
:1049B000009BAA6F28009A1A6B6FE11A2B6889195D
:1049C0001F690139089B013EB847002EDDD00F2139
:1049D000089BFC3519400B0119430098EB6C7210D1
:1049E00058430419686864100019CCE7E11A8F195C
:1049F000B942CAD02B684C1C1E69019A089B28003A
:064A0000B0472100F4E7BD
:104A0600F0B51F000300FF335B7E89B004000E0083
:104A1600002B00D165E1030085331B78002B00D005
:104A26005FE1436FC06E9C4666440196864200DB9A
:104A360057E1A56F53190293029A236F9A4200DB3E
:104A46004FE1626E964202DAB61ABF190192A66E5D
:104A5600029AB24204DA0E99921B8A180E920296B4
:104A6600019AD219904201DA019A871A029A0E998E
:104A76005218934202DA029A9B1A0E93002F00DC18
:104A86002FE10E9B002B00DC2BE12600FC36029A60
:104A9600F36C5343019A9B1803932300F4331B785A
:104AA600102B26D121003A000F9BF8311D0A1B025C
:104AB6001D43039B5B000193013A16D20E9B7F00B8
:104AC6005D1E013D00D20CE1F26C039B94466344EB
:104AD60003932300F8331968039B3A005800019B9F
:104AE6000818C91812F01BFDEBE70868C552023317
:104AF600E2E7082B1FD10F9B1C221D0AE0231D4055
:104B06000F9B9B0913401D430F9BDB069B0F1D4309
:104B16000E9B5A1E0E9200D2E3E02600FC36336846
:104B2600039A290098183A0012F08BFD039AF36C49
:104B3600D3180393ECE7042B00D0B2E00F260F9BAB
:104B4600019933400593059A1B011A4304920123E8
:104B56003A001A4019423CD1039B5D10002A11D13C
:104B66007F100E9B5A1E0E9200D2BAE02600FC362B
:104B760073683A005819049912F063FDF36C5B10E0
:104B8600ED18EEE77B1E5B1003930E9B5A1E0E92EA
:104B960000D2A6E0012F07D02300FC335868039A01
:104BA6004019049912F04DFD0E9B029A20009A18A6
:104BB600A36FD21A019BD919636F0139C91A2368E9
:104BC6001E69059BB0472300FC33DB6C5B10ED18B8
:104BD600DBE7039D01356D10002A27D07B1E5B1095
:104BE600039305960E9B5A1E0E927AD30E9B029A3B
:104BF600616F9A18A36F0598D21A019B591A2368F8
:104C06001B691E000F9B03402000B047012F07D0F1
:104C16002300FC335868039A4019049912F011FDD9
:104C26002300FC33DB6C5B10ED18DBE7BB1E5B106F
:104C3600069307960E9B5A1E0E9252D3029A0E9B0D
:104C4600616F9B180593079A0F9B200013400393EF
:104C5600059AA36FD21A019B591A23681B691E0075
:104C6600039BB047012F16D0A36F059A2000D21AD6
:104C7600019BD919636F0139C91A23681E69039B01
:104C8600B047022F07D02300FC335868069A401914
:104C9600049912F0D6FC2300FC33DB6C5B10ED1894
:104CA600C8E76246019B9B1A0193029B5D1B0E9B04
:104CB600EB180493049B9D4213D0019B0199DB19C9
:104CC6000293029B8B420AD04B1C039323682A0053
:104CD6001B6920001E000F9BB0470399F1E70135C1
:064CE600E8E709B0F0BD93
:104CEC0007B544300378002B1AD000236A460370B2
:104CFC00137101330B495371019A0B48009105F064
:104D0C00C9FBD02380221B0692039A610723074913
:104D1C000A685340CF221340802252010A43136089
:104D2C0007BDC046C0FC9B0194A9002000C00340F5
:104D3C00F0B595B003931CAB1F780300049102925D
:104D4C00853319780400002900D015E22F331A6836
:104D5C00002A00D02BE1039BFF2B00D90CE2049B13
:104D6C00426F9D18C36E9C469D4200DB04E2826F2D
:104D7C00029B006F9E18864200DBFDE106237B43FD
:104D8C00626E5B19934200DCF6E1A36E0593FB00A7
:104D9C009B191900059B994200DCEDE1012395421A
:104DAC000FDB0621627F514349198C4509DD0599BA
:104DBC008E4206DBD2009219C30FD11782424B41AF
:104DCC00DBB2012F73D11A9A1B998A426FD0002B38
:104DDC006DD1220044321178002918D0137012AA18
:104DEC00CF4913715771139ACE48129105F052FBAB
:104DFC00D02380221B0692039A610723CA490A68B2
:104E0C005340CF221340802252010A431360226880
:104E1C00F11D0091D26B6B1D9446290032002000CD
:104E2C006546A8470522039BC0495A43002312A894
:104E3C005218D15C19540133052BFAD100230822E6
:104E4C0002254371B84B0021465C3E422AD0DE68F5
:104E5C002E42FCD01A9E01319E600529F4D17F00B0
:104E6C00FFB2D9682942FCD01B99013AD2B29960A1
:104E7C00002AE8D1220045321278002A00D07BE1CA
:104E8C0044342278002A00D076E1013222700F32AD
:104E9C00D9681142FCD10422D968114200D161E1D8
:104EAC009968F9E7DE682E42FCD01B9ED3E72300FD
:104EBC00012245331A700523039908925943049B28
:104ECC00099106930023059300230393059B052B5F
:104EDC0005D0099A954BD318059A9B5C0393012F27
:104EEC0042D11A9B1B9A93423ED1029D2B00083350
:104EFC000793089B039A1A4209D0049B059A200039
:104F0C00991823682A001B691E001A9BB047039B43
:104F1C0001355B080393079BAB42EAD1059B013338
:104F2C000593069BDB190693059B062BCCD123001E
:104F3C00220046331B7845321370002B00D01BE146
:104F4C0044342378002B00D016E1774A01332370C8
:104F5C0010211300D0680842FCD10422D9681142F8
:104F6C0000D1FFE09968F9E70825029B0793089B9D
:104F7C00039A1A4215D023681A9A019200975B6A19
:104F8C00079A1E0006993B002000B047039B013D89
:104F9C005B080393079BEDB2DB190793002DE6D159
:104FAC00BCE71A9B1B9A9342F0D02368E5E7138960
:104FBC000398984200D2DFE05089039DA84200D2AA
:104FCC00DAE020000125453005700398C31A0C2047
:104FDC009BB24343506812681B180F921A880992AF
:104FEC001A7906925A79109207229A561B7A0792CE
:104FFC005BB20893AF4233D96B461C229B5E0A937B
:10500C006B4620229B5E0B9300260D960396109BFD
:10501C00039A934200D88BE094460B9B029A63440C
:10502C000E937B439B181193002305936A460699B4
:10503C00127D914244D9002E07D109990F9A8036DE
:10504C00525C0D920A00013209920D9A32400C9278
:10505C0009D001339BB2059A760801320592E5E737
:10506C000B910A91D0E7002BF5D02068012F14D1B9
:10507C000299089A521803995518049A0799891895
:10508C00059A89181A9AC91A0092026A2000944645
:10509C002A006546A8470C9BDDE71A00059D0A9976
:1050AC007A434919C91A7943049B0097C9181A9B6A
:1050BC000193436A20001D001300119AA847EAE7E8
:1050CC00002B12D02068012F14D10299089A049D4C
:1050DC0052180399521807994919069D49191A9D96
:1050EC00C91A0095056A2000A847039B0133DBB25F
:1050FC0003938CE71A007A4394460E9A02997A43EA
:10510C00069D52180A9900974919C91A7943049BAC
:10511C00C9181A9B0193456A63462000A847E4E727
:10512C00C0FC9B0194A9002000C003400A2002107F
:10513C002300220046331B7845321370002B1BD101
:10514C0044342378002B17D10C4A013323701021DF
:10515C001300D0680842FCD10422D968114201D056
:10516C009968FAE701221A62D02380221B06920367
:10517C005A61034805F08DF915B0F0BD00C003402D
:04518C0094A90020C2
:10519000F0B585B00193030085331B780500002B23
:1051A00000D0A4E0406F0F18696E8F4200DA9EE0D5
:1051B000A96F5618AA6E964200DA98E0EA6E9742F6
:1051C00000DB94E02A6F964200DB90E0494A4A4CAB
:1051D000AA65EA652A0044321178002916D01370B6
:1051E00002AA1371013353714449039A444802914E
:1051F00005F056F9D02380221B0692039A610723FB
:1052000022685340CF2213403E4A13601023E268C5
:105210001A42FCD10723226853400F221340394A17
:105220001360EB6D9F4215D0D02380222A211B06EC
:1052300052039A61A1601A39E0680842FCD15A61B0
:105240003B0AA360A760A3601023A760EF65E26834
:105250001A42FCD1AB6D9E4215D0D02380222B2167
:105260001B0652039A61A1601B39E0680842FCD119
:105270005A61330AA360A660A3601023A660AE65DE
:10528000E2681A42FCD1D02380222C211B06520353
:105290009A61A1601C39E0680842FCD15A61019B07
:1052A0001B0AA360019BA3601023E2681A42FCD191
:1052B0002B0045331B78002B19D144352B78002B5C
:1052C00015D101332B700F33E2681A42FCD104234D
:1052D000E2681A4201D0A268FAE701238022236221
:1052E000D02392031B065A61054805F0D8F805B093
:1052F000F0BDC046FFFF000000C00340C0FC9B01A2
:0853000094A9002000D0034035
:1053080010B544300378002B17D10C4A01330370D1
:1053180010211300D0680842FCD10422D968114238
:1053280001D09968FAE701221A62D02380221B066D
:1053380092035A61024805F0AEF810BD00C0034060
:0453480094A9002004
:10534C00020073B54432137805000E001B4C002B81
:10535C0019D0002313706A46137101335371184925
:10536C00019A1848009105F095F8D02380221B066D
:10537C0092039A61072322685340CF221340802264
:10538C005201224313601023E2681A42FCD1042319
:10539C00E2681A4201D0A268FAE701232362DB1803
:1053AC00E2681A42FCD02B00A66045331B78002B18
:1053BC0002D12800FFF7A2FF73BDC04600C0034016
:0853CC00C0FC9B0194A9002024
:1053D400F0B504001D00230085331B7889B0080054
:1053E40016000E99002B00D0B7E0230001224533AC
:1053F4001A708A1BD317D2185A402B1ADF17DB19DD
:105404007B409C469A4205DC0F0029003D00370092
:10541400060038008E4205DC2F00050038000F001E
:1054240031003E00771A0697471BFB17FF185F40B1
:105434000797771A7B10012703930597A84202DC8C
:105444000120404205900491002362454CDD049AFA
:10545400964225DB0398079A0133821A039212D5E8
:105464002268012B13D1136920001F000A000F9B2F
:105474002900B847059B039AED18049B591C069B09
:10548400D31803930023049A01320492DFE70F98A0
:105494000090D269200017000A002900B847E9E704
:1054A400002B07D00F9822680090D6690A002900C3
:1054B4002000B0472300220046331B784532137086
:1054C400002B4AD144342378002B46D1244A01339B
:1054D400237010211300D0680842FCD10422D9683B
:1054E400114230D09968FAE7049A964223DB039874
:1054F400079A0133821A039211D52268012B12D123
:10550400136920001F002A000F9BB847059B039ACC
:10551400ED18049B591C069BD31803930023049A8B
:1055240001320492E0E70F980090126A20001700FD
:105534002A00B847EAE7002BBCD00F9822680090F5
:10554400166A2A00B4E701221A62D02380221B06BD
:1055540092035A61034804F0A0FF09B0F0BDC046AD
:0855640000C0034094A90020DF
:10556C008023010010B5DB050020994212D880235E
:10557C000200DB01994202D99B000132FAE70020BC
:10558C001C188C4201D8091B181949005B08F7D16B
:06559C00D040C0B210BDBA
:1055A200F7B50091111C1C1C151C071CFBF75FFEB4
:1055B200211C061C0098FBF75AFE011C301CFBF74D
:1055C200E4FA291C0190281CFBF751FE211C061C41
:1055D200201CFBF74CFE011C301CFBF7D6FA011C09
:1055E2000198FBF76CFCFE2189050FF07CFA002183
:1055F2000FF063FA061C011C281CFBF738FE011C85
:10560200381CFBF766FF311C051C201CFBF72FFE24
:10561200011C0098FBF75DFF291C041C281CFBF7EA
:1056220026FE211C051C201CFBF721FE011C281C48
:10563200FBF7ABFA0FF08DFA0899041C301CFBF74C
:0A56420016FE211CFBF7A1FAFEBDC5
:10564C00022010B5044B013A04D3DC680442FCD0B0
:0C565C009960F8E710BDC04600C0034094
:10566800F0B51E00030085331B7887B00400002BBB
:105678006AD1436FCB18416E03938B4264DBC16ED2
:105688008B4261DA836FD518036F9D425CDA816EB5
:105698008D4202DA6D1A76190D00AA19934200DAC2
:1056A8005E1B002E50DD270044373B78002B1AD0B4
:1056B800002204AB1A713A70013224495A71059AD2
:1056C8002348049104F0E8FED02380221B069203AD
:1056D8009A6107231F490A685340CF22134080224A
:1056E80052010A431360AB192268013B0093D36B44
:1056F80020009C46039B2A0019006546A8470C9B7E
:10570800200099B232004534FFF79CFF2378002B24
:105718001AD13B78002B17D10E4A01333B70102168
:105728001300D0680842FCD10422D968114201D084
:105738009968FAE701221A62D02380221B06920395
:105748005A61034804F0A7FE07B0F0BDC0FC9B01F6
:0857580094A9002000C00340E9
:10576000F0B51E00030085331B7887B00400002BC2
:105770006BD1836FD318826E0393934265DB436FC3
:10578000CD18C36E9D4260DA039A016F8A425CDADB
:10579000426E954202DAAD1A76191500AA199342A3
:1057A00000DA5E1B002E50DD270044373B78002BCB
:1057B0001AD0002204AB1A713A70013224495A718E
:1057C000059A2448049104F06BFED02380221B0626
:1057D00092039A61072320490A685340CF2213405D
:1057E000802252010A431360039922680091D26B10
:1057F000AB19944620000A00013B29006546A847E2
:105800000C9B200099B232004534FFF71FFF23782C
:10581000002B1AD13B78002B17D10F4A01333B7074
:1058200010211300D0680842FCD10422D96811422B
:1058300001D09968FAE701221A62D02380221B0660
:1058400092035A61034804F02AFE07B0F0BDC04637
:0C585000C0FC9B0194A9002000C0034094
:10585C00F0B51F00030085331B7887B00400002BC4
:10586C007ED1436FC06ECD18854279DAA36FD618FE
:10587C00236F9E4274DA626E954202DAAD1A7F197A
:10588C001500A16E8E4204DA0C9A761A92190E004B
:10589C000C92EA19904200DA471B0C9AB218934208
:1058AC0001DA9B1B0C93002F5ADD0C9B002B57DD50
:1058BC002300443303931B78002B1BD00022039B43
:1058CC0028491A7004AB1A7101325A71059A26488C
:1058DC00049104F0DFFDD02380221B0692039A6111
:1058EC00072322490A685340CF22134080225201D9
:1058FC000A4313600C9A2168B218013A0092CA6BE1
:10590C00EB19944629002000013B32006546A8475C
:10591C000D9B0C9A99B220007A434534FFF790FE08
:10592C002378002B1CD1039B1B78002B18D1039AD6
:10593C00013313700D4A10211300D0680842FCD1BA
:10594C000422D968114201D09968FAE701221A623F
:10595C00D02380221B0692035A61034804F099FD60
:10596C0007B0F0BDC0FC9B0194A9002000C003400F
:10597C00F0B591B0049316AB07921A7803008533F7
:10598C001B7804000D00002B02D0002011B0F0BDDC
:10599C000029FAD0012A25D1427F036802920269BC
:1059AC000192C26800925E69049A0B000799B04795
:1059BC002300B4331A68002A03D10623607F5843AE
:1059CC00E4E713899D42E0D35189A942DDD3ED1A56
:1059DC000C23ADB25D435268637F5519A8795843C7
:1059EC0000B2D3E7203D931EADB2062B01D85F2D3C
:1059FC00CBD8022A2AD1C249AB00CB580593C14B54
:105A0C005B5D069310230A93616F079B8C46A16F15
:105A1C0063448C460893049B607F63440993069B04
:105A2C0008994343656E5B18AB4202DBE66EB142EC
:105A3C0021DB0A99099E41438919A66EB14203DB09
:105A4C000999266FB14216DB069BC8E7D31E052BBE
:105A5C000CD80C215143AC4BA8005E585B1859680C
:105A6C008059495D059006911B7ACCE7002305937C
:105A7C000A930693C8E708990127A94210DBE16E47
:105A8C008B420DDA099BA16E8B4209DB0A9B0999AB
:105A9C004343256F5B18D917EE0FAB427141CFB260
:105AAC00022A00D0B7E1069B22690633DB100B9368
:105ABC00E368934204D0012802D1002F00D127E1E2
:105ACC002300012245331A70002309930A9B099A7B
:105ADC00934200D1F6E02169E3688B420AD0627FE1
:105AEC002068069B019100925343456A049A0799DA
:105AFC002000A847002308930B9A0899637F8A42D9
:105B0C0000D1D3E00A000599555C002D5CD0D6007D
:105B1C006AB2012B5BD1079BF118002A05DA2368C6
:105B2C00049A1F692000E368B84740231D4208D03F
:105B3C00079B049A591C236889191F692000E36884
:105B4C00B84720231D4208D0079B049A991C236850
:105B5C0089191F692000E368B847EB0608D5079B35
:105B6C00049AD91C236889191F692000E368B84777
:105B7C002B0708D5079B049A191D236889191F69DF
:105B8C002000E368B8476B0708D5079B049A591D9A
:105B9C00236889191F692000E368B847AB0708D54B
:105BAC00079B049A991D236889191F692000E368D3
:105BBC00B847EB0708D5079B049AD91D23688919A8
:105BCC001D692000E368A847089B013393E75E43F7
:105BDC0007997718002A08DAE16822680191009386
:105BEC00566A3900049A2000B04740231D4209D060
:105BFC00637FE068226801900093566AF918049A52
:105C0C002000B04720231D420AD0637FE068226841
:105C1C00019059000093566AC919049A2000B047A4
:105C2C00EB060BD50321637FE06859432268019092
:105C3C000093566AC919049A2000B0472B070AD55D
:105C4C00637FE0682268019099000093566AC91935
:105C5C00049A2000B0476B070BD50521637FE068E1
:105C6C005943226801900093566AC919049A20007E
:105C7C00B047AB070BD50621637FE0685943226818
:105C8C0001900093566AC919049A2000B047EB079B
:105C9C009AD50721637FE0685943226801900093ED
:105CAC00556AC919049A2000A8478DE7049AD3189D
:105CBC000B9A04939446099B01330993059B634407
:105CCC00059303E72300220046331B7845321370FB
:105CDC00002B00D0F7E1230044331A78002A00D0BF
:105CEC00F1E101321A70094A10211300D068084200
:105CFC00FCD10422D968114200D1DAE19968F9E7A4
:105D0C0028260210A82D02100825021000C00340FE
:105D1C00230044331A78002A18D01F700EAB587128
:105D2C00D3491F710F9AD3480E9104F0B3FBD023C3
:105D3C0080221B0692039A610723CF490A685340BD
:105D4C00CF221340802252010A431360069A089B0B
:105D5C000A989B18099A21681218013A0092013B83
:105D6C00CD6B2000099A0899A847002302200493C0
:105D7C000A9B049A934233D0059B0B9A9F18069B5F
:105D8C00BD4A059DAF421ED02D78802607951D007B
:105D9C00083D002B15D007990E420DD0D168014259
:105DAC00FCD0E168013B91607608AB42F1D1059BD8
:105DBC00013305932B00E4E7D1680142FCD0216943
:105DCC00F0E71D00F3E7002B05D0AB4BDA6802427D
:105DDC00FCD022699A60049B059701330493C7E7B2
:105DEC00230045331B78002B00D06CE12300443397
:105DFC001A78002A00D066E101321A709E4A1021EE
:105E0C001300D0680842FCD10422D968114200D199
:105E1C004FE19968F9E7230044331A78002A1AD025
:105E2C0000221A700EAB1A71013291495A710F9AF5
:105E3C0090480E9104F02EFBD02380221B06920377
:105E4C009A6107238C490A685340CF221340802261
:105E5C0052010A43136023000122453306991A703C
:105E6C000A9B4B4321690B93E3688B426DD1002F46
:105E7C0000D0A1E0637F1A005A43013BD2B2DBB2DF
:105E8C000D9207930B9BBB4200DCF7E0059B059A38
:105E9C001B78013205925AB2002A53DA7F22134042
:105EAC000133069938000C93FAF752FC079B002B30
:105EBC0036D0667F089B71434643CD18099BF31877
:105ECC0004930C9B0A930A9B013BDBB20A93FF2BB6
:105EDC0023D004980799226809180091D26B079B6C
:105EEC0016005B19020029002000B047079B002B0D
:105EFC001BD1614B0221DA680A42FBD0E2689A603E
:105F0C00637F069A08995A43ED1852189542DADBCA
:105F1C00049A0D00D3180493D5E70C9BFF18B1E736
:105F2C00089B5D18099B1B18CAE70D9B524A013B45
:105F3C00DBB2FF2BE4D00220D1680142FBD0E16838
:105F4C009160F4E70133DBB2E8E7637F012B32D1D8
:105F5C0000230C939F4231D10998069A8446089BE2
:105F6C0021689B180A9A013B6244013A0092CD6B5E
:105F7C00020008992000A8477F250B9B002B00DC12
:105F8C007CE0059B1A7853B2002B0DDA0B9B2A4050
:105F9C0001329B1A0B93E36899B22000FFF750FB78
:105FAC00059B01330593E8E70B9B0132D2B29B1A98
:105FBC000B932369F0E7170000230C930B9B0C9AAF
:105FCC0093425BDD059B1D7801336AB20593E36850
:105FDC00002A36DA9BB209937F2301271D400C98C7
:105FEC000699FAF7B5FB667F0A0031005143079B0F
:105FFC004643C918049B0135F31808930C9BEDB26A
:10600C005B190C930023013DEDB2FF2D21D0013320
:10601C00069E98188642F6DC002F0AD0627F099EF5
:10602C002068019600925343426A20001600089A99
:10603C00B047089A637F0799D318089300231A0076
:10604C00E1E7226992B2099222699A42C7D10027EC
:10605C00C5E7002BB2D0002FB0D0627F099D20681D
:10606C00009201955343456A089A2000A847A5E77A
:10607C00C0FC9B0194A9002000C003402300220017
:10608C0046331B7845321370002B1CD1230044334C
:10609C001A78002A17D101321A700C4A10211300F9
:1060AC00D0680842FCD10422D968114201D0996809
:1060BC00FAE701221A62D02380221B0692035A614E
:1060CC00034804F0E6F9607FBEE4C04600C003401C
:0460DC0094A9002063
:1060E00030B5A5300378002B0CD102240B48013ABF
:1060F00013D30B885BBA9BB2C5682542FCD0836082
:106100000231F4E70224054B013A06D3D868204255
:10611000FCD0088802319860F6E730BD00C003402B
:106120000B4B0C4A1B689B019B1880225204196878
:106130001142FCD110230849CA681A42FCD10F222F
:106140000B689A4380235B010B431A607047C0467B
:0C61500034A500201000005000C00340E7
:10615C00F0B504001500002785B001930AAB04CB01
:10616C0061671B7885670393019B0292C367031DCC
:10617C00DA6780331F705F70036847665B6B8766F6
:10618C000E0098472368E0661B6B20009847206739
:10619C00BE4203DA019B9B193E000193002D03DAEA
:1061AC00029B5B1900250293019B2000F7182368C2
:1061BC005B6B9847874205DD236820005B6B984733
:1061CC00831B0193029B2000EF1823681B6B9847DD
:1061DC00874205DD236820001B6B9847431B029305
:1061EC00019B002B02DD029B002B12DC002363675A
:1061FC00A367236820005B6B98472368E0671B6BE1
:10620C0020009847231DD86701238534237005B0DF
:10621C00F0BD039B002B0CD16367A36723682000A0
:10622C005B6B98472368E0671B6B20009847231D26
:10623C00D867019B6666F618029BA566ED186B463F
:0A624C00E66625671B7B8434E0E75B
:1062560002000023843270B513705370436783675E
:1062660043668366036804005B6B051D98472368D5
:10627600E0661B6B20009847236820675B6B200055
:1062860098472368E0671B6B20009847E86770BD56
:10629600F0B5040085342478059D002C01D000203B
:1062A600F0BD466F0C68A4190C60866F1468A419BB
:1062B6001460466F1C68A4191C602C68866FA619AA
:1062C6002E600C68C76EA446BC42E8DA17683C002C
:1062D600076FBC42E3DA476E1C68BC42DFDB846EA4
:1062E600A642DCDB6446BC4200DA3C000C60846EED
:1062F6001168A14200DA21001160C26E196891424C
:1063060001DD013A1A60036F2A6801209A42C7DD4F
:06631600013B2B60C4E70F
:10631C00F7B5002504002C4B456008330360431C83
:10632C0005724572DD77831DDD77C31D0F00DD77A8
:10633C002900019205641422B83011F07FF9230072
:10634C000126CC335E771D605D609D60DD601D6154
:10635C005D619D611D7720331D60019B2765A764DE
:10636C006365E3642000FFF770FF2300022294337F
:10637C001D605D600C3B1D605D609D6028331D7071
:10638C00FF320E3B1D705E709D70E26122000F4B60
:10639C00A532E36025616361A5611570613A1670E1
:1063AC00557095706232167056709670D570A365E4
:1063BC00E3652300064A9C33256625636563A56364
:1063CC00E56320001A60FEBDD0250210FFFF00001F
:0463DC00D681000066
:1063E00010B50121152006F007F90121152006F04E
:1063F00041F90121142006F0FFF80121142006F0D4
:1064000039F90121162006F0F7F80121162006F0CF
:0464100031F910BD91
:10641400F0B5050085B0019144352B7806002C4F6A
:106424002C4C002B16D0002302AA13712B700133BD
:1064340053712949039A2948029104F02FF8D02373
:1064440080221B0692039A61072322685340CF22BD
:1064540013403B60D02380221B0652039A61102311
:10646400E2681A42FCD10723226853400F221340EA
:106474003B60019BA3601023E2681A42FCD10F2306
:106484002268453693433B608022D02352031B0687
:106494005A613378002B18D12B78002B15D1013396
:1064A4002B700F33E2681A42FCD10423E2681A42CB
:1064B40001D0A268FAE7012380222362D023920349
:1064C4001B065A61054803F0E8FF05B0F0BDC0465D
:1064D40000D0034000C00340C0FC9B0194A90020ED
:1064E400F0B5050085B0019144352B7806002C4F9A
:1064F4002C4C002B16D0002302AA13712B700133ED
:1065040053712949039A2948029103F0C7FFD02304
:1065140080221B0692039A61072322685340CF22EC
:1065240013403B60D02380221B0652035A61102380
:10653400E2681A42FCD10723226853400F22134019
:106544003B60019BA3601023E2681A42FCD10F2335
:106554002268453693433B608022D02392031B0676
:106564009A613378002B18D12B78002B15D1013385
:106574002B700F33E2681A42FCD10423E2681A42FA
:1065840001D0A268FAE7012380222362D023920378
:106594001B065A61054803F080FF05B0F0BDC046F4
:1065A40000D0034000C00340C0FC9B0194A900201C
:1065B40073B5050044352B7804000E00002B1AD067
:1065C40000236A462B701371013331495371019AC8
:1065D4003048009103F062FFD02380221B0692030F
:1065E4009A6107232C490A685340CF221340802222
:1065F40052010A43136003231E402000E67736212C
:10660400FFF706FFE07F03280BD8F9F72BFF0223DF
:106614002B2D08212000FFF763FFA36C2365E36C97
:1066240063650A2005F0C0FF230045331B78002B67
:1066340026D12B78002B23D1174A01332B7010213C
:106644001300D0680842FCD10422D96811420DD04D
:106654009968FAE768212000FFF742FFE36C23659D
:10666400A36CDDE7C821D5E7A821F4E701221A626B
:10667400D02380221B0692035A61064803F00DFFC3
:10668400064B2000A365E365FFF7E3FD73BDC04639
:10669400C0FC9B0194A9002000C00340FFFF000040
:1066A4000300F0B50700A63385B001931B780400FE
:1066B4004537002B42D0FFF791FE194803F01FFF26
:1066C40023000026012546331E70023B3E7029003C
:1066D4001D701520009305F08DFF2900152005F08D
:1066E400C7FF2900142005F085FF2900142005F0B8
:1066F400BFFF019B1E703B78B3421FD1009B1B78E8
:10670400B3421BD1009B074A1D7010211300D068AF
:106714000842FCD10422D968114205D09968FAE7ED
:1067240094A9002000C0034001221A62D0238022D1
:106734001B0692035A61204803F0AFFE2500012195
:10674400162005F057FF00212000FFF761FE01210C
:10675400162005F08DFF052005F022FF00211620EC
:1067640005F086FF142005F01BFF0121162005F01B
:106774007FFF4435962005F013FF2B78002B21D0A2
:10678400002302AA13712B7001330C495371039A2D
:106794000948029103F082FED02380221B06920353
:1067A4009A61072306490A685340CF221340802286
:1067B40052010A43136005E094A90020C0FC9B0128
:1067C40000C00340EF212000FFF722FEEB21200050
:1067D400FFF71EFE14212000FFF782FEFE21200099
:1067E400FFF716FEEF212000FFF712FEEB21200039
:1067F400FFF70EFE14212000FFF772FE8421200013
:10680400FFF706FE40212000FFF76AFE85212000E5
:10681400FFF7FEFDFF212000FFF762FE8621200026
:10682400FFF7F6FDFF212000FFF75AFE8721200025
:10683400FFF7EEFDFF212000FFF752FE8821200024
:10684400FFF7E6FD0A212000FFF74AFE8921200018
:10685400FFF7DEFD21212000FFF742FE8A21200000
:10686400FFF7D6FD00212000FFF73AFE8B21200020
:10687400FFF7CEFD80212000FFF732FE8C2120009F
:10688400FFF7C6FD01212000FFF72AFE8D2120001D
:10689400FFF7BEFD01212000FFF722FE8E2120001C
:1068A400FFF7B6FDFF212000FFF71AFE8F2120001D
:1068B400FFF7AEFDFF212000FFF712FEB6212000F6
:1068C400FFF7A6FD00212000FFF70AFE202120008B
:1068D400FFF706FE3A212000FFF79AFD052120006C
:1068E400FFF7FEFD90212000FFF792FD0821200014
:1068F400FFF7F6FD08212000FFF7F2FD0821200034
:10690400FFF7EEFD08212000FFF7EAFDBD2120007E
:10691400FFF77EFD06212000FFF7E2FDBC212000E9
:10692400FFF776FD00212000FFF7DAFDFF212000AC
:10693400FFF76EFD60212000FFF7D2FD012120004A
:10694400FFF7CEFD04212000FFF7CAFDC32120007C
:10695400FFF75EFD13212000FFF7C2FDC4212000D4
:10696400FFF756FD13212000FFF7BAFDC9212000CF
:10697400FFF74EFD22212000FFF7B2FDBE212000CB
:10698400FFF746FD11212000FFF7AAFDE1212000B9
:10699400FFF73EFD10212000FFF7A2FD0E2120008D
:1069A400FFF79EFDDF212000FFF732FD21212000AB
:1069B400FFF796FD0C212000FFF792FD0221200035
:1069C400FFF78EFDF0212000FFF722FD4521200076
:1069D400FFF786FD09212000FFF782FD0821200032
:1069E400FFF77EFD08212000FFF77AFD2621200015
:1069F400FFF776FD2A212000FFF772FDF121200028
:106A0400FFF706FD43212000FFF76AFD70212000F7
:106A1400FFF766FD72212000FFF762FD362120009A
:106A2400FFF75EFD37212000FFF75AFD6F2120009C
:106A3400FFF756FDF2212000FFF7EAFC4521200074
:106A4400FFF74EFD09212000FFF74AFD0821200031
:106A5400FFF746FD08212000FFF742FD2621200014
:106A6400FFF73EFD2A212000FFF73AFDF321200025
:106A7400FFF7CEFC43212000FFF732FD70212000F8
:106A8400FFF72EFD72212000FFF72AFD362120009A
:106A9400FFF726FD37212000FFF722FD6F2120009C
:106AA400FFF71EFDED212000FFF7B2FC1B212000A3
:106AB400FFF716FD0B212000FFF712FDAE21200089
:106AC400FFF7A6FC77212000FFF70AFDCD21200067
:106AD400FFF79EFC63212000FFF702FD70212000D8
:106AE400FFF796FC07212000FFF7FAFC072120009E
:106AF400FFF7F6FC04212000FFF7F2FC0E21200032
:106B0400FFF7EEFC0F212000FFF7EAFC092120002B
:106B1400FFF7E6FC07212000FFF7E2FC0821200034
:106B2400FFF7DEFC03212000FFF7DAFCE821200058
:106B3400FFF76EFC34212000FFF7D2FC6221200015
:106B4400FFF766FC18212000FFF7CAFC0D21200086
:106B5400FFF7C6FC71212000FFF7C2FCED212000E5
:106B6400FFF7BEFC70212000FFF7BAFC7021200063
:106B7400FFF7B6FC18212000FFF7B2FC0F2120001C
:106B8400FFF7AEFC71212000FFF7AAFCEF212000E3
:106B9400FFF7A6FC70212000FFF7A2FC7021200063
:106BA400FFF79EFC63212000FFF732FC1821200030
:106BB400FFF796FC11212000FFF792FC71212000C1
:106BC400FFF78EFCF1212000FFF78AFC70212000E2
:106BD400FFF786FC70212000FFF782FC18212000BB
:106BE400FFF77EFC13212000FFF77AFC71212000BF
:106BF400FFF776FCF3212000FFF772FC70212000E0
:106C0400FFF76EFC70212000FFF76AFC642120006E
:106C1400FFF7FEFB28212000FFF762FC292120005A
:106C2400FFF75EFCF1212000FFF75AFC0121200050
:106C3400FFF756FCF1212000FFF752FC0021200051
:106C4400FFF74EFC07212000FFF74AFC66212000D5
:106C5400FFF7DEFB3C212000FFF742FC002120006F
:106C6400FFF73EFCCD212000FFF73AFC672120000E
:106C7400FFF736FC45212000FFF732FC45212000B8
:106C8400FFF72EFC10212000FFF72AFC0021200032
:106C9400FFF726FC00212000FFF722FC0021200042
:106CA400FFF71EFC67212000FFF7B2FB0021200044
:106CB400FFF716FC3C212000FFF712FC0021200006
:106CC400FFF70EFC00212000FFF70AFC0021200042
:106CD400FFF706FC01212000FFF702FC54212000ED
:106CE400FFF7FEFB10212000FFF7FAFB3221200002
:106CF400FFF7F6FB98212000FFF7F2FB7421200038
:106D0400FFF786FB10212000FFF7EAFB8521200016
:106D1400FFF7E6FB80212000FFF7E2FB00212000C3
:106D2400FFF7DEFB00212000FFF7DAFB4E212000F5
:106D3400FFF7D6FB00212000FFF7D2FB98212000AB
:106D4400FFF766FB3E212000FFF7CAFB0721200066
:106D5400FFF7C6FB35212000FFF75AFB2121200055
:106D6400FFF756FB11212000FFF752FB782005F0B6
:106D740017FC29212000FFF74BFB142005F010FC21
:106D84003B78002B1AD12B78002B17D1124A0133F0
:106D94002B7010211300D0680842FCD10422D9685A
:106DA400114201D09968FAE701221A62D0238022A5
:106DB4001B0692035A61094803F06FFBE17F200030
:106DC400FFF7F6FB0121002005F014FC012100204F
:106DD40005F04EFC05B0F0BD00C0034094A90020AE
:106DE400F0B589B0029303008533040018780028B5
:106DF40000D0A8E0636FCD18E16E8D4200DBA2E005
:106E0400A36FD618236F9E4200DB9CE0626E95420E
:106E140000DB80E0501B0390039D0298471B150084
:106E24000020A26E0490964206DA901B0490049E01
:106E34000E98801B16000E90EA19914200DA4F1B3F
:106E44000E9AB218934201DA9B1B0E93002F7ADD3F
:106E54000E9B002B77DD230044331A78002A1AD0C6
:106E640000221A7006AB1A71013238495A71079A16
:106E74003748069103F012FBD02380221B069203AD
:106E84009A61072333490A685340CF221340802272
:106E940052010A4313602300453305930123059AE5
:106EA400216813700E9AEB19B218013A0092CA6B5A
:106EB400013B94462900320065462000A847029B06
:106EC400049D5D43039BED180F9B6D005D19029BB0
:106ED4005E00BB4222D1029A0E9B29005A43200035
:106EE400FFF7FCF8230046331B78059A1370002B38
:106EF40029D144342378002B25D1164A0133237039
:106F040010211300D0680842FCD10422D968114230
:106F14000FD09968FAE7029F039081E70E9B5A1EEF
:106F24000E92DFD329003A002000FFF7D7F8AD19FD
:106F3400F4E701221A62D02380221B0692035A61CD
:106F4400034803F0AAFA09B0F0BDC046C0FC9B0197
:086F540094A9002000C00340D5
:106F5C00F0B593B002AFBB626023FB181B88040032
:106F6C007B616B463B61030085331E78002E00D09D
:106F7C0006E1436FCB18C16E3B63994200DCFFE026
:106F8C00836FD3187B637A6B036F934200DCF7E05B
:106F9C00426E386B824200DC98E0161AB86A3A638B
:106FAC00801BF862A26E786B0025824204DD151AF4
:106FBC00B86D7A63401BB8653A6BF86A1218914247
:106FCC0002DA3A6B8A1AFA627A6BB96D52189342EA
:106FDC0002DA7A6B9B1ABB65FB6A002B00DCCFE0F4
:106FEC00BB6D002B00DCCBE0220044321378002B6D
:106FFC001DD0002313703C22BA1813703D220133AC
:10700C00BA1862491370FA6B6148B96303F042FA1B
:10701C00D02380221B0692039A6107235D490A68DC
:10702C005340CF221340802252010A4313602300A5
:10703C00012245331A70BB6A5D43AE199640FB6D55
:10704C009B193B62FB6A93406A460833DB08DB0002
:10705C00D31A9D4602ABBB612300A5331B78002BD2
:10706C0003D1BB8A5BBA9BB27B617A6BBB6A9446D9
:10707C005B00FB60BB6D6344BB607B6BBA68934287
:10708C005AD03A6BFB6A944663447B603B6A00259A
:10709C00FB610123BA627A627A6A79688A422FD0DC
:1070AC00FA69796912888A4213D0002B01D07B6A65
:1070BC00BB62B9696B005A5200230135ADB27A6AD2
:1070CC0001327A62FA690232FA61E5E7BA6AFA6267
:1070DC0068E70123002DF2D0796B2268BB6A00911E
:1070EC00D26BEB18013B1600B96A7A6B2000B047E3
:1070FC002A00B9692000FEF7EDFF00250123DEE729
:10710C00002D10D0796B2268BB6A0091D26BEB1802
:10711C001600B96A7A6B2000013BB0472A00B969A6
:10712C002000FEF7D7FFFA687B6B944601337B6334
:10713C003B6A63443B62A0E72300220046331B7882
:10714C0045321370002B1BD144342378002B17D1FC
:10715C00104A0133237010211300D0680842FCD16F
:10716C000422D968114201D09968FAE701221A6207
:10717C00D02380221B0692035A61054803F089F93B
:10718C003B699D46BD4611B0F0BDC046C0FC9B019D
:08719C0094A9002000C003408B
:1071A400F0B58FB002AF7B6128237862F818C3185A
:1071B4001B787B606B46FB607B6A85331E78002EF0
:1071C40000D08CE17B6A5B6FCD187B6AD96EA942D3
:1071D40000DC84E19B6FD318FB617B6AFA691B6F47
:1071E400934200DC7BE17A6A526EAA4200DCB3E08F
:1071F400501B1500B861BC697869001B38627A6A53
:10720400F869926E0026824204DD161AB86CFA619F
:10721400801BB8643A6AAA18914201DA4A1B3A629E
:10722400FA69B96C5218934202DAFA699B1ABB6480
:107234003B6A002B00DC52E1BB6C002B00DC4EE10E
:107244007A6A44321378002B1DD0002313702C2249
:10725400BA1813702D220133BA18A3491370FA6AAD
:10726400A248B96203F01AF9D02380221B069203C4
:107274009A6107239E490A685340CF221340802213
:1072840052010A43136001227B6AB86C45331A70B9
:107294007A6A7B6A1168A533FA693B611B78121814
:1072A400013ABB603B6A0092CA6BEB18013B1400C5
:1072B4002900FA69786AA0476A463B6A5B0008338A
:1072C400DB08DB00D31A9D4602ABFB617B68002B15
:1072D4004ED000220121150014003B6949421A7066
:1072E400844BBB627B6AAC3319607B695E43BB69C8
:1072F400F618FB6C9E19BB6C5A1EBA6400D2C5E02A
:1073040031003B6AFA69F3183B613B69994227D023
:10731400786A0B78AC30B8610068984217D00724BB
:1073240018209D082C40DD08054025431F201C0023
:1073340084432C43DD0085433D6028251C387D199A
:107344001840285C3D680543B869EDB203601470C9
:10735400557001310232D8E77A69BE613A624EE76C
:107364003A6AF969786AFEF7B9FE7B69F618C2E7EA
:107374007B6D002B4DD001213B697A6919705E4BFE
:1073840052181340BA695E430A407A6131D0BA692F
:10739400013A96190E41FA6C5B109619BB61BB6CED
:1073A4005A1EBA6472D37B69002B26D00F2132781F
:1073B400FB690A40796D5200525AF96902330A8016
:1073C4003A6A701C511E00291BD00278140964000B
:1073D400A44665467C6D2C5B1C80012911D00F24CA
:1073E40022407C6D5200125B01305A800239043312
:1073F400E9E7BA6996197610CDE7FB693000396A76
:10740400E1E73A6AF969786AFEF768FEBB69F6183B
:10741400C5E735007B6D3A6913707B690733DB1070
:107424007B61BB6CF318AB4230DDBA69386AFB6927
:10743400101890421EDDFC6CD110615C07241440CE
:10744400A4463961802461460C4121003C692142F3
:1074540009D0796A4969090A1970796A49695970C0
:1074640001320233E5E7796A8969090A1970796A90
:107474008969F4E77A69FB6C9446F96963443A6A6A
:10748400786AFB640135FEF729FECAE77B6A3A7A1B
:10749400A5331A707B6A7A6A46331B7845321370B7
:1074A400002B1CD17C6A44342378002B17D1104A5A
:1074B4000133237010211300D0680842FCD1042248
:1074C400D968114201D09968FAE701221A62D023DF
:1074D40080221B0692035A61044802F0DEFFFB6817
:1074E4009D46BD460DB0F0BDC0FC9B0194A9002093
:0C74F40000C00340000B151FFEFF00004D
:10750000F0B597B002AF040048203B632823381839
:10751000C3181B7848203B622C233818C3181B78EB
:10752000BB626B467B61230085331E78002E00D042
:107530007EE2636FCB18E16E3B64994200DC77E238
:10754000A36FD3187B647A6C236F934200DC6FE2E5
:10755000626E386C824200DCC4E0161A386B3A6402
:10756000801BB8630020A26E7863786C824206DDCF
:10757000101A78637D6BB86E7A64401BB8663A6CFB
:10758000B86B1218914202DA3A6C8A1ABA637A6CB2
:10759000B96E5218934202DA7A6C9B1ABB66BB6BC7
:1075A000002B00DC44E2BB6E002B00DC40E222003A
:1075B00044321378002B1DD0002313704C22BA18CC
:1075C00013704D220133BA18C6491370FA6CC648BD
:1075D000B96402F065FFD02380221B0692039A61F2
:1075E0000723C2490A685340CF2213408022520128
:1075F0000A43136023000122210045331A70A5318C
:107600000B786846FB60BB6B93400833DB08DB00FC
:10761000C31A9D4602ABFB63BB6A002B00D196E008
:107620000022B34B0A70BB64012123004942AC33F2
:107630001960396B7B6B7A624B43396C9B195B1A0F
:10764000F96EBA61CB18B96EFB618C467B6C6344F2
:107650007B607B6C7A68934200D1C2E13A6C002572
:107660009446BB6BFA6263447A63B96AFA6BBB6097
:107670007B6BB86883424FD0786BFB691B5C386AC0
:10768000834232D0002901D0796BF9622000AC30FE
:10769000016838618B4217D0072118209E100E40D8
:1076A000D9100140314318001F26B0430843B86188
:1076B0004820D900B1431C3E1E403818865D314336
:1076C000C9B2796239690B603B7E002113702423B3
:1076D000FB181B7801355370ADB202327B6B01335E
:1076E0007B63C5E73A6BBA633CE7B96A002DF5D016
:1076F000FB6A796C2268EB180091013BD66BF96A42
:107700007A6C2000B0472A00F96B2000FEF7E8FCF5
:107710000025B96AFA6BE1E7002D0FD0FB6A796C9E
:107720002268EB180091D66BF96A7A6C2000013B55
:10773000B0472A00F96B2000FEF7D2FC3A6B7B6C55
:10774000944601337B64FB696344FB6181E7BB6F53
:10775000002B00D1D0E00A70396B664B0131194023
:107760007B6B3240FA614B43002A00D0013EFA6E37
:10777000F3185B10D318BA6E3B6394464B103B6111
:107780007B6C6344BB607B6CBA68934200D128E198
:10779000BB6BBB62FB69002B53D00F223B6B1B788A
:1077A00013403A6A934249D0BA6F5B009B5AFA6B16
:1077B0000125138000233A6C0132FA623A6B0132E0
:1077C0007A62BA6B013ABA623A6C7A63BA6A002A90
:1077D0006CD07A6A396A1278BA6112098A4237D053
:1077E000002B01D0FB6A7B63B96F5200525AF96BD0
:1077F0006B005A5200220135ADB2BB6A012B55D045
:107800000F21BB690B40396A994238D0002A02D057
:10781000FA6A01327A63B96F5B005B5AF96B6A00EE
:10782000535200230135ADB2FA6A0232FA627A6A23
:1078300001327A62BA6A023ABA62C7E700250123C6
:10784000B9E73B6CFD69FB623B6B7B620123BBE7E5
:107850000122002DD1D0796C22687B6B0091D26B14
:10786000EB18013B1600796B7A6C2000B0472A00B8
:10787000F96B2000FEF734FC00250122BDE701234F
:10788000002DD1D0796C22687B6B0091D26BEB1804
:10789000013B1600796B7A6C2000B0472A00F96B27
:1078A0002000FEF71DFC00250123BDE7002D10D0B0
:1078B000796C22687B6B0091D26BEB181600796BA8
:1078C0007A6C2000013BB0472A00F96B2000FEF7DC
:1078D00007FC3A693B6B944663443B637B6C013322
:1078E0007B6450E7C0FC9B0194A9002000C00340CA
:1078F000000B151FFEFF0000BB6F3A620B703B6B65
:107900000733DB10BB617B6BBB627A6B7B6C9B1AB2
:10791000BA6A9B187B62BA6E7B6B9B18BA6A9342F9
:107920005FDD00223B6C3E63FB623B6AFA633A6CAC
:10793000396B921B5518BA6BB1183A6B914231DD15
:107940000720D110FA6E515C3A6B10408022024140
:1079500010000840F8610BD0002B00D0FD62FD6BD9
:107960000135ABB2FB6300233A6B01323A63DEE7C9
:10797000FA6B3B6A002AF7D0FB6A796AD31822684F
:107980000091D26B013B1500F96A7A6A2000A84782
:107990006369FA6B99B22000FDF758FEFA693B6AF9
:1079A000FA63E1E7FB6B002B12D0FA6BFB6A796A92
:1079B000D31822680091D26B013B1500F96A7A6AEC
:1079C0002000A8476369FA6B99B22000FDF73EFEDC
:1079D000BA69FB6E94466344FB66BB6A0133BB62C3
:1079E00093E723003A7BA5331A7022005F3B1B7894
:1079F00045321370002B1BD144342378002B17D150
:107A00000E4A0133237010211300D0680842FCD1C4
:107A10000422D968114201D09968FAE701221A625A
:107A2000D02380221B0692035A61054802F037FDDD
:107A30007B699D46BD4615B0F0BDC04600C0034001
:047A400094A90020E5
:107A440013B5426D03680092002201915C6A110033
:067A5400036DA04713BD05
:107A5C00F0B587B0039303004533150005931A0066
:107A6C0001230F00040013700D9A036800921E6A24
:107A7C002A003900039BB0470D990C9A2368AA1869
:107A8C0000911E6A3900013A039B2000B0470C9A02
:107A9C006B1C961E0D9A049323680092DA693900C8
:107AAC0015003300049A2000A847039A2368B918DC
:107ABC000D9A01390092DF69049A33002000B8470F
:107ACC00220046321378059A1370002B1BD14434D4
:107ADC002378002B17D10D4A01332370102113008A
:107AEC00D0680842FCD10422D968114201D09968AF
:107AFC00FAE701221A62D02380221B0692035A61F4
:107B0C00034802F0C6FC07B0F0BDC04600C00340FD
:047B1C0094A9002008
:0A7B2000C1600261B03003707047CD
:047B2A0081777047A8
:107B30000300E8331B78002B03D0BE300023C05E67
:107B40007047427F012907D1B4300368002B03D06E
:107B5000187B504300B2F3E70C234B430149C9188B
:087B6000087AF6E7082502107F
:0A7B680010B5017FFFF7E0FF10BD2C
:107B7400F7B5089C10251419013C01942B4CCB1823
:107B8400C46584652A4C013B2000E6682E42FCD182
:107B94008027D02507262D067F03AF612568754011
:107BA4000836354080267601264335602A25D026BE
:107BB400A56010243606C5682542FCD10C0A7761FD
:107BC40084608160190A816083601023C16819424E
:107BD400FCD1D02380212B241B06490399618460A6
:107BE4001B3CC5682542FCD15961130A8360019B83
:107BF40082601B0A8360019B83601023C2681A425F
:107C0400FCD1D02380222E211B0652039A6181606D
:107C14001E39C4680C42FCD15A610423C2681A425A
:107C240001D08268FAE701230362F7BDFFFF000079
:047C340000C0034049
:107C3800020013B5443213780400002B1AD0002335
:107C480013706A46137101330E495371019A0E4835
:107C5800009102F021FCD02380221B0692039A6136
:107C680007230A490A685340CF2213408022520151
:107C78000A431360220001234632453413702370EF
:107C880013BDC046C0FC9B0194A9002000C003405E
:107C980070B50200050000234632453513702B707D
:107CA8000400FEF739FA2B78002B07D12300443360
:0E7CB8001B78002B02D12000FCF7D8FD70BD18
:107CC800F7B51D0008AB16001F78099A0C4B040085
:107CD80001919A4204D1036832009B6B984709903E
:107CE800099A29003800FCF723F9050023683200B7
:107CF8001F69019903002000B8472800FEBDC0464F
:047D0800FFFFFF007A
:107D0C00F0B591B004000A9115000393002B00DC30
:107D1C00E8E0030001260A0045331E70039B03991B
:107D2C00B340511A026816989B190090176A2000EC
:107D3C002A00B847039B09961A005B430D939319CD
:107D4C001A0005935B430E93039B5B199B1A0693D6
:107D5C00039BED1AAB180493039B0893039B089A9F
:107D6C0001330C939B1A5B43099A0F93059B9F1A43
:107D7C000C9BDB1B0793079A059B934266DD38002F
:107D8C0078430F9BC0180D9B83425FDA0E9B834296
:107D9C0059DDFDF7E5FBC643F6B2F62E56D8082E94
:107DAC002BD90A9B179ADB1B09930A9BFD184E4B88
:107DBC009A4226D10192169B069A099900962000A8
:107DCC00FFF77CFF179B069A01932900169B0096E0
:107DDC002000FFF773FF179B049A01932900169B51
:107DEC0000962000FFF76AFF179B00960193049AF8
:107DFC00169B09992000FFF761FF079B013F099330
:107E0C00B6E7179B00960193069A169B09992000DA
:107E1C00FFF754FF23680B901B69069A1E0029007C
:107E2C0003002000B0472368049A1B6929001E0038
:107E3C0020000B9BB0472368049A1D6909990B9B82
:107E4C002000A847D9E7099B0793D6E70A9A079B16
:107E5C00944663441E00059B169AF61A7D0023680F
:107E6C00013500921F6A069A2B0031002000B8479A
:107E7C00169A236800921F6A049A2B003100200086
:107E8C00B847089B013B0893069B013B0693049B58
:107E9C0001330493089B002B00D05FE723002200E2
:107EAC0046331B7845321370002B1BD14434237896
:107EBC00002B17D10D4A0133237010211300D06809
:107ECC000842FCD10422D968114201D09968FAE722
:107EDC0001221A62D02380221B0692035A610448A5
:107EEC0002F0D7FA11B0F0BDFFFFFF0000C0034055
:047EFC0094A9002025
:107F0000F0B593B0040004911998002103921D1C50
:107F1000F8F792FC002800D06DE100211A98F8F7DC
:107F20008BFC002800D066E1291C0498F9F7D2FAEE
:107F300040004008B149F8F77FFC00280FD018999D
:107F40000398F9F7C7FA40004008AC49F8F774FC09
:107F5000002804D0281CA949F8F718FE051C199917
:107F60000498F9F7B7FA1A990290281CF9F7B2FAAF
:107F7000011C061C02980CF0B7FD0CF055FDF9F73A
:107F800083FC1A990E90281CF8F700FE0499071C30
:107F90001998F8F7FBFD391C0CF090FD0CF0FAFC79
:107FA000F9F772FC1A990F901898F9F793FA199942
:107FB000071C0398F9F78EFA391C0CF095FD0CF0AC
:107FC00033FDF9F761FC189910901A98F8F7DEFD67
:107FD0000399071C1998F8F7D9FD391C0CF06EFDB0
:107FE0000CF0D8FCF9F750FC11AB1190009310AADB
:107FF0000FAB0EA92000FEF74EF90590002800D126
:10800000F9E0311C0298F8F72BFC189B002800D1EE
:10801000039B181CF9F738FC1A9907901998F9F77F
:1080200059FAFC21099089051998F8F7AFFD1C9BB6
:1080300004999BB20A90281C0693F9F74BFA03990E
:108040000B901898F9F746FA23680C905B6C2000A7
:1080500098472300012245331A700E9B079F08930F
:10806000FE239B050293119BBB425ADB3800F9F7B4
:108070002BFC0399F9F72EFA0026089D0D900F9B13
:10808000AB424CDB002E06D0F42102988905F8F7AC
:10809000DDFB002843D12800F9F716FC0499F9F715
:1080A00019FA099B0B9A00930D990C9BFDF779FA2D
:1080B000011C0A98F9F70EFAF42189050290F8F7E5
:1080C000C5FB002810D1002E00D108954C4902981C
:1080D0002668F8F7C5FB002808D036691B9B3A00D4
:1080E00029002000B047059E0135C8E7454B1C9A82
:1080F0009A4205D1B36B3A002900200098470690B8
:1081000041490298F9F7B4F8F8F74AFC069AC0B268
:108110001B99FBF72DFF226803001669DFE7013783
:10812000A1E70E9B079F0893109B013FBB4258DCC1
:108130003800F9F7C9FB0399F9F7CCF90026089D37
:1081400007900F9BAB42EFDB002E06D0F421029884
:108150008905F8F77BFB0028E6D12800F9F7B4FB86
:108160000499F9F7B7F9099B0B9A009307990C9BAF
:10817000FDF717FA011C0A98F9F7ACF9F421890503
:108180000290F8F763FB002810D1002E00D108956B
:108190001B4902982668F8F763FB002808D0366967
:1081A0001B9B3A0029002000B047059E0135C8E717
:1081B000144B1C9A9A4205D1B36B3A002900200057
:1081C0009847069010490298F9F752F8F8F7E8FB3B
:1081D000069AC0B21B99FBF7CBFE22680300166912
:1081E000DFE7220023004632127845331A702368F5
:1081F00020009B6C984713B0F0BDC0460AD7233CC3
:0C8200000000783FFFFFFF0000007F43FC
:10820C00F0B50D1CFC2187B0040089050D981F1CCE
:10821C00161CF9F727F80F9B029004930E9B019004
:10822C0003930C9B321C0093291C3B1C2000FFF772
:06823C0061FE07B0F0BD79
:10824200FC20D200C0001040DB10C9081843C9024C
:048252000843704726
:108258000300F0B50400002085331B7889B0029034
:10826800834200D0B0E0606F02930918606E0491F9
:10827800814200DAA8E0A16F5618A26E964200DA91
:10828800A2E0049AE16E8A4200DB9DE0226F9642EA
:1082980000DB99E022002700453203921278443728
:1082A80005924B4D002A1AD0039A13703B78002B85
:1082B80015D101333B700F33EA681A42FCD104230D
:1082C800EA681A4201D0AA68FAE7012380222B62E1
:1082D800D02392031B065A613E4802F0DCF82000C6
:1082E800FDF71AFF3B78002B10D0002206AB1A715D
:1082F8003A7001325A713849079A3648069102F0A5
:10830800CBF8D02380221B0692039A610123320006
:10831800009304992000FFF729FC2E4F0021380014
:1083280002F074F80021380002F070F80021029081
:10833800380002F06BF800210600380002F066F8F9
:108348000299030032002000FFF777FFD023802234
:108358001B069203039902905A61097800290AD1F1
:10836800210044310878002805D1013008705A618D
:10837800380002F090F807228026CF272B68760174
:1083880053403B402E433360059B002B1CD04434A4
:108398002378002B15D0002206AB1A712270013207
:1083A8005A710E49079A0B48069102F075F8D023C6
:1083B80080221B0692039A612B6807255D402F4097
:1083C80037600123039A1370029809B0F0BDC046C4
:1083D80000C0034094A9002080969800C0FC9B012F
:1083E800030030B5A8331B78002B02D18DB22800CA
:1083F80030BD4AB2431C002A02DB0022DA77F5E7D7
:10840800DD7F002D16D11F220C009443C02C07D10C
:108418008A01F821C9000A4042840122DA77E6E796
:108428000F220C0094432200E02CDFD10903418481
:10843800DE3AF3E72222845E022D09D1FC2289016B
:10844800120111400122214341840025DA77CEE749
:0E8458003F22114021438DB245840022DEE711
:108468000300F0B585331B7887B004000F00002B9C
:1084780013D1FFF7B5FF011E04900ED00D2F0CD0BD
:108488002300E8331B78002B0AD01F2801D80A2FB5
:1084980003D123682000DB6C9847012007B0F0BDAA
:1084A800049B0A2B01D1163304932600B436336893
:1084B800002B6AD1227F022A1DD1049B203B9BB24C
:1084C8005F2BEAD8049A654B9B18203B1A78102337
:1084D8000632D208D20025002600617F8C354B4336
:1084E800883605930A2F20D12A68944663442B6066
:1084F80000233360D1E7D11E05290FD8049B203B08
:108508009BB25F2BC9D80C214A435549049B891853
:108518004A689B18203B1A780B7ADCE7012A01D0BD
:108528001A00D8E708230622D5E72300A3331B78CF
:10853800002B0FD0514333682000CF1823685B6BA2
:108548009847874206DD2A68059B944663442B605A
:10855800002333602300A4331B78002B08D0236842
:1085680020001B6B2F689847B84201DC00232B6062
:10857800227F236800929F6A32682B680499200042
:10858800B84733681818306087E70A2F0AD12200E5
:10859800002188321160617F1B7B4B4351685B1857
:1085A80053607AE75A8904998A4200D275E71A8992
:1085B800914200D271E78A1A0C21250092B24A43EF
:1085C8005B688835D31805931B79002B3ED0059A34
:1085D8005279002A3AD02200A3321278002A18D001
:1085E8000727059A2000D757FB18677F5F432B683A
:1085F800FF1823685B6B984787420ADD0023220037
:108608002B6033688C32197B637F4B4311685B188E
:10861800136023002700A4331B788C37002B08D065
:10862800236820001B6B3E689847B04201DC00239A
:108638003B60627F23680292226920000192E2680F
:1086480000925E693A68049B2968B047059B9A794D
:10865800637F53432A689B182B601EE7A82D0210DE
:0486680008250210CF
:10866C00F0B515889C466B1C9BB21380A8304E5DF0
:10867C000078B4B2002814D070B2002811DA1F2090
:10868C0037008743C02F0ED1604601280BD9023525
:10869C001580CC5C3F20F8230440DB00B00118406F
:1086AC0004432000F0BD0F2037008743E02FF8D1A2
:1086BC0060460228F5D9AF1CBFB21780CC5CFC23F6
:1086CC00A4011B011C403F2303351580C85D1840D5
:0A86DC00330303431C43A4B2E3E799
:1086E800F0B51500FC261A0028000A4FF6003A409B
:1086F800384033403540801A8C104443E81A4843C8
:10870800A409000AA218C0183A403040104380B2A9
:08871800F0BDC0461FF8FFFF91
:10872000F02270B504000D001100FDF7F7FD124BAB
:1087300021000833220023600023F032FF312000A3
:108740008B7615601025F4309365D36505704F382E
:1087500003704B76012120380170D3621363536399
:108760009363D3631364D3612300A9331970633B0C
:0C8770002000197070BDC0467825021072
:10877C0070B5022B0ED8002B0ED00400F4342578E3
:10878C00102D0BD15943080002215043C0180DF095
:10879C0075FB70BD0223F0E70123EEE7082D05D130
:1087AC005943080050430121C018F0E78CB2FC304B
:1087BC00042D0AD1012101348C4324B2C46420005D
:1087CC00584350430841C018E1E7072107348C4354
:1087DC0024B2C464C465E4105C4362430639D01807
:0287EC00D5E7CF
:1087F000030070B5FF335B7E0D001600002B1AD00E
:10880000002900D10C4DFC3003690400002B04D179
:10881000022110200DF038FB2061331C102E00D9EE
:1088200010230022DBB25B009A4204D0A95A2069CF
:0C88300081520232F8E770BDEA1F02100E
:10883C00F0B585B002930300FF3303935B7E060013
:10884C000F001400002B03D0FC36B06805B0F0BD4F
:10885C00002901DC0020F9E7002AFBDD0500FC35CE
:10886C00AA652A6502008832E9656965E9641360C6
:10887C005360AB63EB63AB642964029B6C642200B2
:10888C00FFF776FF3300F8332860A860E860043BFC
:10889C00586068601B78102B0ED1029B012B04D9F9
:1088AC007C43640001340419EC600028D2D03300FE
:1088BC000122FF335A7622E0082B04D1029B012BB4
:1088CC00F3D97C43EEE7012B0AD1029B012BECD9A7
:1088DC0007373F04FF1467430137C719EF60E4E71C
:1088EC000028B7D0012203994A76042B07D12B69B3
:1088FC00002B04D10F320F493000FFF773FF00211A
:10890C000123F1770193AB6D0A00009330006B6D7E
:10891C00FDF71EFC2A6DE96CD30F9B18CA0F521879
:10892C0031005B105210603162360A80A8683380C7
:08893C008CE7C046EA1F02109F
:1089440070B50500FC3504002869002803D00EF03A
:10895400B7FA00232B612600FF36737E002B08D064
:10896400A8680EF0ADFA002385342B6073760133CA
:04897400237070BD3F
:108978000300F0B5FF335B7E87B00500002B1DD0E8
:10898800030007002E00F037F433FC361C783868F3
:108998000597B76D736D04970027102C10D104004C
:1089A800F835A534267827702C680194049C009427
:1089B800FEF714FA059B1B68A5331E7007B0F0BDBF
:1089C800042C09D134690297039474680194049CB7
:1089D8000094FEF7E3FBF1E7083C65426C4103971E
:0689E80002943468F2E77E
:1089EE00F0B51C000300FF335B7E8BB00500002B3F
:1089FE0024D00300F4331B782E009C460300FC3673
:108A0E00F03309931868736DB76D07936346089733
:108A1E000027102B14D195339C4684446346F835B9
:108A2E001E781F7002942B680193089B0093079B7E
:108A3E00FEF78DFA099B1B68A5331E700BB0F0BDB7
:108A4E00082B0FD101250497039527121E35AF432E
:108A5E001433A5111D40E4062F43A40F274302979C
:108A6E00336808E0042B0DD10F2533692C40049395
:108A7E000397029473680193089B0093079BFEF77C
:0A8A8E0038FDDBE704970397E9E7E2
:108A9800020070B5FF32527E0B00002A1FD0020080
:108AA8000400F4321178FC34256B626B102917D15D
:108AB800E16CF8304A430168521952005352236B53
:108AC800A26A01332363934209DD236AE26A2363BE
:108AD800636B01336363934201DD636A636370BD53
:108AE800082905D1E16C4A4321684D19AB54E6E7E2
:108AF800042911D10F26E16C33404A4361685219A9
:108B080052108A181078E90704D41B013040184322
:108B18001070D4E7B043FAE701680E692900B0473E
:028B2800CDE797
:108B2C00F0B591B0059316AB07921A780300853314
:108B3C001B7804000D00002B02D0002011B0F0BDFA
:108B4C000029FAD0012A25D1427F036802920269DA
:108B5C000192C26800925E69059A0B000799B047B2
:108B6C002300B4331A68002A03D10623607F5843CC
:108B7C00E4E713899D42E0D35189A942DDD3ED1A74
:108B8C000C23ADB25D435268637F5519A8795843E5
:108B9C0000B2D3E7203D931EADB2062B01D85F2D5A
:108BAC00CBD8022A2AD1AD49AB00CB580693AC4B9B
:108BBC005B5D089310230C93616F079B8C46A16F30
:108BCC0063448C460A93059B607F63440B93089B1C
:108BDC000A994343656E5B18AB4202DBE66EB14209
:108BEC0021DB0C990B9E41438919A66EB14203DB24
:108BFC000B99266FB14216DB089BC8E7D31E052BD9
:108C0C000CD80C215143974BA8005E585B1859683F
:108C1C008059495D069008911B7ACCE70023069396
:108C2C000C930893C8E7012109910A99A94211DB19
:108C3C00E16E8B420EDA0B9BA16E8B420ADB0C9B16
:108C4C000B994343256F5B18D917EE0FAB4271415B
:108C5C00CBB20993022A00D006E1089B0633DB1045
:108C6C000B9300230A930C9B0A9A934200D140E287
:108C7C002169E3688B420AD0627F2068089B0191CE
:108C8C0000925343456A059A07992000A847002390
:108C9C0009930B9A0999637F8A4200D1D2E0069A14
:108CAC00565C002E5CD0CD0072B2012B5BD1079BC1
:108CBC00E918002A05DA2368059A1F692000E36881
:108CCC00B84740231E4208D0079B059A591C2368BD
:108CDC0049191F692000E368B84720231E4208D0B9
:108CEC00079B059A991C236849191F692000E368A2
:108CFC00B847F30608D5079B059AD91C2368491970
:108D0C001F692000E368B847330708D5079B059A0D
:108D1C00191D236849191F692000E368B8477307B8
:108D2C0008D5079B059A591D236849191F6920000E
:108D3C00E368B847B30708D5079B059A991D2368C4
:108D4C0049191F692000E368B847F30708D5079B4A
:108D5C00059AD91D236849191E692000E368B0479C
:108D6C00099B013394E75D4307996D18002A08DAD3
:108D7C00E168226801910093576A2900059A200046
:108D8C00B84740231E4209D0637FE06822680190F7
:108D9C000093576AE918059A2000B84720231E4211
:108DAC000AD0637FE0682268019059000093576AEB
:108DBC004919059A2000B847F3060BD50321637FA8
:108DCC00E0685943226801900093576A4919059A43
:108DDC002000B84733070AD5637FE068226801900A
:108DEC0099000093576A4919059A2000B8477307F0
:108DFC000BD50521637FE0685943226801900093ED
:108E0C00576A4919059A2000B847B3070BD50621B4
:108E1C00637FE0685943226801900093576A4919AF
:108E2C00059A2000B847F3079AD50721637FE068BD
:108E3C005943226801900093566A4919059A2000FB
:108E4C00B0478DE7059AD3180B9A059394460A9B65
:108E5C0001330A93069B6344069304E72826021009
:108E6C00A82D0210082502100C9B089AE1685343A8
:108E7C000D932300F4331B78102B5ED10A020F0ADA
:108E8C0017433AB20E922269102B66D1160A1702BA
:108E9C003E4335B2914200D08DE0099A002A00D0B1
:108EAC00CDE0012B00D1C9E0030043430138DBB214
:108EBC000F93C3B2079313000593059A0D9B93422E
:108ECC0000DC16E1069B069A1B78013206925AB218
:108EDC00002A6BDA7F2213400133089905980C9312
:108EEC00F7F736FC079B002B4BD0667F0A9B714330
:108EFC004643CD180B9BF6180C9B0993099B013B21
:108F0C00DBB20993FF2B37D007992268079B89198D
:108F1C0000915B19D76B290032002000B847079BE2
:108F2C00002B33D00F9F013FFFB2FF2F33D06B4686
:108F3C002000198FFFF7AAFDF5E7082B01D00AB224
:108F4C00A0E7E0221C260D0A15408A093240154381
:108F5C00CA06920F15430E9595E7082B01D015B252
:108F6C0098E7E025170A2F409609C43D35402F435A
:108F7C00D506AD0F3D438DE70C9A059B9446634493
:108F8C009AE70A9B5D180B9B1E18B5E76B462000F1
:108F9C00198FFFF77BFD637F089A0A995A43ED18E6
:108FAC0052189542AADBF6180D00A7E70133059A73
:108FBC00DBB2D31880E701283FD1099A002A3ED1B1
:108FCC00012B3BD00B98089A84460A9B21689B186E
:108FDC000C9A013B6244013A0092CE6B02000A9952
:108FEC002000B0477F270D9B002B00DC81E0069B07
:108FFC001E7873B2002B12DA0D9B3E4001369B1B80
:10900C000D93013EF6B2FF2E05D06B462000198F52
:10901C00FFF73CFDF5E7069B01330693E3E70D9B59
:10902C000136F6B29B1B0D93013EF6B2FF2EF2D029
:10903C00A9B22000FFF72AFDF6E7012309930027C8
:10904C000D9BBB4255DD069B1D7801336AB206931E
:10905C00E368002A36DA9BB20B937F231D407E3BDC
:10906C00099338000899F7F773FB667F8C467143B8
:10907C00079B4643C918059B0135F3180A93002337
:10908C00EDB27F19013DEDB2627FFF2D22D060461B
:10909C000133089E18188642F4DC0998002809D080
:1090AC000B9E2068019600925343426A20001600E2
:1090BC000A9AB0470A9A637F0799D3180A93002338
:1090CC009C46DFE7226992B20B9222699A42C8D180
:1090DC000023C5E7002BB3D009980028B0D00B9D16
:1090EC002068009201955343456A0A9A2000A847CC
:0890FC00A6E7607F80E5C04695
:10910400030073B5FF335B7E04000D00002B35D0E4
:10911400030085331B78002B30D1436F002B1ED105
:10912400836F002B1BD10368C66F5B6B9847B042FB
:1091340015D12300F4331B78102B28D1231DD86FAD
:109144002B0AE9B2DBB2994219D12300FC33DA6C61
:10915400F8344243206852000EF074FA0EE0A36E15
:10916400A26F616F9A1A636E591A230001CB01959D
:10917400DB6F0093456AE36F2000A84773BD236843
:10918400019500905D6AA26EE36F616EF4E7082BAF
:1091940011D12300E0200434E26F1C24FC33D96C89
:1091A4004A43290A0140A8092040ED060143AD0FB6
:1091B40029431868D0E7042B0ED123000434FC3370
:1091C400D96CE26FEDB24A430F2129402D012943A6
:1091D4005210C9B25868BFE7012BCFD1FC34E36DFC
:1091E400A26DDB105A4320680132FF21002DB3D158
:0491F4000021B1E7BE
:1091F80070B50500CC3504002868002803D00DF0B0
:109208005DFE00232B602500D0352868002803D098
:109218000DF054FE00232B602500D4352868002863
:1092280003D00DF04BFE00232B602500D8352868AD
:10923800002803D00DF042FE00232B602500DC350A
:109248002868002803D00DF039FE00232B60250084
:10925800E0352868002803D00DF030FE00232B608D
:109268002500E4352868002803D00DF027FE0023E8
:109278002B6022000023B832E8341360237070BDDD
:1092880010B50400074B08330360FFF757FB2300B2
:10929800E8331B78002B02D02000FFF7A9FF20003D
:0892A80010BDC046782502103C
:1092B000020010B5EC321368591C1160981C197823
:1092C00010605878090600040143D81C1060181D6E
:0E92D0009C781060D87824020843204310BD1B
:1092DE000300F0B5BC331D881C2304006B436E00E5
:1092EE0085B01833300000930DF0DBFD2300CC3336
:1092FE00186028000DF0D5FD2300D033186028002B
:10930E000DF0CFFD2300D433186028000DF0C9FDF9
:10931E002300D833186030000DF0C3FD2300DC337A
:10932E00186028000DF0BDFD2300E0331860A80082
:10933E000DF0B7FD23000025E43318602300BC3385
:10934E001B88AB425ED92000FFF7ABFF2300CC3366
:10935E00019327001B686A00985220000293FFF7C2
:10936E00A0FFD0373B68260058552000FFF799FF25
:10937E002300D43302931B68DC3658552000039328
:10938E00FFF78FFF2300D8331B6858552000FFF7D7
:10939E0088FF33686A0098522000FFF782FF23008F
:1093AE00E0331B6858552000FFF77BFF32686800DA
:1093BE00125E20003B68C8305B1919788A1A018842
:1093CE008A4209DD01996E000968895B0E00213E13
:1093DE007E2E13D87F2913D12200E4320098126812
:1093EE00A9008850029A1B781268525D01355343CA
:1093FE00C3180093ADB203F0E2F89FE7FF29EBD953
:10940E000280E9E723002200C633C83212881B8887
:10941E0007219B182200BE3213802300C233002086
:10942E00185E2300C43300229B5EC034C018400077
:0A943E00F7F7A7F8208005B0F0BD95
:10944800F8B50500E8352B7804000E00002B01D094
:10945800FFF7CEFE3100300003F010F822002300A1
:10946800EC321268B8331A602000FFF71DFF2300A2
:10947800BC3318802000FFF717FF26002000FFF7F5
:1094880013FFBE3630802000FFF70EFF27002000B4
:10949800FFF70AFFC23738802000FFF705FF2300D7
:1094A8002200C43318803B88C63280B213805080B3
:1094B8001818230080B23080C03380081880012338
:0A94C80020002B70FFF707FFF8BD2E
:1094D4001FB5040000290ED00300EC33196001A865
:1094E400054902F0BAFF2000002201A9FFF7AAFFF4
:0C94F40001A802F063FF1FBD74250210E8
:109500000300F0B5BC331E880023CC309CB2A642C9
:1095100008D907685D00ED5B01338D42F6D101206B
:089520001480F0BD0020FCE7FF
:109528000300F7B5E8331E7804000D00002E44D080
:109538000026297800293CD02000FEF751FF01358C
:10954800011EF6D0202804D12300C0331B88F6184A
:10955800EFE76B469F1D00233A0020003B80FFF792
:10956800CBFF002820D03B88002E06D12200E03215
:109578001268D256002A00DA56422A78002A04D104
:109588002200A2321278002A04D02200D8321268AF
:10959800D35CDCE722002100E032D431126809688C
:1095A800D256CB5CD318D2E72300C0331B880133D3
:1095B800CDE7A234217030B2FEBD931E062B14D81D
:1095C8000C235343274AD218536819001F3B2039EC
:1095D8002A78002A19D01000203801355F2802D8CF
:1095E8008A5CB618F4E7DA7FFBE70700B4373B6814
:1095F800002B12D1063B4B4306210E006E4301356A
:109608006A1E1278F618002AF7D123000022A23326
:109618001A70607F704300B2CEE729780029F4D031
:109628002000FEF7DDFE3B6801351A899042F4D32D
:1096380059898142F1D3801A0C2280B250435B6869
:10964800C0182B78002B04D12300A2331B78002BE1
:1096580002D08379F618E0E707230279C3569B18EE
:08966800F8E7C04608250210D6
:10967000F0B58FB01D0014AB1B7817001A00040062
:1096800006930A91FFF750FF83B20493637F9AB267
:109690000992D2000592069A012A23D12200B432FF
:1096A0001268002A24D02200E8321278002A3ED123
:1096B0002200A03210789AB242430592AD186A4651
:1096C000167DA27F063A022A08D82200A13210781D
:1096D0009AB25043059A101882B20592069A0892DF
:1096E000652203E00022089216000132039203E093
:1096F00006990391160008922200E8321278002A97
:1097000019D023002000C6331E78FEF72DFA83B24D
:109710000593A07F00282FD001380A282CD8F6F70F
:10972000A3FE1B2328585F65676C70727700069A4A
:1097300003920022DEE7069A012AEAD00C21514367
:10974000A74A20005218567A5E436B461821595E8C
:10975000F6B2FEF7EDF9DAE7049B5B08FF1A039B0C
:109760000133DBB2039307E0049BFF1A039B023330
:10977000F7E7059B5B08ED1A0A980EF065FA0023DF
:109780000793089B002B78D0E3682269934274D03A
:109790002300A03386B2187801331B780AAAC018B8
:1097A000099B43439BB205930E239B186A460020F6
:1097B000928B1A800E220AABD2181388B3422BD296
:1097C000002829D1F31A9BB20A992000FEF74EFF18
:1097D000F0E7049B5B08FF1A059B5B08ED1ABEE7E8
:1097E000049BFF1A059B5B08ED1ABFE7059BC2E7C8
:1097F000049B5B08FF1A059BF0E7049BFF1A059B7F
:10980000F2E7AD1BB8E7049BAD1B5B08FF1AA6E7A8
:10981000049BAD1BFF1AA9E723000022B4331B6889
:1098200007921989884224D35A89824221D3401A47
:109830000C2180B248435B68627F1818C379534398
:109840005BB20793002B4ADC049B07995B1A9BB21F
:1098500004932300A0331B7820695A43079B01908F
:109860000598D919236800905E6AAA1A049B200003
:10987000B047039B643BDBB203930A980EF0E4F914
:1098800083B20B930E230AAA9B1800221A8023008E
:10989000E8331E7896425BD0603B3AB21A602AB237
:1098A0005A6022009032126828331E78002A03D0B2
:1098B000002E01D101221A700E220AABD218138891
:1098C0000B998B420ED2CB1A9BB20A992000FEF75D
:1098D000CDFE23680100DB6C20009847ECE70023F5
:1098E0000793B6E72300B0331E706B4610229A5ED2
:1098F0000992230090331B68049A934263DD226926
:10990000E16891425FD004990798C919091808982D
:1099100009B200280DD007983F182000A030007829
:1099200084466646607F70432D1A09983E1830B20F
:1099300009900398022829D0032847D0012842D152
:1099400004981B1A0192059A20680092476A37E032
:1099500009960E220AABD21813880B998B42C8D2F3
:10996000CB1A9BB20A992000FEF780FE099B0100EA
:109970000698DA19236800909B6A20001E002B00CD
:10998000B047099B1E1833B20993E2E7049801928D
:10999000059A1B1A20680092426A5B10160020008C
:1099A0002A00B0472300206990331B68049A019075
:1099B00005989B1A22685B100090F91A576A09B241
:1099C0002A002000B84709980FB0F0BD8B4200DA9A
:1099D00019B20498049BC019CB1A411AB2E7C046C9
:0499E0000825021044
:1099E40070B504001E0023001500012286B0A233C6
:1099F4001A700800093203A902F08BFD237F2A00A4
:109A0400009303A933002000FFF730FE06B070BDB9
:109A1400F0B504000500C36895B006930369883463
:109A24009835029322682B680700934203D0030001
:109A340094331A602A60202944D828D13B003E0080
:109A4400B0331B7894360396002B16D03B00C033FA
:109A54001B8839009B18326838689B1A6A46128939
:109A6400BE31019209880091426A039916003A00B6
:109A74008C32126809683800B047C03722683B88C6
:109A84009B18039A236013602B6015B0F0BD0A295C
:109A940018D13B000026943326601E602E603D00E2
:109AA4008C355C8D2B68E4183B002C60A4331B7848
:109AB400B342EAD03B6838001B6B98478442E4DB2E
:109AC4002E60E2E70E2510ABED1800232A003800C3
:109AD4002B80FFF713FD002800D10FE26B461B8B90
:109AE4000D936B461B890E933B00FF335A7E012373
:109AF4005A40089200D121E13A003800BE32D430F5
:109B04000021525E00682988415C3800FEF794FE0B
:109B14000D9B0E9A934204D06B4638001989FFF7C7
:109B2400EFFA3A00E03212682B88D3563A005B42CF
:109B340088321360D36013613B0000228C331A60B7
:109B44003B000E21B8331B6810A8091811930C8828
:109B54003B0039008C33DC311A6809683A331B88BE
:109B64006000455A9918491B89B2109140206946F2
:109B740009180020095E03913900883108685831BA
:109B8400096880B20957411889B2099169462426A7
:109B9400895F04913900B0310978002900D11DE1B1
:109BA4003E003900D836943136680968345D401A6D
:109BB400201800B20590002800DC0CE15B1B1BB2EE
:109BC400002B07DD3C69386800930194446A059BC7
:109BD4003800A0473B0094331968049B994210DA7B
:109BE40038693A6801900E2010AC00193C00D0345A
:109BF400246800885B1A205C0090546A3800039A39
:109C0400A0473B00002294330C921B68049A9A42AA
:109C140003DA099A9B1A1BB20C930E2310AA9B1801
:109C24001A883B00D4331B683800995C049B883045
:109C3400C9183B00D8331B6800689B5C1B18994209
:109C44000CDA3C69386801943C00D03424685B1A0F
:109C5400A25C0092446A039A3800A047049B0B93C9
:109C640007930E9B0A9300230E243A00029310AB31
:109C7400E418D03223881268D25C029B9A4200DC3A
:109C840002E10026350034000E2310AA9B181A881E
:109C94003B00D4331B689B5CB34200DCD6E0390044
:109CA4000298E4310968920043435158119A921979
:109CB400D3185B5C0F93002B00D1A6E0002D0BD0D2
:109CC4000A993B6800911B6A039A9C4682182B00F0
:109CD4000B9938006546A8470F9BFF2B00D18AE0FB
:109CE400029B039A9D18002C09D06B463A681B8B83
:109CF400012C76D1146907992A003800A047049BE7
:109D04000E9A9C190D9B934206D13B682A009B6BCB
:109D14002100380098470A900A9B0D9A0F99380041
:109D2400FEF7E0FC3A68030012692100944638000B
:109D34002A006446A0470025002464E03B00A333C6
:109D44001B78002B22D03A002B883D00D4321268B5
:109D54008835D45C2A683800A4183A00E0321268C6
:109D6400D356E4183B685B6B984784420EDD3A0097
:109D74003B008C32BE3311681B88CB181360089BE0
:109D8400089A2B603B0094331A605A603B00A4335A
:109D94001B78002B0ED03D003B008C35BE331C8855
:109DA4002B683800E4183B681B6B9847844201DD3C
:109DB40000232B603A0088321368002B00D0BFE6E2
:109DC40010A90E335B183900E03109681B88CB56A3
:109DD4005B421360B4E600230593FBE605910C9106
:109DE4003CE70093136A07999C462A002300380035
:109DF4006446A04783E7002C03D1099B9B191BB23F
:109E040007930025013401363EE7002C0DD0694646
:109E1400029B039A098B9A183B6800911B6A079965
:109E24009C46380023006446A0473B000024B0331E
:109E34001B78A342E7D00C9BB342E4DCA54203D1D8
:109E4400099B9B191BB20B93013575E7002C0BD0B2
:109E54006946029B039A098B9A183B6800911E6A13
:109E6400079923003800B047002D0AD0029B039ABB
:109E74000A999A183B6800911C6A0B992B003800C8
:109E8400A047029B0133EFE6059B002B19D03B0052
:109E940039008C33BE3109881B685B1810995B1A32
:109EA4009B1A1BB2002B0CDD039938698A18396898
:109EB400019000934D6A39009431059B096838007C
:109EC400A84739003A00D831096823888832CB5C26
:109ED40011685B181360089B002B09D03B008C337E
:109EE40038001A680499FEF745FD3800FEF728FD8E
:109EF4003B0088331A68DA601A61C6E53A00390013
:109F0400C6328C31096812883B00521869463D00FC
:109F1400C2330020185E098BC0352B880090019154
:109F2400121A21683800FDF797FD2B882268013347
:069F34009B182360DCE72E
:109F3A00F0B504000500C36893B007930369883439
:109F4A009835099322682B680700934203D00300CF
:109F5A0094331A602A60202944D828D13B003E0055
:109F6A00B0331B7894360396002B16D03B00694613
:109F7A00C0331B88898C9B18326838009B1A3A6850
:109F8A0001913900BE3109880091526A039916007D
:109F9A003A008C3212680968B047C03722683B8899
:109FAA009B18039A236013602B6013B0F0BD0A2933
:109FBA0018D13B000026943326601E602E603D00B7
:109FCA008C355C8D2B68E4183B002C60A4331B781D
:109FDA00B342EAD03B6838001B6B98478442E4DB03
:109FEA002E60E2E70E2500260EABED182A00380097
:109FFA002E80FFF780FA3B00B04200D1CEE1A333B6
:10A00A001B78B3421DD03A00D4322B88126838002C
:10A01A00D55C2268AD183A00E0321268D356ED18C2
:10A02A003B685B6B984785420BDD3A003B008C32FC
:10A03A00BE331B881168CB1813603B00943326602B
:10A04A001E603B003D00A4331B788C35002B0CD0DE
:10A05A003B00BE331E882B683800F6183B681B6B22
:10A06A009847864201DB00232B600E230EAA9B1819
:10A07A0019883B00E0331A6823685218002B03D171
:10A08A000023D3565B4223603B00B8331B683C0075
:10A09A000F933B00C63303931B882868DC34C3182C
:10A0AA0020684900095A3E005B1A9BB20B936B4623
:10A0BA002C215B5E883604930023D356326838001D
:10A0CA00D3189BB208936B4620229B5E0693FDF73A
:10A0DA00AEFD3B00B0331B78002B00D1D8E00E2335
:10A0EA000EAA9B183A009432116844321B881268EF
:10A0FA003068D25C401A121812B20592002A00DCAB
:10A10A00C3E05A002068039B125A1B889B1A1BB291
:10A11A00002B08DD38693A6801900093546A059B60
:10A12A002A683800A0473B0094331968069B994275
:10A13A0010DA38693A6801900E200EAC00193C001A
:10A14A00D034246800885B1A205C0090546A380076
:10A15A00049AA0473B00002294330D921B68069A8A
:10A16A009A4203DA089A9B1A1BB20D930E230EAA7F
:10A17A009B181A883B00D4331B683800995C069BED
:10A18A008830C9183B00D8331B6800689B5C1B18D1
:10A19A0099420CDA3C69386801943C00D03424684E
:10A1AA005B1AA25C0092446A049A3800A0476B4684
:10A1BA009B8C0A93069B0C93099300230E243A0066
:10A1CA0003930EABE418D03223881268D25C039B47
:10A1DA009A4200DCB2E00026350034000E230EAAB3
:10A1EA009B181A883B00D4331B689B5CB34200DC83
:10A1FA0086E039000398E4310968920043435158D4
:10A20A000F9A9219D3185B5C0E93002B57D0002D2E
:10A21A000BD00A993B6800911B6A049A9C468218E3
:10A22A002B000C9938006546A8470E9BFF2B3CD0A3
:10A23A00039B049A9D18002C09D06B463A689B8BA5
:10A24A00012C28D1146909992A003800A0473B6CCF
:10A25A00002B08D00B9A03995118089A89B29019C1
:10A26A0080B298470A906B460E999A8B38000A9BDF
:10A27A00FEF735FA069A030091193A68380014690C
:10A28A002A00A0470025002417E0002305934AE787
:10A29A0005930D938BE70093136A09999C462A004C
:10A2AA00230038006446A047D1E7002C03D1089B5D
:10A2BA009B191BB209930025013401368EE7002C45
:10A2CA000DD06946039B049A898B9A183B680091C2
:10A2DA001B6A09999C46380023006446A0473B0044
:10A2EA000024B0331B78A342E7D00D9BB342E4DCD1
:10A2FA00A54203D1089B9B191BB20C930135C2E7F7
:10A30A00002C0BD06946039B049A898B9A183B68E8
:10A31A0000911E6A099923003800B047002D0AD01F
:10A32A00039B049A0A999A183B6800911C6A0C9933
:10A33A002B003800A047039B01333FE7059B002B06
:10A34A0019D03B0039008C33BE3109881B685B1871
:10A35A000B995B1A9B1A1BB2002B0CDD0499386906
:10A36A008A183968019000934D6A39009431059B27
:10A37A0009683800A84739003A00D83109682388A3
:10A38A008832CB5C116838005B181360FDF77FFCDC
:10A39A003B0088331A68DA601A6106E63A00390027
:10A3AA00C6328C31096812883D0052186946C23398
:10A3BA000020185E898BC0352B8800900191121AF3
:10A3CA0021683800FDF745FB2B88226801339B186A
:04A3DA002360DDE738
:0EA3DE0010B50400182108F02CF8200010BD66
:10A3EC0010B5064C022303220021200000F0A4F833
:10A3FC00034A0449200007F0D3FD10BD94A90020A6
:08A40C0040020020A93F0010EE
:10A414000B000F2130B50122172487B069440B705B
:10A42400C3686C44186803680092DD682300A84779
:06A43400207807B030BDE6
:10A43A00F8B5427A036805000C00CFB29B680E0A91
:10A44A00002A0FD13900FF2798472B68BC430443E1
:10A45A009B683100280098470302200038401843BF
:10A46A0080B2F8BD31009847FF262B6800023440BD
:10A47A0004439B68390028009847B4432043EFE718
:10A48A0013B5C368186803680092DC680B00A0471C
:02A49A0013BDF0
:02A49C00704707
:02A49E00704705
:10A4A00037B5436804000D0000910192994204D130
:10A4B0006B469A8803899A4210D06B461A79E368F2
:10A4C0000821186804F037FBE3682900186804F0D5
:0EA4D0004EFB201D062269460DF024F837BD14
:10A4DE00C36810B50400002B0BD01868002808D0F4
:10A4EE0003685B6898470421E06807F0A2FF002329
:04A4FE00E36010BD4A
:10A5020037B5C5680400002D04D1042007F067FFA9
:10A51200E0600560E3681B68002B11D1302007F072
:10A522005EFF1422A35E05001021625E1220215EEE
:10A53200012040420090280004F0C1FAE3681D6047
:02A5420037BD23
:10A5440070B51D000C4B1600083301220360002374
:10A554000400436003724272C360C8B201F0FAFFA0
:10A564002082F0B201F0F6FF6082E8B201F0F2FF5F
:0CA57400A082200070BDC046882F02109D
:10A5800070B5102001F0E8FF0500132001F0E4FF92
:10A590000400122001F0E0FF094A0A4B08321A6059
:10A5A0000121002259725A601A72DA609882064AB2
:10A5B000064918001D825C8207F0F8FC70BDC04699
:10A5C000882F0210D895002040020020A93F0010DB
:10A5D00070B5104C10492068104A114B88420FD1B9
:10A5E000606890420CD1A068984209D100250D48BE
:10A5F000256009F0BDFC03008020290080049847F5
:10A60000216009480021A360626009F013FB002368
:10A61000236070BD14100020DE8116F0299B72BDEE
:0CA620007ABE59D355420000A08601000C
:10A62C000B00F0B50F2700260E33023902003A401A
:10A63C00D5B22C0000093034092A00DD07341C7017
:0AA64C005E70023B9942F1D1F0BDAF
:04A656001E2070470B
:02A65A00704747
:10A65C0013B50400684608F0F9FE21000098FFF7D6
:10A66C00DFFF210001981031FFF7DAFF202016BD23
:10A67C0010B5192001F06AFF0400044809F072FCBF
:10A68C00030001200021A0409847C046554200001D
:02A69C00704705
:0AA69E0010B50C220CF03FFF10BDB8
:0EA6A800C36810B5002B01D09B68984710BD09
:0CA6B60010B50400FFF7F5FF200010BDF8
:10A6C4009C2370B55B00C35C05001400002B1CD1F7
:10A6D4000368DB699847F0210C4B09012140C91834
:10A6E4004B1E9941F0232340303B5A4253410F22E1
:10A6F4000731144001330D3A012C02D0023C62426E
:10A704006241A869006804F0B0FB70BD00FDFFFF62
:10A714009C2310B55B00C35C0400002B05D1A36926
:0CA72400186804F0D2FB0028F9D010BD2A
:10A730009C2370B55B00C55C0400002D14D18369B7
:10A74000002B0CD01868002809D00368DB689847F4
:10A75000A36904211D60A06907F072FEA5610023B2
:0AA76000FC34E3622363636370BD01
:10A76A009C23F7B55B00C35C0400002B2AD180252B
:10A77A00FF276D00A369186804F088FB002821D020
:10A78A0007F0A1F9A369012218686B46DE1D036868
:10A79A0031005B6998472300FC335A6BAA420ED0FA
:10A7AA005A6BAA420BD02200D96A30782832505408
:10A7BA00DA6A01323A40DA625A6B01325A6307F0B6
:06A7CA0098F9D7E7F7BD86
:10A7D0009C2210B552000300805C002806D00120A6
:10A7E00001F0E0FE054801F06AFA10BD9B69002BFC
:10A7F000FBD01868431E9841C0B2F6E7F0950020E0
:10A8000070B504000D0001F05AFA030000208342E5
:10A8100004D0236829001B6C2000984770BD08B441
:10A82000024B9C46024BC01A08BC604701A80010AE
:04A8300040010000E3
:10A8340037B56B46DC1D9C2321705B00C35C0500AF
:10A84400002B04D0C9B20A48FFF7D8FF3EBDAB695C
:10A85400186804F03AFB0028F9D0AB6901221868A3
:10A86400210003681B6998470130431E9841EDE7B6
:04A87400F09500203B
:10A87800F7B5060001911700002401F01CFAA04268
:10A888000DD0A7420BD93D1B402D00D94025019B77
:10A898002A001919300000F039FF6419F1E7200087
:10A8A800FEBD08B4024B9C46024BC01A08BC604768
:08A8B80079A800104001000026
:10A8C0009C2370B55B00C35C05000E001400002BD8
:10A8D00005D00F48FFF7D0FF0400200070BDAB6922
:10A8E000186804F0F4FA0028F9D0AB6901211B685C
:10A8F00018005B6F74301B6B9847AB6922001868B7
:10A90000310003681B699847431CE6D10024E4E743
:04A91000F09500209E
:10A91400F0B5C3B0050001F0BBF9932380229B007E
:10A92400E918CB6852000400D31A984201DDCC68C0
:10A93400141B01AB220002A92800A82600F0E5FFA1
:10A944000021019802AB241A76001C19932380225B
:10A954009B00EB18DF685200974211D081420FD060
:10A96400DF6897420AD05A68675CAA1897555A68F4
:10A974000132D2B25A60DA680132DA600131E5E7B5
:04A9840043B0F0BD2F
:10A9880070B5040000F0A0FB2000FFF7BFFF932381
:10A998009B00E318DD68200000F09DFB280070BDD7
:10A9A80008B4034B9C46034BC01A08BC6047C0461A
:08A9B80089A900104001000014
:10A9C0009C2310B55B00C35C0400002B05D0064837
:10A9D000FFF7DAFF0400200010BDFC3407F078F820
:0CA9E000646B07F08BF8F6E7F0950020A0
:10A9EC0070B5040000F06EFB2000FFF78DFF932381
:10A9FC009B00E318DA68002A09D0A8229B68520051
:10AA0C00E3189D5C200000F064FB280070BD01255C
:10AA1C006D42F7E708B4034B9C46034BC01A08BCC5
:0CAA2C006047C046EDA90010400100008A
:10AA38009C2310B55B00C35C0400002B05D00B48B9
:10AA4800FFF7D0FF0400200010BD07F03DF82300F9
:10AA5800FC335A6B002A05D01B6B2834E45C07F0E2
:10AA680049F8F0E701246442F9E7C046F095002070
:10AA780070B5040000F028FB2000FFF747FF932380
:10AA88009B00E318DA68002A10D0A8219A684900C8
:10AA9800A218555C9A680132D2B29A60DA68013A13
:10AAA800DA60200000F017FB280070BD01256D4218
:10AAB800F7E708B4024B9C46024BC01A08BC604733
:08AAC80079AA00104001000012
:10AAD0009C2310B55B00C35C0400002B05D00E481E
:10AAE000FFF7CAFF0400200010BD06F0F1FF2300AD
:10AAF000FC335A6B002A0CD01A6B2834A45C1A6BF6
:10AB00000132D2B21A635A6B013A5A6306F0F6FF69
:0CAB1000E9E701246442F9E7F095002019
:10AB1C00802210B50400520000210CF08FFD2300A0
:0EAB2C000022FC335A6020009A60DA6010BDEF
:10AB3A0010B542680368086854100019D20701D595
:08AB4A000268D358984710BDC2
:0CAB520010B501000430FFF7EFFF10BD4C
:10AB600010B5024BC3601CC91CC010BDC42F02101D
:10AB700010B586B00400684603910092436004ABB0
:10AB800006C806C3200003A9FFF7EAFF200006B0AD
:02AB900010BDF6
:0CAB920013B50400FFF7EBFF200016BD18
:10ABA0009C2370B55B00C35C86B004000D00002BD5
:10ABB00036D18669002E04D1042007F011FCA06173
:10ABC0000660A369186800282CD1783007F008FCCB
:10ABD00006002223E25E2023E15E2B0004F05CFCF1
:10ABE000A3691E602423E25E531C06D0A0692621BF
:10ABF000635E0068032104F05DFCA3691D68002DFD
:10AC00000ED00026094A3300210002A8FFF7C1FF39
:10AC10002800320002A904F0BDF902A8FFF74BFD9D
:10AC200006B070BD290004F011F9DBE76BA7001036
:08AC300010B5FFF78EFF10BD07
:08AC380010B5FFF7F9FF10BD94
:10AC4000F7B51A4B1A4DFA260024083300932B60EF
:10AC50002023B600AE606C6016486B61AC61EC619D
:10AC6000FFF75CFF9C22012752002000AF5401F047
:10AC700073FC0190380001F06FFC20230E4D009909
:10AC80006B616B469B88AE602B84012368845B42BA
:10AC90006C600A482960AC61EC61AB84EB84FFF71F
:10ACA0003DFF9C225200AC54F7BDC046D02F02108D
:10ACB000E49900200C9A0020A8980020D098002049
:04ACC00000207047B9
:02ACC4007047D7
:02ACC6007047D5
:10ACC80010B5054BC458002C05D0236820005B68DC
:0CACD8009847A468F7E710BD8C05000049
:10ACE40070B50D00054BC458002C06D02368200015
:10ACF4009B6829009847A468F6E770BD8C0500009E
:08AD040000487047A030021066
:10AD0C0010B50400044B036005F024FF200005F08F
:0CAD1C00E1FF200010BDC04620300210F6
:10AD280010B50400FFF7EEFFB2212000C90007F0BC
:06AD380083FB200010BDAA
:10AD4000F0B50F4B0500C458002385B0019102AA4D
:10AD5000D61C002C12D023680199DF68320003ABA7
:10AD60002000B84731780300042905D0039A280051
:10AD700005F032F905B0F0BDA468E8E73178F5E7F1
:04AD80008C0500003E
:10AD840070B50E0005000021002A0CD10A4BC458EE
:10AD9400002C0ED0236800221B6931002000984744
:10ADA400002804D00121280004F0D4FE70BDA4685A
:0CADB400EEE72100F7E7C0468C05000028
:10ADC00070B50E0005000021074BC458002C07D0B9
:10ADD0002368310020005B699847A4680100F5E70B
:0CADE000280004F0C9FF70BD8C050000C5
:10ADEC00F8B505000E001700084BC458002C07D00E
:10ADFC00236820009B693A0031009847A468F5E766
:10AE0C002800012105F020F8F8BDC0468C05000093
:10AE1C00F0B5002187B0040005F0BEFA6B460022A5
:10AE2C00DA80238901A9A588E28889260B731B0A7D
:10AE3C004B730F4BEF27CB81042376000E80113E12
:10AE4C00FF3ECE704E710D728A72FF330A34013E92
:10AE5C002D0A120AC871CA720F718E714D720B8253
:10AE6C00122220000CF058FB200007B0F0BDC046A9
:04AE7C0001020000CF
:10AE8000F8B506000C000500002730000CF0DCFED1
:10AE9000AB1B984205D92B786770237001350234BB
:08AEA000F3E74000C0B2F8BD69
:10AEA80070B504000C4BC558002D07D02B6828003E
:10AEB8001B6A9847002802D1AD68F5E72800A92544
:10AEC800064BED006353064BE118FFF7D5FF635DB2
:10AED800C0186055601970BD8C05000002030000A1
:04AEE8004A05000017
:10AEEC0070B5A125064BED004353064B0400C11869
:10AEFC000548FFF7BFFF635DC0186055601970BD52
:0CAF0C00020300000A05000004300210DF
:10AF180070B59925064BED004353064B0400C01845
:10AF2800FFF798FB635DC0186055601970BDC04697
:08AF380002030000CA0400003E
:10AF40000023F0B587B003A98B71B123DB00C35C8C
:10AF500005000B7101234B71BF33CB713A330B7278
:10AF6000CE2309249B00154AC718039238000922F2
:10AF70000CF0D8FA124BEE58002E17D0336800218F
:10AF80001B6830009847C37882781B021343093B43
:10AF90000193CE2301009B00E01828180931019A83
:10AFA0000CF0C0FA019BB668E418E5E73800054BE1
:10AFB000EC54054B2412EC5407B0F0BD0902FFFF1E
:0CAFC0008C0500003A0300003B03000079
:10AFCC0073B504000D00160008F040F880235B00F8
:10AFDC00010000932A003300200005F029FE024BEB
:0CAFEC002000236076BDC046203002101B
:10AFF80010B50E4A04008358002B12D18150B1239A
:10B00800DB00E25C48790A71E25C1218E2540B68D2
:10B0180008005B6A9847238918182081012010BD11
:10B0280013009A68002AFBD19960E8E78C050000B4
:10B038001FB5040005F0AAF90100684604F000FBFA
:10B048004021684604F072FB074BE458002C06D0F8
:10B0580023682000DB6969469847A468F6E76846D4
:0CB0680004F0F5FA1FBDC0468C05000086
:10B0740010B50400FFF7DEFF200005F0FDF810BD59
:10B0840070B50D4D2B78BFF35B8F0C4CDB0711D4DF
:10B09400280006F09DFF00280CD0C022084920009B
:10B0A400FFF792FF280006F0B5FF064A0649200084
:10B0B40006F07AFF200070BD249B0020089E00202B
:0CB0C4008A2E0000400200200DAD00109C
:0EB0D00010B5FFF7D7FF03685B6F984710BD00
:0EB0DE0010B5FFF7D0FF03689B6F984710BDB9
:0EB0EC0010B5FFF7C9FF0368DB6F984710BD72
:08B0FA0010B504F054FC10BD78
:08B1020010B504F00AFC10BDB9
:08B10A0010B504F03AFC10BD81
:02B11200704784
:02B11400704782
:02B11600704780
:08B11800436A78331878704790
:06B12000FC30806A70475C
:04B12600012070474D
:08B12C000048704708320210D0
:10B13400F0B505009BB007AC4B220F0020000021A6
:10B144000CF080FA2B00FC339B6A05215A1E9341B4
:10B1540000202E795B421940731CDBB20193AB7B58
:10B1640002932B7B03936B7B0493874200D0A5E06F
:10B174006176534906A86183102161770B39E17721
:10B184002421471D0922F9772527627406A8053A68
:10B19400C019A274033A027006A8C71D0320494BC4
:10B1A400F8772380BF3BFF3BA370812308AFFA7776
:10B1B40004275B00A380823BE37162754E3B2276D9
:10B1C400A27706A80832121823722A3BD777637233
:10B1D4000A220333A3723C4B06A8A381022312184C
:10B1E400D1770591073706A97F18FB770627052134
:10B1F40009A8C77711A801702D2006A94018242199
:10B20400E672A373E674A375E37501702E2006A994
:10B21400401807702F204018694606700E7912A84E
:10B2240006703126072006A9761830703226761863
:10B2340005213170332606A9761869460F7A06A9C6
:10B244003770224E1027268637267618377009273E
:10B2540014AE377039260427761837703A267618D4
:10B2640069460F7906A93770194E1D352687412680
:10B27400761830703B30401805210170432106A830
:10B28400091868464426007B0870124906A88019EC
:10B29400018011492800D1874A2206A9521869461B
:10B2A400097C11704B2206A952181370402219AB65
:10B2B4001A7021000B320CF033F928001BB0F0BDDA
:10B2C40005240000090200000202000003400000FF
:0CB2D400020A0000024000000705000014
:10B2E00010B504000A4B08330360FFF7CBFE05F0EE
:10B2F00037FC2000D03004F0B6FA20007C3004F097
:10B30000B2FA2000703004F0AEFA200010BDC04642
:04B31000C031021036
:10B3140010B50400FFF7E2FF94212000490007F074
:06B324008DF8200010BDB1
:08B32A0010B5FFF7DEFE10BDB7
:10B3340010B50400024B036004F048F9200010BD6E
:04B34400E8300210DB
:10B3480010B50400FFF7F2FF2000282107F074F879
:04B35800200010BD04
:10B35C0010B50400024B036004F034F9200010BD5A
:04B36C00B8300210E3
:10B3700010B50400FFF7F2FF2000342107F060F859
:04B38000200010BDDC
:10B3840010B50400024B036004F020F9200010BD46
:04B39400D0300210A3
:10B3980010B50400FFF7F2FF2000382107F04CF841
:04B3A800200010BDB4
:10B3AC0070B50D000400072217490F300CF0B4F8EB
:10B3BC0040220221280004F0A9F940222073022126
:10B3CC00280004F0AAF9402260730321280004F03D
:10B3DC009DF9A073280004F039F9002804D1AF229C
:10B3EC000A490B4806F0C0FA2200210000237832EB
:10B3FC0085311165536513701373D934503213743E
:10B40C005465936570BDC04604310210A33102101F
:04B41C00AE3102103B
:10B42000F0B504000E0087B01500FFF75FFEF2884C
:10B4300023799A4236D1002D34D173780593012BAC
:10B440002DD1F378202B26D13789072F23D1230044
:10B450000F33039307333A001900039804930CF059
:10B460003BF8059D002816D03A00049903980CF08B
:10B4700059F8217CE07B09020918607CE77C000414
:10B480000918A07C0097000609182068237D476BE7
:10B49000627D2000B847F378212B00D101252800D8
:08B4A00007B0F0BD0025FAE73A
:10B4A80070B50400FFF71EFEFFF7E8FD217B05F0ED
:10B4B800DDF923002200C833853225001A602000F8
:10B4C80000234732843513607C302B7004F07FF9F9
:10B4D8002B78002B03D123682000DB6B984770BDC5
:10B4E80070B504002500FC35FFF7FCFD6E6A002EE0
:10B4F80005D0DE220E49FF320E4806F037FA230047
:10B50800D9332B62FFF7BAFD617B05F001F9686258
:10B5180025002000D8352E70D03004F058F92B784B
:10B52800002B03D1236820009B6B984770BDC04651
:08B53800A331021010310210D2
:06B540000023C360704708
:10B54800022370B543710023040083600C4B15007F
:10B5580008330360703004F02DF920007C3004F0CB
:10B5680029F92000D03004F025F92300FC339D622E
:10B57800FFF784FD2100FFF73BFD200070BDC046AA
:04B58800C0310210BC
:10B58C0070B504000D00FFF7ABFD230078331D7080
:10B59C00002D42D1260084363378002B05D0FFF7DE
:10B5AC006BFD217B04F014FF357023002200250075
:10B5BC000026C83385327C3528001A605E6004F0A2
:10B5CC0004F9280004F0FAF8B04205D1A22215497A
:10B5DC001548520006F0C8F92500D8352B78002BF9
:10B5EC0005D0FFF749FD217B04F0F2FE2E702300FD
:10B5FC002200FC33D93225001A620022D0352800F3
:10B60C005A6204F0E2F8280004F0D8F8002804D1BB
:10B61C00A722044952000548DCE72000703004F0F2
:10B62C00D4F870BDA33102101E3102102F3102105C
:10B63C0010B50400FFF754FD00212000FFF7A0FF18
:02B64C0010BD2F
:10B64E0070B50D000400FFF74AFD042D03D0002154
:08B65E002000FFF794FF70BD0E
:10B66600F8B5040016000D001F00FFF73CFD04238B
:10B676003370EA88237900209A4210D16A78012A29
:10B686000DD1EB78212B06D0222B09D0202B19D1F6
:10B696003070163401E032700F3407203C60F8BD7C
:10B6A600A988114000D011002000FFF76CFF01228D
:10B6B600AB8800201340E366AB8892181340A3665C
:0AB6C6003270ECE703233370E9E76C
:10B6D00010B504008AB0FFF7FBFC684603F068FF72
:10B6E00020000A4B694670300093099404F08AF8F0
:10B6F0002000FFF7F4FC064B00211A68684603F0AF
:10B700001DFF6846FFF716FE0AB010BDE8300210B4
:04B710000C310210E6
:10B7140070B504000E008EB01500FFF7D7FC01A829
:10B7240003F044FF20000B9600260D4B01A90C9555
:10B734007C300DAD01930A942E7004F061F8200062
:10B74400FFF7CBFC074B31001A6801A803F0F4FEA5
:10B754002C7801A8FFF700FE20000EB070BDC04693
:08B76400B83002100C31021094
:10B76C0070B5040025008435FFF7BAFC2B78002B4C
:10B77C0010D12600CC363368002B0BD0FFF77CFCA5
:10B78C002200217B8532336805F002F8002801D0B5
:06B79C0001232B7070BDBB
:10B7A200F0B585B01F000AAB1B7804000393029129
:10B7B2000192FFF78CFC00233B60230078331B7857
:10B7C200002B21D0230084331B78002B1CD12600B0
:10B7D2004025CC363368ED1A019B9D4200D91D00ED
:10B7E200019B002B06D02300C83318682A00029957
:10B7F2000BF097FE33685B193360039B3D60002BAF
:10B8020002D02000FFF7B1FF2000FFF767FC05B070
:02B81200F0BD87
:10B81400F0B50400406A85B0030078331D78012632
:10B82400002D05D1303425703500280005B0F0BD59
:10B834000027009603ABE26AA16A0397FFF7AFFF04
:10B84400039AE36AA16A9B1A8A18E362A262BB4262
:10B8540002D130342670E8E7606AFFF785FF3D00C7
:02B86400E3E718
:10B86800F0B51C0093B0019205000F00FFF72CFC07
:10B8780063426341DBB20093002C00D103AC002685
:10B8880004A8266003F090FE6A46109428003D2420
:10B898000F4B12780493019B04A90F9311AB1A70F4
:10B8A80002ABE418D03026700D950E9703F0A6FF72
:10B8B8002800FFF710FC074B31001A6804A803F0B2
:10B8C80039FE247804A8FFF759FD200013B0F0BD15
:08B8D800D03002100C31021007
:10B8E000030070B5FC335B6A0400002B0ED1050029
:10B8F000D8352B78002B09D1FFF7C4FB2200402359
:0EB90000D932617B04F0A6FE01232B7070BDCE
:10B90E00F8B506001F0000233B60330078331B7828
:10B91E000800002B19D03300D8331B78002B14D11C
:10B92E003400FC34656A954200D915002A00216A5C
:10B93E000BF0F1FD3D60236A5B192362636A5D1BA8
:0CB94E00656202D13000FFF7C4FFF8BDB5
:10B95A0037B50400406A030078331D78002D04D1FE
:10B96A0035342570013528003EBD0023E26A019373
:10B97A00A16A01ABFFF7C6FF019BA26AD218A262B5
:10B98A00226B1168CB181360E36A01995B1A2100D4
:10B99A00E36234310978002902D11268002A01D100
:10B9AA00002B03D1012335342370DCE7606AFFF7EB
:06B9BA0092FF0025D7E713
:0EB9C00010B504000021FFF7BBFD200010BDF4
:0CB9CE0010B50400FFF7F5FF200010BDCD
:10B9DA0010B542680368086854100019D20701D5E7
:08B9EA000268D358984710BD14
:0CB9F20010B501000430FFF7EFFF10BD9E
:10BA000010B5024BC3601CC91CC010BDF830021039
:10BA100010B586B00400684603910092436004AB01
:10BA200006C806C3200003A9FFF7EAFF200006B0FE
:02BA300010BD47
:0CBA320013B50400FFF7EBFF200016BD69
:10BA4000F0B58BB00400FFF751FBFFF71BFB0600BE
:10BA500006ADA77B00212800FFF7B9FF39000323BB
:10BA600040220095300004F025FC2800FEF723FE5C
:10BA7000FFF708FB0700267B21002800174A002358
:10BA8000FFF7D7FF3100022340220095380004F071
:10BA900011FC2800FEF70FFEFFF7F4FA0600677BA3
:10BAA000210028000E4A0023FFF7C3FF39000223BC
:10BAB00040220095300004F0FDFB2800FEF7FBFD5E
:10BAC000FFF7E0FA2200FC32617B4023126A04F0A7
:10BAD000C1FD0120D83420700BB0F0BDA9B4001016
:04BAE000E9B40010B5
:08BAE40010B5FFF784FF10BD4F
:08BAEC0010B5FFF7F9FF10BDD2
:06BAF400162040427047DD
:0ABAFA000020814200D11938704786
:04BB04000120704765
:06BB0800162040427047C8
:06BB0E00162040427047C2
:04BB14001120704745
:02BB1800704774
:02BB1A00704772
:02BB1C00704770
:10BB200010B503689B6C984710BD08B4024B9C4647
:10BB3000024BC01A08BC604721BB00104001000046
:04BB40007047704793
:04BB4400704770478F
:10BB480010B504000120783400F028FD207810BDDD
:10BB580008B4034B9C46034BC01A08BC6047C04658
:08BB680049BB00104001000080
:10BB7000012270B501235242FF210B4806F0FAFD65
:10BB800000F000FD0500094C78342378002B03D029
:10BB9000012000F007FDF8E700F0F4FC401BC72887
:10BBA000F6D9FEF76BFD70BDC89B0020F095002014
:10BBB00007B50122019101A9FFF7ACFD002801D0D2
:0ABBC00001980EBD01204042FBE792
:10BBCC0008B4034B9C46034BC01A08BC6047C046E4
:08BBDC00B1BB001028010000BC
:10BBE40013B56B46DC1D0023012221002370FFF7EF
:10BBF40039FE002801D0207816BD01204042FBE721
:10BC040008B4034B9C46034BC01A08BC6047C046AB
:08BC1400E5BB0010280100004F
:10BC1C00F7B5040001930E001500FFF761FA9C23A1
:10BC2C009B00E758002F04D0089B019A2900300094
:10BC3C00B84798239B00E650019A0433E55004332F
:0ABC4C00E250089A0433E250F7BDFD
:10BC5800962310B5DB00984203D10121014806F074
:08BC680067FD10BDC89B002020
:04BC700000687047B1
:04BC74000C307047D9
:0CBC780010B5FFF7FBFF0023036010BDB8
:10BC8400CB6810B5C360002B01D05B68984710BD2A
:10BC940070B50500FFF71AFA2B000024D8331B787F
:10BCA400A34205D12B00FC335C6A402C00D940240C
:0ABCB4002800FFF712FA200070BD0F
:06BCBE00783000787047A9
:10BCC400F0B585B003930AAB1E880BAB04001F8844
:10BCD4000D00029207F0BEF9039B0100029A01973E
:10BCE40000962000FFF72EFC200029300021FF30B1
:10BCF40005F06EFC2300FA2200264133FF33920044
:10BD04005E609A60184B194A23602300FC33DA62A0
:10BD1400174A20001A63174A51305A6480223100AE
:10BD2400FF3052000BF08EFC93239B00E3185E60FF
:10BD34009E60DE609D239B00E6184033E7183000C8
:10BD44001036FFF73BFEBE42F9D1AD22002392002C
:10BD5400A350443AA3509D4202D02000FFF7B6FC02
:10BD6400200005B0F0BDC046DC320210543302108E
:08BD7400B4330210C4330210C5
:10BD7C00104B70B5036003000F4AFC33DA620F4AB4
:10BD8C0004001A630E4A5A649D239B00C618403364
:10BD9C00C518AE4204D0103D2800FEF786FCF8E72B
:10BDAC0020002930FF3005F03BFC2000FFF792FA11
:10BDBC00200070BDDC32021054330210B433021078
:04BDCC00C43302106A
:10BDD00008B4034B9C46034BC01A08BC6047C046DE
:08BDE0007DBD001028010000E8
:10BDE80008B4034B9C46034BC01A08BC6047C046C6
:08BDF8007DBD00102C010000CC
:10BE000010B50400FFF7BAFFAE212000890006F04C
:06BE100017FB200010BD2D
:10BE180008B4034B9C46034BC01A08BC6047C04695
:08BE280001BE00102C01000016
:10BE300008B4034B9C46034BC01A08BC6047C0467D
:08BE400001BE00102801000002
:10BE480070B504000D00884205D0FEF729FC2900D2
:0ABE58002000FFF713FF200070BD6B
:10BE620010B5FFF706FF0068431E9841C0B210BD2F
:10BE740010B50400FFF7F3FF002804D1054A064972
:10BE8400064805F075FDE068FFF7F0FE03002000AA
:10BE9400984710BD02020000BD320210C8320210E1
:10BEA400F8B5AD2706000025FFF71EF9BF00F359CA
:10BEB400AB420ED99D2292002B01B418E418200045
:10BEC400FFF7CDFF002804D02000FFF7D1FF013594
:04BED400EDE7F8BDE1
:10BED80010B5044B0822C3600B68002108C00BF0A2
:08BEE800AFFB10BD2C3202106B
:10BEF00013B504000191002903D1FFF7BDFE200016
:0ABF000016BD01A9FFF7E8FFF9E7FD
:10BF0A0010B542680368086854100019D20701D5B1
:08BF1A000268D358984710BDDE
:0CBF220010B501000430FFF7EFFF10BD68
:10BF300010B5024BC3601CC91CC010BD20320210DA
:10BF400010B586B00400684603910092436004ABCC
:10BF500006C806C3200003A9FFF7EAFF200006B0C9
:02BF600010BD12
:0CBF620013B50400FFF7EBFF200016BD34
:10BF700030B589B00400FFF7ABF89C23274A9B003B
:10BF8000E2502000FFF7ABF80023254A210004A867
:10BF9000FFF7E7FF2000FFF79BF8AD239B00E05879
:10BFA000032808D8421CE2500001403BC01820186A
:10BFB00004A9FFF749FF2000FFF791F804A8FEF756
:10BFC0007AFBBC2006F00CFA0500164B08C0FFF700
:10BFD000F7FC28000021403006F058FC28005430BF
:10BFE00006F0F0FB8022104B520000932800002343
:10BFF000182106F0C9FC97239B00E5500B4904A8C3
:10C00000FFF776FF04A9280006F0C8FC04A8FEF795
:10C0100052FB2000FEF77EFC09B030BD59BC001079
:10C0200015A90010CC4702103832021071BB001065
:10C0300008B4034B9C46034BC01A08BC6047C0467B
:08C0400071BF00104001000077
:08C0480010B50368984710BD14
:08C0500010B5FFF7F9FF10BD68
:08C0580010B5FFF762FF10BDF7
:08C0600010B5FFF7F9FF10BD58
:10C0680037B50E4C200006F059FB0D4D0D492A003E
:10C07800200005F097FF012201920B4AF823009255
:10C0880000220A4C5B0111002000FFF717FE2A006E
:10C098000749200005F086FF37BDC046C89B002031
:10C0A800400200204327011012200000F0950020D4
:04C0B8007DBD00103A
:06C0BC0010B509F0DBFEE7
:10C0C200F0B589B00191037D0400012B00D08AE014
:10C0D200021D0292100001220493002352421C000E
:10C0E2001500049E03920178002900D06EE0417889
:10C0F200002900D06AE0511C65D001335BB204997B
:10C102008B4201DD049303920134E1B202304CB25E
:10C112000829E8D100263700039BBB4204DC049BBC
:10C12200039A9B18BB4253DC0F22029B1D782B11F2
:10C132001540029ADCB25278111107916946097FC3
:10C1420005910F2111400691002B08D02100573193
:10C15200092B00DC2739019800F0D2F836182C435D
:10C1620008D029005731092D00D82739019800F04D
:10C17200C7F83618059B1C430AD01900079B573194
:10C18200092B01DC05993031019800F0B9F8361815
:10C192000699069B5731092B01D8190030310198B5
:10C1A20000F0AEF83618072F04D03A21019800F0BB
:10C1B200A7F83618029B013702330293082FABD13E
:10C1C200300009B0F0BD2200330098E72A009BE757
:10C1D200039BBB42EED1002BE7D13A21019800F03C
:10C1E2008FF83618E1E703000500002613331035F7
:10C1F200029329780A22019800F0D3F82E21070031
:10C20200019800F07DF8029B3F180135F6199D4216
:10C21200EFD1E17C0A22019800F0C3F83618CFE78B
:10C2240010B50400054B017508330360102200218A
:10C2340004300BF007FA200010BDC046F0330210A2
:10C24400F7B50F0000211D0008AB1B780400019313
:10C25400084B16000833036001750C2204300BF000
:10C26400F1F96B461B7927746674A5742000E37496
:08C27400FEBDC046F0330210CC
:10C27C0007B501210548FFF7CFFF002104480091C5
:10C28C000B000A00FFF7D8FF07BDC046489C0020F2
:04C29C00609C002082
:10C2A000F7B506000D000C008B180193019B671B6E
:10C2B0009C4207D0336821781B68300098470134CE
:08C2C0000028F3D13800FEBD97
:10C2C80070B5040008000D000BF0BAFC23680200EA
:0AC2D80029005B682000984770BD44
:10C2E20010B50B1E02D0FFF7EEFF0300180010BDC1
:08C2F20010B5FFF7F5FF10BDC8
:08C2FA0010B5FFF7F1FF10BDC4
:0AC3020010B503681B68984710BDD2
:10C30C0010B50249FFF7DAFF10BDC046FC3302102E
:10C31C0070B50400FFF7DFFF05002000FFF7F0FF0A
:04C32C00401970BD87
:10C3300070B50400FFF7D5FF05002000FFF7E6FF0A
:04C34000401970BD73
:10C34400F0B58BB06B461500002205330600DA7792
:10C354000800012D00D80A2509AC2900F4F712F9C8
:10C36400CAB2130037330700DBB2092902D813001D
:10C374003033DBB2013C2370002FEED121003000BA
:08C38400FFF7ADFF0BB0F0BDA7
:10C38C0010B5002A04D10368C9B21B68984710BDC8
:08C39C00D2B2FFF7D1FFFAE76E
:08C3A40010B5FFF7F1FF10BD19
:10C3AC0070B50500FFF7ECFF04002800FFF7A8FFAD
:04C3BC00201870BD18
:10C3C00010B504000068002801D00AF07BFD2000B1
:02C3D00010BD9E
:10C3D20010B504000068002801D00AF072FD0023A5
:08C3E2002360A360636010BD3D
:10C3EA0070B504000D00006801310BF0F6F9031E68
:08C3FA0001D0012028C470BD30
:10C40200036810B50400002B04D043688B4201D3AB
:10C41200012010BD2000FFF7E7FF0028F9D0A36834
:0AC42200002BF5D122681370F3E738
:10C42C0070B50E00110004001500FFF7E4FF0028A2
:10C43C0004D12000FFF7C7FF200070BD2A00310097
:10C44C00A56020680BF068F800232268A16853549B
:02C45C00F2E705
:10C45E00002370B504000D000360436083609942B1
:10C46E0007D008000BF0E9FB290002002000FFF7BF
:06C47E00D6FF200070BD96
:10C4840010B50B000400884205D00968002904D0C7
:10C494009A68FFF7C9FF200010BDFFF798FFFAE77D
:10C4A400F0B50C008BB01600002926D0931E222B69
:10C4B4002DD80A2A05D1002803DA0127404201AD0C
:10C4C4000AE00027FBE73100F4F75CF8CBB2092956
:10C4D40016D830332B7001352A000028F3D101AB74
:10C4E400AB42F0D02300002F02D02D21631C217019
:10C4F40001A98A4206D800221A7020000BB0F0BDB0
:10C504005733E7E7013A117819700133F0E7002453
:02C51400F3E74B
:08C5160010B5FFF7C4FF10BDD2
:10C5200010B500F047F8FEF798F8FEF7ABFDFEF700
:10C53000A1FDE12106484902FFF71AFDF7F7AEFB1E
:10C54000F7F7E8FA034B002BFAD000E000BFF7E75B
:08C55000F0950020000000003E
:10C5580010B50400FEF77BF8844203D2034B240194
:10C56800E05E10BD01204042FBE7C04648020020C3
:0CC5780010B5040002F048FE200010BDC9
:10C5840007B50649684602F080FE00980199FA2230
:10C5940000239200F4F794F90EBDC0466010002009
:08C5A40010B506F0A5F910BD69
:08C5AC0010B506F08FF810BD78
:10C5B40010B5044C200002F035FE200002F032FEDB
:08C5C40010BDC046601000200C
:08C5CC0010B506F0A3F910BD43
:10C5D40010B5054C200002F095FE044A04492000E1
:10C5E40005F0E2FC10BDC0466010002040020020AF
:04C5F40079C50010F5
:10C5F800F7B504000D00FEF72AF884422ED21A4E31
:10C608002701F319D868002802D0042105F014FF87
:10C618002000FFF79DFF0190042005F0DDFE0023B8
:10C628000400038083700199F61904F00AFCF46091
:10C63800012D10D0002D06D0022D10D0200002F0C0
:10C64800C4F9022103E0200002F0BFF9290020000C
:10C6580002F0C6F902E0200002F0ACF9F7BD2000B4
:0CC6680002F0B3F90121F2E748020020C3
:10C67400F7B507000E00FDF7ECFF87421AD20E4D06
:10C684003B01ED18EC68002C10D13800FFF762FF75
:10C694000700042005F0A2FE002304000380837039
:10C6A40001220096390004F0DEFBEC60310020002A
:0CC6B40006F0F0FCF7BDC0464802002074
:10C6C000F7B50500FDF7C7FF002485421AD20E4FCB
:10C6D0002B01FF18FE68A64210D12800FFF73CFF8F
:10C6E0000500042005F07CFE060004808470230011
:10C6F00000942200290004F0B8FBFE60300006F030
:0CC70000D7FCC4B22000FEBD480200209F
:10C70C00010010B5002807D10420404200F0D3F9F5
:10C71C0004235B42180010BD132001F0E5FD00233B
:10C72C009842F7D10120404200F0C5F90123F0E70F
:10C73C0080B5EFF30583002B03D1EFF31083002BAF
:10C74C0006D00620404200F0B6F90620404280BDDB
:0CC75C00014F00DFFBE7C0460DC70010D6
:10C76800030010B500282BD00468806800280FD07B
:10C77800032102000A40084203D1D96813000F2997
:10C7880013D809210020494202F06CF8002016E075
:10C79800DB68002BF5D1104A104B1068002811D027
:10C7A80000F04CFB002814D00123F32283700023EF
:10C7B80002708360C3600A4A084B44605A6610BD21
:10C7C8000400E8E7043301221021D86F00F0BBFA17
:10C7D800E8E705214942D7E7B804002028040020EB
:04C7E800B9C80010BC
:10C7EC0070B5041E02D00378F32B07D0042120006F
:10C7FC00494202F035F80420404270BD8368002B9A
:10C80C000DD003256D42200001F020FB00222900F1
:10C81C0001F0C6FCA0680028F5D101F0A9FB0023AB
:10C82C002370A378DB0701D40020E6E7074A084B06
:10C83C001068002803D0210000F011FBF4E704334A
:10C84C002100D86F00F0B1FAEEE7C046B804002022
:04C85C00280400208C
:10C8600070B50300022510000124284014402A421C
:10C8700014D1EFF3108672B6DA6815000D40002C63
:10C8800006D0A94206D110008843D860100001E00C
:10C89000281EF8D1002E00D162B670BDD8680B00FA
:10C8A0000340002C03D09942F7D00020F5E75A1E30
:08C8B00093415B421840F0E7E0
:10C8B800F8B505008468002C00D1F8BD231D2800B8
:10C8C800DA7F616AA768FFF7C7FF061E07D0200056
:10C8D80001F0C8FA00223100200001F063FC3C009E
:02C8E800E9E77E
:10C8EC00F8B504000D0016001F00002804D00378D2
:10C8FC00F32B01D1002907DA04212000494201F071
:10C90C00AFFF04204042F8BDFFF7A4FF0028FAD186
:10C91C00002F10D03900433001F0E6FC002808D07D
:10C92C00064B20005F69390001F07AFA04373D624A
:10C93C00FE770220E6E70320E4E7C0462804002047
:10C94C00F7B506000C00002804D00378F32B01D1B6
:10C95C00002908DA042130000424494201F080FF48
:10C96C0064422000FEBDEFF3108372B6C26814431C
:10C97C00C460002B00D162B6B568002D03D128002D
:10C98C0001F0F6FAEDE7AB68300000932B1D019334
:10C99C00DA7F696AFFF75EFF071E0FD002222B1D9C
:10C9AC00DB7F0400134201D16B6A9C43280001F029
:10C9BC0057FA00223900280001F0F2FB009DDCE759
:10C9CC0080B5EFF30583002B03D1EFF31083002B1D
:10C9DC0006D006210020494201F042FF002080BD14
:0CC9EC00014F00DFFBE7C04669C70010E8
:10C9F800B0B5EFF30583002B03D1EFF31083002BC1
:10CA08001AD0002804D00378F32B01D1002907DAC3
:10CA180004210424494201F025FF64422000B0BDEE
:10CA2800EFF3108372B6C4680C43C460002B00D1C6
:10CA380062B601F0F5F8F1E7014F00DF0400EDE719
:04CA48004DC90010C4
:10CA4C00B0B5EFF30584002C03D1EFF31084002C68
:10CA5C0015D0002806D00478F32C03D1002B01D17B
:10CA6C00002906DA0421494201F0FAFE0420404272
:10CA7C0007E0FFF7EFFE002803D10320F7E7014F93
:08CA8C0000DFB0BDEDC8001091
:10CA940080B5EFF30583002B03D1EFF31083002B54
:10CAA40006D00621494201F0DFFE0620404280BD47
:0CCAB400014F00DFFBE7C046EDC700109B
:02CAC0007047BD
:02CAC2007047BB
:10CAC40070B5514C237A012B00D19AE0002B06D08B
:10CAD4000120404201F0B8FE0120404270BD4B4DA0
:10CAE400EB682A8AE3652300EE6A54331A80AB6844
:10CAF4003000296B236400F00DF9002801D0231DB8
:10CB0400DE676E69A969300000F004F9002801D1DC
:10CB1400231DDE6F6667EE69296A300000F0FAF8BB
:10CB2400002801D1231DDE6FA6676E6AA96A300052
:10CB340000F0F0F8002801D1231DDE6FE6676E6B6C
:10CB4400002E08D0F3683000B268316800F051F963
:10CB540023000833DE67AE6B002E08D0F368300084
:10CB6400B268316800F045F9230088331E60EE6B2B
:10CB7400002E08D0F3683000B268316800F039F94B
:10CB840023008C331E602E6C002E08D0F368300016
:10CB9400B268316800F02DF9230090331E606E6C8A
:10CBA400002E08D0F3683000B268316800F021F933
:10CBB400230094331E60AE6C002E08D0F36830005E
:10CBC400B268316800F015F9230098331E60EE6CEA
:10CBD400002E08D0F3683000B268316800F009F91B
:10CBE40023009C331E602D6D002D08D0EB682800B7
:10CBF400AA68296800F0FDF82300A0331D60012312
:10CC0400237200206AE7C0462804002014C80110DB
:10CC1400F8B51E4C0720257A012D04D101F0ACFB98
:10CC2400002807D101200126404201F00DFE764282
:10CC34003000F8BDFF23164A1B04116A154F0B433D
:10CC44001362136AD1695B029B0E9B060B437868DF
:10CC54001149D36101F084FC061EE3D101F0C4FC48
:10CC6400206101F0A5FC0D4801F0F4F801F07CF915
:10CC74003B682B4207D0022383F31488BFF36F8FE2
:10CC840002232372D4E70323F6E7C04628040020D6
:10CC940000ED00E014C80110D50300104404002086
:02CCA4007047D7
:10CCA60070B50D000400FFF708FF2900200001F011
:04CCB60084FD70BDCC
:10CCBC0080B5FFF7F1FFEFF30583002B03D1EFF302
:10CCCC001083002B06D00620404201F0B9FD06204F
:10CCDC00404280BD014F00DFFBE7C046C5CA0010D3
:10CCEC0080B5EFF30583002B03D1EFF31083002BFA
:10CCFC0006D00620404201F0A3FD0620404280BD34
:0CCD0C00014F00DFFBE7C04615CC001013
:10CD1800030010B5002813D002000A4307241000AE
:10CD2800204022420DD117290AD91022196008394A
:10CD3800C91899605A60086099684A60D8600120EB
:06CD480010BD0020FCE715
:10CD4E000300F0B5002815D0081E13D00020032ACA
:10CD5E0010D81D0003260F310730814308352C00F3
:10CD6E002D686768281BB743C01B814203D928680A
:10CD7E000028F4D1F0BD58681E68081858609B1939
:10CD8E00083B5E68B04200D9586060680A430028CC
:10CD9E0003D1200062600830ECE70323984320188B
:08CDAE00056042602060F6E719
:10CDB600020010B5002811D0081E0FD01300002461
:10CDC600083908338B420AD10321586888435168D1
:10CDD600091A5160002C08D15C60012010BD18684A
:10CDE6001C000028FAD00300ECE71B682360F4E778
:10CDF60030B504000800002C1BD0002914D0002AEE
:10CE060019D0002B19D02160002161601100414327
:10CE16005D18A260E360636125611C00013800288B
:10CE260003D1891A5850013030BDA51825602C0051
:0ECE3600F4E72000F8E71000F6E71800F4E734
:10CE4400EFF3108100280BD072B64369002B04D095
:10CE54001A684261426801324260002901D0180018
:06CE6400704762B6FBE717
:10CE6A00EFF31082002811D0C3688B420ED80369F1
:10CE7A008B420BD972B643690B6043684161013B2F
:10CE8A004360002A00D162B6002070470420404265
:02CE9A00FBE7B4
:10CE9C0070B5EFF31085036B002B1DD00024CE78FA
:10CEAC00DA78B24210D31A004A608C60002A11D092
:10CEBC009160002C13D0616072B6836A0133836277
:10CECC00002D00D162B670BD5A681C00002AEBD050
:10CEDC001300E5E7C162ECE74B608B60C162016354
:02CEEC00EAE773
:10CEEE00EFF3108272B6836A002B13D0013B83627C
:10CEFE00002A0DD00123C06A00280ED072B68178A8
:10CF0E008370002A00D162B6002907D08068F3E74B
:0ECF1E0062B6EFE7002A00D162B6002070472D
:10CF2C004B688A68002B05D09A608A68002A03D067
:0CCF3C0053607047C262F8E70363FAE735
:10CF4800F8B587780400002F31D0C56800262F0077
:10CF580001000C372800FFF7E5FF21003800267094
:10CF6800FFF77FFFAB68B34246D03800FFF766FF94
:10CF78000400B04240D0280000F06AFF07003200E9
:10CF8800310001F00FF9380000F0E8FF0700200039
:10CF9800B9686A6A0C300AF0C1FAF923A6702370DE
:10CFA800FB68E37021002800FFF774FF24E0856820
:10CFB800AB68002BF6D05B78832BF3D1280000F008
:10CFC80047FF06003A00390001F0ECF8300000F0A5
:10CFD800C5FF210006006A6A80680C310AF09EFAD3
:10CFE800F368002B01D0E2781A7000232800210092
:0ACFF80023700C30FFF735FFF8BD81
:10D00400F0B587B017000190029100280AD00029DA
:10D0140008D0F3F737FC04000298F3F733FC001947
:10D024001F2808DC04210020494201F037FC0024B9
:10D03400200007B0F0BD0322029B033393430C335B
:10D0440005930599019B4B430393002F21D03B6823
:10D05400BC683D697E690493002C06D0144202D159
:10D06400FB68332B04D80921DDE7FB68002BFAD1D8
:10D07400002D09D003222B001340154202D1039A3C
:10D08400B24253D90A21CEE7002EFBD1002C0FD196
:10D0940001E03D000497274A274B106800281BD065
:10D0A400FFF7CEFE041E15D00123002D27D11E004C
:10D0B400214F00220399F86FFFF747FE051E18D190
:10D0C400002E07D03B00A033186800280BD02100A5
:10D0D400FFF7C9FE0521A6E7043301223421D86FE6
:10D0E400FFF733FEDEE704372100F86FFFF761FE38
:10D0F400F0E70021039A0AF0A5FA02233343FA2247
:10D10400A370049B2000636000232270029AA36032
:10D114006262A362059AE362236301992B000C30D7
:10D12400FFF767FE044B054A1A6781E7002CE6D136
:10D13400B1E7C046C80400202804002049CF0010ED
:10D14400F7B504000E0017000193002804D00378FB
:10D15400FA2B01D1002907D104212000494201F012
:10D164009DFB042040421AE08368002B18D05B78B2
:10D17400832B15D100F06EFE05000122002101F081
:10D1840013F8280000F0ECFE050031008068626AA4
:10D194000AF0C6F9EB68002B00D01F700020FEBD1A
:10D1A4000C30FFF74DFE051E0ED03100626A0C30C4
:10D1B4000AF0B6F9F9232B70002329002000AB7084
:10D1C400EF70FFF769FEE9E7019B0320002BC9D04C
:10D1D4001900932001F08CF8002801D10220C1E746
:10D1E400044B2000596900F01FFEEFF309839E6091
:08D1F400DF60F3E728040020CE
:10D1FC00F7B504000F0016000193002804D0037843
:10D20C00FA2B01D1002907D104212000494201F059
:10D21C0041FB042040421DE0FFF763FE051E3BD09E
:10D22C0001002000FFF77CFE29003800626A0C31F7
:10D23C000AF072F9002E01D0EB783370270000262B
:10D24C000C37290038002E70FFF709FEA368B34293
:10D25C0001D10020FEBD3800FFF7EEFD051EF8D011
:10D26C00200000F0F3FD07003100012200F098FFD0
:10D27C00380000F071FE07002800B968626A0C30B3
:10D28C000AF04AF9F923AE702B70FB6829002000D4
:10D29C00EB70FFF7FDFDDCE7019B0320002BB9D001
:10D2AC001900832001F020F8002801D10220B1E7F9
:10D2BC00044B2000596900F0B3FDEFF309839F6024
:08D2CC00DE60F3E728040020F6
:10D2D400064B10B59A6ED86E0821FFF791FE044BE9
:10D2E400D86443425841404210BDC04614C801109E
:04D2F40028040020EA
:10D2F800F7B506001C0000910192EFF30583002B9F
:10D3080003D1EFF31083002B29D0002E07D03378F8
:10D31800FA2B04D1009B002B01D0002C07D004214C
:10D328003000494201F0B8FA0420404216E03000CB
:10D338000C30FFF783FD051E17D0726A00990C3078
:10D348000AF0ECF8F9232B70019B2800EB70009B86
:10D35800AC706B60AE6000F063FC2000FEBD230083
:10D368000099019A024F00DFF8E70320DDE7C04685
:04D3780045D100108B
:10D37C00F7B5040016000191EFF30582002A03D1E2
:10D38C00EFF31082002A26D0002C07D02278FA2A3C
:10D39C0004D1019A002A01D0002B07D004212000CF
:10D3AC00494201F077FA0420404213E02000FFF7D5
:10D3BC0098FD051E14D00100626A01980C310AF028
:10D3CC00ABF8002E01D0EB7833702800EC6000F045
:10D3DC0025FC0020FEBD32000199024F00DFF9E769
:08D3EC000320E1E7FDD1001070
:10D3F400030070B5002837D00468456880680028A9
:10D404000FD0032102000A40084203D1D968130057
:10D414001B291AD809210020494201F02DFA0020C5
:10D424001EE0DB68002BF5D1114A124B106800286E
:10D4340006D1043301221C21D86FFFF786FC01E0DA
:10D44400FFF7FEFC00280CD00123F5228370002393
:10D454000270C57044608360C360036143610376F6
:10D4640070BD05214942D8E704000500DCE7C04649
:08D47400BC0400202804002084
:10D47C002A4B70B55D6904000E00002D06D1082101
:10D48C00494201F0F5F90120404219E0002802D090
:10D49C000378F52B06D004212000494201F0E8F96D
:10D4AC000420F1E7037E002B0BD10361EB6AC5600E
:10D4BC004361002B00D018610123EC62002023761D
:10D4CC0070BDC278D1070CD5C168A94209D1FF2B18
:10D4DC0005D11021494201F0CBF90320D4E70133E7
:10D4EC00ECE7002EF9D092070BD51F221F21E06824
:10D4FC006B1C9A56431C5956914202DADA7700F0AB
:10D50C00BAFC3100532000F0EFFE002801D10220BC
:10D51C00BAE72900200000F083FCF8E7280400207B
:10D52C00354B70B55B690400002B06D108214942CC
:10D53C0001F09EF9012040421FE0002802D0027841
:10D54C00F52A06D004212000494201F091F904206B
:10D55C00F1E7027E0F21002A03D0C168994206D060
:10D56C000E212000494201F083F90320E3E7013A40
:10D57C00D2B20276002A01D0002070BD4269002A86
:10D58C0001D0016911612169002922D04A61022070
:10D59C009A1CD27FDD6A52B2002D1CD10133DA778E
:10D5AC00A368002B11D0200000F050FC06002A00CC
:10D5BC00290000F0F5FDF36AE66025616361002B3C
:10D5CC0000D01C610123F4622376002000F0D0FC13
:10D5DC00D2E7DA62DBE7E97801420AD0A9680029D0
:10D5EC0007D00131C97F0E1C49B2914200DA161CDA
:0CD5FC0072B26D69D0E7C0462804002020
:10D6080070B5041E02D00378F52B07D00421200042
:10D61800494201F02FF90420404270BD037E002BDF
:10D628001FD06369C068002B01D022691A61226982
:10D63800002A1DD053610225831CDB7FC26A5BB2BE
:10D64800002A17D11F21421C5156994202D0D37784
:10D6580000F013FC03256D42A06800281AD100F0E1
:10D6680089FC00232370A378DB071BD40020D4E7B0
:10D67800C362E0E7D17829420AD09168002907D02F
:10D688000131C97F0E1C49B2994200DA1E1C73B2DF
:10D698005269D5E7200000F0DBFB0022290000F0EA
:10D6A80081FDD9E7074A084B1068002803D02100FC
:10D6B800FFF7D7FBDAE704332100D86FFFF777FBD2
:0CD6C800D4E7C046BC0400202804002069
:10D6D400F8B50400002C00D1F8BD0822E37867698E
:10D6E400134216D00026A3682676B34211D0200038
:10D6F40000F0B0FB05003200310000F055FDEB6A8C
:10D70400E56026616361B34200D01C610123EC62D1
:06D7140023763C00DEE775
:10D71A0070B50225C3782B4220D01F22C068431956
:10D72A009A56C46AE3782B420DD0A3688B4200D183
:10D73A008B68002B07D00133DB7F1E1C5BB2934240
:10D74A0000DA161C72B26469002CEBD11F21431C4B
:0ED75A005956914202D0DA7700F08EFB70BD76
:10D7680080B5EFF30583002B03D1EFF31083002B73
:10D7780006D006210020494201F07CF8002080BD37
:0CD78800014F00DFFBE7C046F5D30010A6
:10D7940080B5EFF30583002B03D1EFF31083002B47
:10D7A40006D00621494201F067F80620404280BDB8
:0CD7B400014F00DFFBE7C0467DD40010F1
:10D7C00080B5EFF30583002B03D1EFF31083002B1B
:10D7D00006D00621494201F051F80620404280BDA2
:0CD7E000014F00DFFBE7C0462DD5001014
:10D7EC0080B5EFF30583002B03D1EFF31083002BEF
:10D7FC0006D00621494201F03BF80620404280BD8C
:0CD80C00014F00DFFBE7C04609D600100A
:10D818000300EFF3108172B682890020824202D0A1
:0ED82800013A9A810130002900D162B67047A2
:10D83800224B70B50D00411E0400994201D8A84240
:10D8480006D204210020494201F01CF8002070BDD6
:10D85800002A26D090681668002809D00321030002
:10D868000B40084202D1D2680F2A0ED80921E9E7F5
:10D87800D368002BFAD1124A124B1068002812D034
:10D88800FFF7DCFA002815D00123F6228370002365
:10D89800027083600C4A0B4B46608581C4819A668E
:10D8A800D5E71600E7E7043301221021D86FFFF708
:10D8B8004AFAE7E705214942C6E7C046FEFF0000ED
:0CD8C800C004002028040020A5D9001096
:10D8D40010B5002802D00378F62B06D00421494263
:10D8E40000F0D2FF0420404209E08368002B07D0F7
:10D8F40000F0B0FA0122002100F056FC002010BD17
:10D90400EFF3108272B68389C189994205D9013334
:10D914008381002AF2D162B6F0E7002A00D162B610
:0CD924001121494200F0B0FF0320DCE7B5
:10D9300070B5041E02D00378F62B07D00421200016
:10D94000494200F0A3FF0420404270BD8368002BD1
:10D950000DD003256D42200000F07EFA0022290040
:10D9600000F024FCA0680028F5D100F007FB00239C
:10D970002370A378DB0701D40020E6E7074A084BB1
:10D980001068002803D02100FFF76FFAF4E7043392
:10D990002100D86FFFF70FFAEEE7C046C004002061
:04D9A0002804002037
:10D9A400836810B50400002B0AD0FFF733FF00286A
:10D9B40006D0200000F04EFA0022110000F0F4FB23
:02D9C40010BD94
:10D9C80070B504000D00002802D00378F62B08D0AB
:10D9D80004212000494200F055FF04235B4218004F
:10D9E80070BDFFF715FF00239842F8D19D420CD077
:10D9F8002900632000F07AFC002804D0044B2000A2
:10DA0800596900F00FFA0223E8E70323E6E7C04666
:04DA180028040020BE
:10DA1C0080B5EFF30583002B03D1EFF31083002BBC
:10DA2C0006D006210020494200F02AFF002080BDCC
:0CDA3C00014F00DFFBE7C04639D80010A6
:10DA4800B0B50C00EFF30583002B03D1EFF310837F
:10DA5800002B13D0002804D00378F62B01D1002C1A
:10DA680006D00421494200F00DFF0420404204E0A2
:10DA7800FFF7CEFE002804D02000B0BD024F00DF23
:0CDA8800FBE70320F2E7C046C9D90010FC
:10DA940080B5EFF30583002B03D1EFF31083002B44
:10DAA4001CD0002802D00378F62B06D0042149426A
:10DAB40000F0EAFE042040420DE0EFF3108272B65B
:10DAC4008389C18999420CD901338381002A03D007
:10DAD40000F0A8F8002080BD62B6F9E7054F00DF2A
:10DAE400F9E7002A00D162B61121494200F0CCFEC8
:08DAF4000320E0E7D5D8001083
:10DAFC0080B5EFF30583002B03D1EFF31083002BDC
:10DB0C0006D00621494200F0BBFE0620404280BDF3
:0CDB1C00014F00DFFBE7C04631D90010CC
:10DB280070B500F059FD1E4CE3680133E36000F066
:10DB3800DFF9002000F01EFA236D002B00D0984773
:10DB4800226C002A2BD0A369E06BD969984203D0D4
:10DB5800E363002900D1DA61DA69002A1BD1237A4C
:10DB6800022B1CD1656A002D19D0E36B6A1C0133A6
:10DB7800D27FDB7F52B25BB29A4210D1280000F00C
:10DB880071F9E06B00F08CF9280000F0EBF9236CD8
:10DB9800E563EB6103E0013ADA61002ADFD070BD8A
:04DBA800280400202D
:10DBAC0070B51C4B1C4D1C005634288872B622884C
:10DBBC00002A04D162B6002000F0DAF970BD013AF7
:10DBCC0022801A005A321288D96D9600013292B214
:10DBDC007158904200D1002218005A30028062B66F
:10DBEC000029E8D00878F1380828DED8F2F72CFCA8
:10DBFC0005DD09DDDD0B0DDD0F001B6E0800984700
:10DC0C00CFE75B6EFAE79B6EF8E7DB6EF6E71B6F10
:0CDC1C00F4E7C046280400207C0400202F
:10DC2800010070B5EFF31080174B184A1C8872B6C4
:10DC3800150056352B889C421ED901332B801300C2
:10DC480058331B88D56D9E0001339BB2AD199C4299
:10DC580000D100232960110058310B80002800D121
:10DC680062B6537A002B04D18022094B52055A60C0
:10DC780070BD01239372FBE7002800D162B6022031
:10DC8800FFF70DF8F4E7C0467C04002028040020C4
:04DC980000ED00E0BB
:0CDC9C000378F12B00D07047C068F9E756
:10DCA80010B5C46903694169621C0ED1002B00D00C
:10DCB80059614269002A03D013610023436101E0DE
:10DCC800084A13630023C36110BD002B03D0DA692F
:10DCD80059611219DA614269002AEDD1014AD36209
:08DCE800F0E7C046280400200B
:10DCF00001231F2110B54370C3185956094B0A4A16
:10DD00005B6A002B04D05C1CE47F64B28C4206DCAE
:10DD1000C26083609060002B00D0D86010BD1A00F4
:0CDD20009B68EEE728040020440400206B
:0CDD2C00014B58697047C04628040020D5
:10DD3800002310B5827804000380930707D5016B90
:10DD48000E4BD2060FD50833D86FFFF78AF8A378A1
:10DD5800DB0707D50A4A094B1068002807D02100BD
:10DD6800FFF77FF810BD586FFFF721F8EFE704338E
:10DD78002100D86FFFF71BF8F4E7C04628040020FD
:04DD8800B0040020C3
:10DD8C0080B500F08FFD044F00DF012100204942D7
:0CDD9C0000F05EFDFEE7C04611E2001042
:10DDA80070B50300022510000124284014402A42BF
:10DDB80014D1EFF3108672B69A6A15000D40002C44
:10DDC80006D0A94206D1100088439862100001E0ED
:10DDD800281EF8D1002E00D162B670BD986A0B00DB
:10DDE8000340002C03D09942F7D00020F5E75A1ED3
:08DDF80093415B421840F0E783
:10DE0000C37810B5DB0702D4FFF796FF10BD0423DB
:10DE100043700023044AC360536B8360002B00D01F
:0CDE2000D8605063F2E7C04628040020E0
:10DE2C001F2210B54B1C9A568368002B04D05C1C27
:10DE3C00E47F64B2944206DAC8608B608160002B88
:0CDE4C0000D0D96010BD18009B68EEE704
:10DE58000300806882689A60002A00D0D36000239B
:04DE6800C3607047DC
:10DE6C00C268002A06D083689360002B00D0DA6069
:06DE7C000023C3607047A3
:10DE820070B505000400002C09D02378F12B07D0CF
:10DE92002800FFF7EAFF29002000FFF7C6FF70BD48
:04DEA200E468F0E759
:10DEA800012310B5010043700148FFF7BBFF10BD07
:04DEB80044040020FE
:10DEBC00F8B50D4D2E7A022E13D16C6A002C10D0B1
:10DECC001F22631C9A561F236F69791CCB569A42EA
:10DEDC0007D12000FFF7C4FF3800FFF7DFFF6670A3
:0CDEEC00AC610020F8BDC04628040020F6
:10DEF800F8B5194DEC6A002C25D0E369013BE361C4
:10DF0800002B20D1102620276378732B05D008D842
:10DF1800532B19D0BB43432B06D12000FFF7BAFE81
:10DF280002E0B343832BF8D02000FFF79BFF2000CB
:10DF3800FFF7B6FF2469002C04D0E369002BE3D077
:10DF480000236361EC62F8BD2000FFF7A3FE210007
:0CDF5800FFF7DFFBE8E7C04628040020CC
:06DF6400806B20307047C5
:10DF6C0002234370014B98617047C046280400207F
:10DF7C00F8B5154D04002E7A6F69002815D1022EC4
:10DF8C0012D16C6A002C0FD0621C7B1CD27FDB7F01
:10DF9C0052B25BB29A4207DD2000FFF761FF3800F6
:10DFAC00FFF7A0FE6670AC61F8BD022E07D1421CD3
:10DFBC007B1CD27FDB7F52B25BB29A42EFDC20003B
:0CDFCC00FFF76CFFF0E7C04628040020BF
:10DFD800F0B587B0059103900421002813D0002ADA
:10DFE80000D192E01368946802935368156904930A
:10DFF800936956690193002C0DD0A30702D1D36809
:10E00800432B0BD809210020494200F023FC0024AF
:10E01800200007B0F0BDD368002BF3D1002D06D047
:10E028006B0702D1002E00D09EE00B21EBE7019B8D
:10E03800002B67D0019B0C21013B372BE3D8002E26
:10E0480000D097E00027BC4209D14F4A4F4B1068D7
:10E05800002861D0FEF7F2FE041E75D00127002DBE
:10E0680011D14A4B002E5ED1494A566D1A0008322A
:10E07800D06F002857D0FEF7E1FE051E5AD01023B6
:10E088001F4302231F43F223FF332380049B6A4666
:10E09800E370029B12796360002352B2611CA36093
:10E0A800E36023616361A361E361A770CA77A11C80
:10E0B800CA776362A362E3623300FD22403BEB1838
:10E0C800A363039B6284E363324B256366632B601F
:10E0D8002F4B1B685B073FD4A56B34220021280017
:10E0E80009F0AEFA2C4B2D4A6B63039B2000AB63FF
:10E0F80080235B04EB63059B2B62244B1A66FFF7B6
:10E1080039FF85E71823019399E7182315001600AE
:10E1180002920193049298E7043301224421D86FB4
:10E12800FEF711FE98E72A003100586FFEF70BFE44
:10E13800051EA6D1002F07D0134A144B10680028DB
:10E1480004D02100FEF78DFE05215CE70433210091
:10E15800D86FFEF72CFEF7E7B208113ACC219200EF
:10E16800281D09F06DFAB7E7019B002B00D061E785
:10E1780018230193730700D057E73300084A483B38
:10E18800934200D85EE750E7B0040020280400203E
:10E1980014C80110A52E5AE28DDD0010CDE1001043
:04E1A800B7FFFF7F3F
:10E1AC0070B50400836B15001962FFF777FD200032
:10E1BC00002D02D0FFF7DCFE70BDFFF76FFEFBE712
:10E1CC0010B543780400332B0AD1031D416ADA7F62
:10E1DC00FFF7E4FD011E03D000222000FFF7E0FF53
:02E1EC0010BD64
:10E1EE0010B504008069002803D000221100FFF74B
:10E1FE00D6FF6378232B02D10022A3689A6110BD4B
:10E2100070B50E4C267A022E16D1636A002B13D0ED
:10E220006569E86AFFF756FA2800FFF7E0FF08483B
:10E23000FFF712FE4670A061EFF30983AB63002382
:10E2400028006361FFF7DCFD70BDC0462804002094
:04E250004404002062
:10E2540070B5041E02D00378F12B07D004212000EE
:10E26400494200F0F9FA0420404270BD0F2243787D
:10E274001340022B0AD0032B2BD0012B26D00321D1
:10E284002000494200F0E8FA0320EDE7164B1A7A21
:10E29400022AF4D15B6A002BF1D0E06AFFF718FA86
:10E2A4002000FFF7A2FF6578022D18D10F48FFF771
:10E2B400D1FD0D4B45709861EFF30982A2630022F2
:10E2C4005A612000FFF79AFD0020CEE7FFF7CCFD4E
:10E2D400E3E7FFF7C9FD2000FFF7E4FCDDE70020DA
:10E2E400FFF74AFEEDE7C04628040020440400205E
:10E2F40070B51F4C0300227A0020022A18D1626AEA
:10E30400824215D0626953704B1C17D1236B002BCA
:10E314000FD101214942D1615061136100280BD012
:10E3240002611448FFF796FD02234370A0610120A7
:10E3340070BD18001B69EAE72263F2E7E36A002B69
:10E3440002D0DD69A9420CD2D16150611361002869
:10E354000BD00261002BE4D0D8695A61411AD9610B
:10E36400DFE71800491B1B69E9E7E262F2E7C046F0
:08E374002804002044040020ED
:10E37C0070B50D4D00210D48AA6DFFF727FE0C4C12
:10E38C006B6EA0620120002B0DD09847030000207B
:10E39C00834208D1EA6DE16C286EFFF717FEA0648A
:10E3AC00431E9841C0B270BD14C80110B9E70010EB
:04E3BC002804002011
:10E3C00080B5EFF30583002B03D1EFF31083002B0F
:10E3D00006D006210020494200F040FA002080BD0E
:0CE3E000014F00DFFBE7C046D9DF001052
:10E3EC0080B5EFF30583002B03D1EFF31083002BE3
:10E3FC0002D0034B586980BD024F00DFFBE7C046DB
:08E40C00280400202DDD0010A2
:10E4140080B5EFF30583002B03D1EFF31083002BBA
:10E4240007D006210020494200F016FA0620404297
:0CE4340080BD014F00DFFBE7BDDE0010E3
:10E44000B0B5040000F040FAEFF30583002B03D1D0
:10E45000EFF31083002B07D006212000494200F083
:10E46000FDF906204042B0BD2000014F00DFFAE771
:04E4700055E2001061
:10E47400002230B50C4D6B6C002B02D01C698C4211
:10E484000CD901618260C360002B03D01C699860C1
:10E49400611A1961002A05D0D06030BD1A00091B29
:0CE4A400DB68E9E76864F8E72804002062
:10E4B000F8B51B4D6C6C002C2DD023696E69013BA7
:10E4C00023612369002B25D1E368002B01D0A268CA
:10E4D0009A6021006B640023E86C1A001831FEF783
:10E4E0000BFF00280CD0AB69210003206F696B6122
:10E4F000FEF7D9FB6B69002B02D1B74200D11E0099
:10E50000E378012B08D120006169FFF7B3FF6C6C41
:10E51000002CD6D16E61F8BD01236370F7E7C046C9
:04E5200028040020AB
:10E5240010B5FEF7D5FE002803D1034B034A1A6544
:10E5340010BD01204042FBE728040020B1E4001094
:10E5440037B5012504006D422B00002269462000E6
:10E55400FEF712FF0028F7D1009B01989847F3E7D4
:10E56400010010B5002817D00D4B1868F1F784FF8F
:10E57400802301385B0498420ED2FF23094A1B060C
:10E58400116A0B4313620622074B1A60586000207D
:10E594009860064B187010BD01204042FBE7C0464E
:10E5A400D405002000ED00E010E000E055AB0020B1
:10E5B400074B1A78002A05D000221A708022054BD6
:10E5C400D2045A600123044A11680B431360704754
:0CE5D40055AB002000ED00E010E000E07E
:0CE5E000014B1B687047C04610E000E0D3
:06E5EC00012040427047CF
:10E5F400094A0A4B10B51A60094B0A499B1A0B6069
:10E60400094A0A4B0A491A600A4B9B1A0B6000F02C
:10E6140055F800F06DF8C04600FC0320D4A7002094
:10E6240000000420D0A7002084AB0020C8A700204D
:08E63400C4A7002000FC032034
:10E63C0070B50B251C240C480C4B456003600C4B2F
:10E64C00C4608360FFF78AF80A4B18600A480B4BCA
:10E65C00456003600A4BC4608360FFF77FF8094B89
:10E66C00186008F06DFB70BD40A70020A8360210A2
:10E67C0054A7002050A7002038A50020B536021062
:08E68C004CA5002048A5002068
:08E6940010B5FDF743FF10BDB6
:10E69C00012110B5024B49421868FFF775F810BDFF
:04E6AC0050A7002053
:10E6B00010B5024B1868FFF783F810BD50A7002073
:0CE6C00010B504F045FD00F011F810BD8D
:02E6CC00704795
:02E6CE00704793
:10E6D00010B500F043F8FFF7F9FFFFF7AFFFFFF7C2
:0CE6E000F6FF03F055FBFFF7D5FF10BD5F
:08E6EC0010B5FEF7E5FA10BDC0
:10E6F40013B5114B114C0021236180231B0263616C
:10E704004423E3600E4B2200A3601823A3610D4B46
:10E714000D482360FFF752FE031E05D122000B496A
:10E7240000900B4803F03AFBFEF7DEFA0022094999
:10E7340013000092F5E7C04678100020D4A300200F
:10E7440024A90020BF360210D1E60010C4360210FE
:08E754001D010180E0360210F6
:10E75C0030B585B068460200054B32CB32C21B681F
:10E76C001360FEF7FBFF034B186005B030BDC046CD
:08E77C0084C8011074A90020FB
:10E7840073B506000C00150003F002FB00280CD141
:10E794000649A21D063402D3054B9200D15800232A
:10E7A40032002800009303F0F9FA73BDF536021025
:04E7B4001038021007
:06E7B80010B500F099F815
:10E7C00007B5020001380023042823D8F1F74CFED6
:10E7D000030A10161C000093012200230F49104861
:10E7E00003F0DEFA0093022200230E490E48F7E7F9
:10E7F0000093032200230D490D48F1E70093042202
:10E8000000230C490C48EBE70093052200230B4939
:10E810000B48E5E70B490C480093E1E7FD36021091
:10E82000250102801E3702102601028043370210A4
:10E83000270102807837021028010280B3370210C6
:0CE840002A010280F33702100001028060
:10E84C0010B50100014AFFF797FF10BD310101809F
:10E85C0010B5024AFFF790FF10BDC046320101808F
:10E86C0010B5024AFFF788FF10BDC0463701018082
:10E87C0010B5024AFFF780FF10BDC046330101807E
:10E88C000B0010B5113302D0014AFFF775FF10BD14
:04E89C0034010180C2
:10E8A00010B5024AFFF76EFF10BDC0463801018067
:10E8B00010B5FFF79BFD034B1B68002B00D098475A
:08E8C00010BDC046D0A90020E4
:10E8C800034B10B51B68002B00D0984710BDC046FD
:04E8D800D0A90020A3
:10E8DC0010B503F0F7F803F0EFFA03F0EEFA03F0DB
:04E8EC0007F910BD5B
:10E8F00010B5024B1B689847FBE7C046CC040020CC
:08E9000010B5FDF7B7FA10BDD8
:10E9080070B504000D001022002108F099FE2900BE
:0AE918002000FDF7B3F9200070BDE8
:10E92400044B10B51868002803D001214942FEF7B2
:10E934002FFF10BD74A90020044B10B518680028DF
:10E9440003D001214942FEF723FF10BD74A9002022
:10E9540070B50500060010CD002C0FD1FFF7E0FFC5
:10E964003468002C04D1280003F02AFF2C00356001
:10E97400074B1868002801D0FEF720FFAC4204D0F2
:10E984008B220449044802F0F3FF200070BDC04606
:0CE9940074A900204C3802105B380210FF
:0EE9A00010B50368012200211B69984710BDC5
:0EE9AE00002210B5036811001B69984710BDC8
:10E9BC0010B5040003F086F80121200004F09EFB42
:06E9CC0003F096F810BDF7
:10E9D20010B5040003F07BF80021200004F093FB43
:06E9E20003F08BF810BDEC
:10E9E80070B50D00040003F06FF82900200004F052
:08E9F8006DFB03F07FF870BD18
:10EA000037B504000C22835E0A21425E0820215E95
:10EA100060680E25645F0430009405F095FD37BDF5
:10EA200070B50024050003F053F8074B1B68A342A0
:10EA300006DD064B1C78641B6242544164421C4054
:10EA400003F05CF8200070BD149C0020E09B0020C7
:10EA5000084A10B51368002B04DDAF2206490748A9
:10EA600002F088FF34205843591C054B1160C01830
:10EA700010BDC046149C0020973802109F38021029
:04EA8000E09B0020F7
:10EA8400082370B543610023040083610A4B250009
:10EA9400C361FF232835038403F018F82878FFF7AF
:10EAA400BDFF6060002804D1FFF7D0FF60602B78C1
:0CEAB400037003F021F870BD40420F0019
:10EAC00070B5040004A80025405F0D4D218125602C
:10EAD000E0810025200001216281A3812582A574A7
:10EAE0004942103002F0BCF9064B6562E362230034
:10EAF000283320001D70FFF7C5FF200070BDC04601
:08EB0000D038021001EA0010F8
:10EB0800436810B51B6B040083420FD0C36A984753
:10EB180060680023A2696169043005F073FD6068CC
:0EEB2800E169043005F0AAFD63681C6310BDAE
:10EB360070B504000D00160003681B6998476068ED
:10EB46006561036BA661A3420AD100233200290046
:10EB5600043005F058FD236820005B69984770BDB6
:08EB66002000FFF7CEFFF6E7E7
:10EB6E0070B504000D0003681B6998476068E56185
:10EB7E00036BA34208D12900043005F07CFD236805
:10EB8E0020005B69984770BD2000FFF7B6FFF6E7DF
:10EB9E0070B510300D00040004F0CDFA002803D03B
:0AEBAE002900200004F071FA70BD88
:10EBB80070B504001F2503681B699847A31C5D579F
:10EBC8006A1CDA77002D06D12000FFF799FF29008B
:08EBD8002000FFF7E0FF70BD13
:10EBE00010B5821CD37F0400013B5BB2D377002BAE
:10EBF00002D10121FFF7D3FF236820005B6998470A
:02EC000010BD45
:10EC020070B504000D00FFF7D6FF606829000430DC
:10EC120005F03DFD05002000FFF7E1FF280070BD73
:10EC2200F7B504001F0016000D00FFF7C4FF631CB8
:10EC3200DB7F60680193089B320029000093043057
:10EC42003B0005F03CFD05002000FFF7C8FF28004F
:02EC5200FEBD05
:10EC540010B540680830FFF77BFE03F0B9FD10BD26
:10EC640010B540680830FFF773FE03F0CDFD10BD0A
:10EC740010B50400074B0360FFF7EAFF63681A6BE3
:10EC8400A24201D100221A632000FFF7E9FF20000D
:08EC940010BDC046D03802108B
:10EC9C0010B50400FFF7E8FF2000302103F0CAFB99
:04ECAC00200010BD77
:02ECB0007047AB
:10ECB40070B506000400831D3E229A5E0C36031DC7
:10ECC4003E21595E300005F0F5FAE56C236D002D08
:10ECD40001D1DA0711D558102018DB0701D50368D4
:10ECE4005D592300583300229B5E220056320021D6
:10ECF400525E210054310978A8473000E16B05F0D9
:10ED04003EFB30002200024905F078FB70BDC0468E
:04ED14002BF00010D0
:10ED1800F7B50093836C04000E001500002B05D096
:10ED280036222B492B48FF3202F020FE2A4A03657F
:10ED38000368C2641B6898472300270054331E7079
:10ED480002331D800193009B58373B80042E0DD859
:10ED58003000F1F785FB15031015190001232A006F
:10ED680001215B4220000C3005F0B5FB2368200030
:10ED78005B689847F7BD01222B0002215242F1E758
:10ED88002A003100009BEDE72300012270331A703E
:10ED980001350CD0042003F01FFB019B0500002166
:10EDA800595E00230380837002F04BF8E56500226A
:10EDB800BB5E0133DAD0042003F00EFB002205000D
:10EDC8000023F95E0280827002F040F82566CDE7E4
:0CEDD800013902101039021019ED001072
:10EDE40010B50400FBF75EFC2000FCF743FF10BDE8
:10EDF40010B50400FBF756FC2000FCF73BFF10BDE8
:10EE040070B504000D00884205D0FBF74BFC2900C7
:10EE14002000FCF735FF70BD70B504000D0088427A
:10EE240005D0FBF73FFC29002000FCF729FF70BD4B
:10EE340070B504000D00884205D0FBF733FC2900AF
:08EE44002000FCF71DFF70BD6A
:10EE4C0070B5040003680D001B689847200029006A
:10EE5C000C3005F090FA2368E56320005B68984756
:02EE6C0070BD77
:10EE6E00F8B504001F0003680D001B6816009847D4
:10EE7E0020003B00320029000C3005F08CFA23688C
:08EE8E0020005B689847F8BD05
:10EE960070B5040003681B68984720000C3005F025
:10EEA60010FB230070331B780500002B06D0206E64
:10EEB600002803D06942694104F0EBF8236820007A
:08EEC6005B689847280070BD4D
:10EECE0070B5040003681B68984720000C3005F0ED
:10EEDE00FAFA230070331B780500002B05D0E06D85
:10EEEE0004F0DFF8434258410540236820005B6878
:06EEFE009847280070BDDA
:0AEF040010B50C3005F0CEFA10BD78
:0EEF0E0010B50C000C3005F0D0FA200010BD3C
:10EF1C00F7B5002504001F00194B0E000360194BB8
:10EF2C0029004360856001920C30102208F086FBAA
:10EF3C0020001C30FCF73EFD20002C30FCF73AFD85
:10EF4C000222A31CFF32E763DA87019A231DDE87B6
:10EF5C00A31DDA874E33A564E564256522001D7078
:10EF6C00012356325B421380538023007033656655
:10EF7C00A566E56620001D70FFF796FE2000FEBD1D
:08EF8C0030390210B5EC001051
:10EF9400F7B50500036816001B680F0098472B009F
:10EFA40040331B783401002B01D0002E10D02B00ED
:10EFB40041331B78002B01D0012E09D01C343900B9
:10EFC4002819FFF71DFF2B6828005B689847F7BDD9
:10EFD40002F07CFD3800FCF742FF2B001C340C339C
:10EFE4002C190193002812D02000FCF738FF0028C8
:10EFF40001D102F065FF39002000FFF701FF012273
:10F004003100019805F00CFA02F076FDDBE72000F0
:10F01400FCF725FF002801D002F053FF2000FFF782
:06F02400DFFE0022ECE714
:10F02A0009011C3110B544182000FCF715FF00280F
:0AF03A0002D02000FFF75FFC10BDBC
:10F04400F8B504002700036840371B680D00984793
:10F054003B78AB4241D026001C36002D0FD102F084
:10F0640035FD20002A000C30290005F0D9F93000C4
:10F07400FCF7F5FE002822D002F023FF1FE0230056
:10F0840041331B78002B08D1A26863685010201804
:10F09400D20701D50268D358984702F017FD300013
:10F0A400FCF7DDFE00280AD03000FCF7E1FE02F098
:10F0B40007FF2000012200210C3005F0B1F902F015
:10F0C4001BFD3D70002D08D1230041331B78002B1C
:10F0D40003D120000C3005F04DF9236820005B6853
:04F0E4009847F8BD94
:10F0E800F8B504002700036841371B680D009847EE
:10F0F8003B78AB4241D026002C36002D0FD102F0D0
:10F10800E3FC20002A000C30012105F087F93000CB
:10F11800FCF7A3FE002822D002F0D1FE1FE0230056
:10F1280040331B78002B08D1A26863685010201860
:10F13800D20701D50268D358984702F0C5FC3000C1
:10F14800FCF78BFE00280AD03000FCF78FFE02F097
:10F15800B5FE0122200011000C3005F05FF902F025
:10F16800C9FC3D70002D08D1230040331B78002BCB
:10F1780003D120000C3005F0FBF8236820005B6801
:04F188009847F8BDEF
:10F18C001FB50400194B002103606846FCF719FCFD
:10F19C00002269462000FFF7F7FE6846FBF785FA68
:10F1AC0000216846FCF70DFC012269462000FFF7A0
:10F1BC00EBFE6846FBF779FA230040331B78002BF3
:10F1CC0004D1230041331B78002B03D020000C30DA
:10F1DC0005F0CCF820002C30FBF767FA20001C302F
:10F1EC00FBF763FA200004B010BDC04630390210A2
:10F1FC0010B50400FFF7C4FF2000742103F01AF9C6
:04F20C00200010BD11
:10F2100010B5437D0400002B04D0037D002B01D0EA
:08F2200002F051FE200010BDB8
:10F2280013B5040001A802F06DF8637D002B0BD123
:10F23800237D002B01D002F041FE206902F020F866
:10F24800012320606160637501A802F061F813BDB5
:10F2580037B5040001A80D0002F054F8002300227D
:10F26800226063606B7D002B08D0286902F008F8E3
:10F278002A686B68801A99412060616001A802F0D1
:06F2880047F820003EBD26
:10F28E0030B50D0085B0040003A802F038F829004F
:10F29E006846FFF7DAFF009A019BA868E968121822
:10F2AE004B4103A82260636002F02FF8200005B0E6
:02F2BE0030BD61
:10F2C00013B5040001A802F021F8206901F0DCFF69
:10F2D0000022002320606160A260E36001A802F0C8
:04F2E0001BF813BD47
:10F2E40010B50B00040000210020236100232060DE
:10F2F4006160A060E160227520006375FFF7DEFFA6
:04F30400200010BD18
:10F3080010B5040001F0E6FF012201002000FFF71C
:06F31800E5FF200010BD1E
:04F31E000020704714
:0CF322001D20404270471D2040427047F3
:0CF32E00162040427047162040427047F5
:08F33A0001207047012070471B
:08F34200002070470020704715
:10F34A00F8B501230C0006000D001C40194204D038
:10F35A00FFF79CFD431E984104B210273D4205D099
:10F36A003000FFF7AFFD002800D03C432000F8BD75
:10F37C0008B4024B9C46743808BC60474BF3001031
:0AF38C0010B5FFF759FE002010BD78
:10F3980008B4024B9C46743808BC60478DF30010D3
:0AF3A80010B5FFF79DFE002010BD18
:10F3B40008B4024B9C46743808BC6047A9F300109B
:10F3C40010B50400024B0360FFF7DEFE200010BD01
:10F3D4004839021008B4024B9C46743808BC604794
:04F3E400C5F300105D
:10F3E80010B50400FFF7EAFF2000782103F024F8A5
:10F3F800200010BD08B4024B9C46743808BC604716
:04F40800E9F3001014
:10F40C00F7B505000C00161E1AD002F057FB0123AD
:10F41C004340DFB2002F03D02B6828001B689847AD
:10F42C00A319019321782800FFF76BFD019B013490
:10F43C00A342F7D1002F03D02B6828005B689847B4
:04F44C003000FEBDD1
:10F4500008B4024B9C46743808BC60470DF4001099
:10F4600070B504000D00101E0CD0236820001B682E
:10F4700098472000FFF746FD2870236820005B684E
:06F480009847012070BD59
:10F4880008B4024B9C46743808BC604761F400100D
:10F4980010B50400FFF73EFD024B20002360024B2D
:0CF4A800636710BD48390210843902105F
:10F4B400F8B504000D0016001F0003681B68984788
:10F4C4003B00320029002000FFF724FC23682000C1
:06F4D4005B689847F8BDDB
:10F4DA0070B504000D0002F0F6FAA669002E02D1FA
:10F4EA0002F007FB70BD20000830FFF77EFC012206
:10F4FA00631CDA770023A21CE361D577A36102F0CB
:0CF50A00F8FA2100300000F089F9EBE76E
:10F5160010B5002802D003F05AF910BD02F0D5FA52
:02F52600FBE701
:10F5280010B5002802D003F06DF910BD02F0E2FA20
:02F53800FBE7EF
:10F53C00F0B5040089B00E00019202F0C3FAA5697F
:10F54C0002F0D6FA002D27D003AD0021280003F0DD
:10F55C0097F902F0B7FAE369A769002B04D03922B6
:10F56C000E490F4802F000FAE56102F0C1FA002FD3
:10F57C000FD02800019903F08DF9002809D1300033
:10F58C00FFF7C3FF20000121FFF7A1FF3000FFF7B9
:10F59C00C5FF280003F0A1F909B0F0BDE93902104C
:04F5AC00F53902101B
:10F5B00070B500250400054B456003600830FCF77A
:10F5C000FFF92000A561E561258470BD1C3A021099
:10F5D000084B10B5036083690400002B04D0262279
:10F5E0000549064802F0C6F90830FBF764F8200028
:10F5F00010BDC0461C3A0210E9390210033A02104D
:10F6000030B50400250085B0083502F061FA290004
:10F610006846FFF779F92800FFF7ECFB0023E06963
:10F62000A361984201D003F059F902F067FA6846E5
:10F63000FCF717FC002802D06846FFF761F968461E
:08F64000FBF739F805B030BDFD
:0EF64800002343608360013301600373704749
:02F656007047FB
:10F658000300007B002805D00CCB002012689A42DA
:06F668004041C0B27047F2
:10F66E00F0B50125036885B001932B008B402F0068
:10F67E000293040000235740039701995800043168
:10F68E00095C0298084205D030200140002A07D0BC
:10F69E00102907D10233202BEFD10120404210E078
:10F6AE000029F7D010002F0018438740A6683E426D
:10F6BE00F0D1202905D12F00039919438F403E42E6
:06F6CE00E8D105B0F0BD1B
:10F6D40070B5040008001100020020001D00FFF7AF
:10F6E400C4FF021E02DA0020207370BD46082068A1
:10F6F400B300C018C388616859184379D0015D43C9
:10F704004919616001219140A36830430B43A36010
:04F71400C0B2EAE7AE
:0EF7180010B513000A000121FFF7D8FF10BD45
:0EF7260010B513000A000021FFF7D1FF10BD3F
:10F7340070B50D0004000A000021FFF7EBFF2A005A
:0AF7440000212000FFF7EDFF70BD6B
:08F74E000023036043607047D3
:02F756007047FA
:04F75800006870478E
:10F75C0000230B604368002B02D1016041607047AD
:04F76C001960FBE73E
:10F7700003000068002806D00268002A00D15A6001
:08F780001A60002303607047CA
:10F7880010B50468002223008B420ED1002A01D054
:10F798000B6813608C4201D10B68036043688B428D
:10F7A80000D1426000230B6010BD002BFCD01A0072
:04F7B8001B68E9E7FA
:0CF7BC0010B50400FFF7C5FF200010BDD1
:0EF7C80010B5FFF7C5FF43425841C0B210BD57
:10F7D60070B505002800FFF7BCFF041E0ED0043CE0
:10F7E600236820009B689847002807D02800FFF769
:0EF7F600BCFF23682000DB689847EBE770BD7E
:10F8040070B504000D00FFF7A5FFAC610600291DCB
:10F814002000FFF7A1FF002E02D12000FFF7D9FF3F
:02F8240070BDB5
:10F8260070B505000C00FFF794FF0600002C00D011
:10F83600043421002800FFF7A4FFA64202D12800C5
:06F84600FFF7C6FF70BDD4
:10F84C0010B504002000FFF781FF002804D0043815
:0AF85C000368DB689847F5E710BD6C
:10F8660010B50400FFF7EFFF2000FFF771FF20003F
:02F8760010BDC3
:02F878007047D7
:02F87A007047D5
:0AF87C0010B503689B6D984710BD9E
:10F88800C82330B59B00C5580C4B87B001930023A3
:10F8980001A98B808B710A4B44680289CB810A309D
:10F8A8000423039404008A81FF331222CD710B8252
:10F8B80007F034FE200007B030BDC0461201000238
:04F8C8000102000039
:08F8CC0000487047503D021096
:08F8D400004870473E3D0210A0
:08F8DC0000487047283D0210AE
:08F8E40000487047223D0210AC
:08F8EC00004870471A3D0210AC
:08F8F40000487047043D0210BA
:10F8FC00036810B55B6F04009847BB239B00E0586E
:10F90C0003681B6F9847236820009B6F984710BDB6
:10F91C00CD239B00C35870B50400012B16D1C9250B
:10F92C00CA26AD00B6000122A05963590240002B33
:10F93C0001D1002A0AD00021401061512018A15198
:10F94C008A4201D00268D3589847ECE7CD22920046
:10F95C00A358002B04D105490548064A02F004F8C7
:10F96C00013BA35002F0C4F870BDC046493A0210E6
:08F97C00573A0210C606000014
:10F98400CD239B00C35810B5002B04D10249034872
:10F99400034A01F0EDFF10BD493A0210573A021034
:04F9A400CD0600008C
:10F9A80010B5040002F090F8CD229200A35801335C
:10F9B800A350002B05D1D72202490348D20001F0F9
:0CF9C800D5FF10BD493A0210573A02105A
:10F9D400036870B5DB6F04009847BE239B00E55AAB
:10F9E4002B0A022B27D0032B5AD0012B05D12368D5
:10F9F40020001B6B9847002801D1002070BD2368AC
:10FA040020001B6B98470678122EF6D1236820003D
:10FA14001B6B98474578012DEFD1C1239B00E6501D
:10FA2400236820001B6B9847C0239B00E0500833D9
:10FA3400E5540120E2E72368EDB2290020005B6B66
:10FA440098470028D9D0236829005B6B2000984789
:10FA54000378092BD1D1236829005B6B20009847D8
:10FA64004378022BC9D1236829005B6B2000984797
:10FA74002368867829005B6B20009847C122C378ED
:10FA840092001B023343A3502368290020005B6BC0
:10FA94009847C02301229B00E0500833E254C8E792
:10FAA400E8B20528A9D8C1252368AD00F0F7DAFC2F
:10FAB400030D151D252D9B6B20009847037863517A
:10FAC40023689B6B20009847E3E7DB6B2000984793
:10FAD400037863512368DB6BF4E71B6C20009847C1
:10FAE4000378635123681B6CECE75B6C2000984738
:10FAF4000378635123685B6CE4E79B6C20009847B0
:10FB04000378635123689B6CDCE7DB6C2000984727
:0AFB1400037863512368DB6CD4E72B
:10FB1E001F200B78DB0913700B785B069B0F53705D
:10FB2E000B78034093704B78D370CB7888781B0298
:10FB3E00034393804B7908791B020343D380CB791F
:0AFB4E0088791B02034313817047FE
:10FB5800036870B55B6F04000D009847C3239B00D2
:10FB6800E35C022B05D03E220A490B48FF3201F024
:10FB7800FDFEC423C9229B00E554084B9200A35004
:10FB8800CA2300229B00E250236820009B6F9847FD
:10FB980070BDC046493A0210633A021019010110BB
:10FBA800036870B5DB6F04009847C2239B00E35CD1
:10FBB800002B01D0002070BDBB25AD006059036843
:10FBC8005B6C9847C1239B00E2588242F2D3C0265F
:10FBD800B600A159121A0918A151E250002A14D1ED
:10FBE80002210833E1540F4BE15C002908D0E254AC
:10FBF800163BE118236820009B6E98470120DAE73E
:10FC080001212000FFF7A4FFF8E7C8239B00E35871
:10FC18006059934200D913000268146C1A00A04777
:08FC2800ECE7C0460A030000EE
:10FC3000036813B5DB6F04009847C7239B00E35CA0
:10FC40000F49012B05D9C3239B00E35C002B06D091
:10FC50000C4900220C481300009202F0A1F80B4B53
:10FC6000E35C032B0AD02000FFF79EFF002805D19C
:10FC7000BB239B00E0580368DB6C984713BDC0466C
:10FC80008E3A0210B63A02100E0115800B030000E6
:10FC9000036870B5DB6F04009847C2239B00E35CE8
:10FCA0000020012B35D1C1239B00E358834204D1AE
:10FCB0001B4AA15C81422BD0A354C8229200A558B4
:10FCC0009D4200D91D00BB23C0269B00E058B60012
:10FCD00003682A009B6CA1599847C122A35992003E
:10FCE0005B19A351A3585B1BA35011D10C4BE25CD1
:10FCF000002A0DD102210333E1540A4BE15C0029B3
:10FD000008D0E254163BE118236820009B6E984708
:10FD1000012070BD01212000FFF71EFFF8E7C0465B
:08FD2000090300000A030000C2
:10FD2800036813B5DB6F04009847C7239B00E35CA7
:10FD3800012B06D800220B4913000B48009202F051
:10FD48002BF80A4BE35C032B0AD02000FFF79CFF3B
:10FD5800002805D1BB239B00E0580368DB6C98475B
:10FD680013BDC0468E3A02100E0115800B03000029
:10FD7800036870B55B6F04000D009847C3239B00B0
:10FD8800E35C032B05D0C3220A490B48520001F05B
:10FD9800EDFDC423C9229B00E554084B9200A350F3
:10FDA800CA2300229B00E250236820009B6F9847DB
:10FDB80070BDC046493A0210003B0210B90B011051
:10FDC800036810B50400DB6F98470120044BE21864
:10FDD8001D3BE2500433E0500433E05410BDC046EC
:04FDE8001D030000F7
:10FDEC00036810B5DB6F04009847C7239B00E35CE6
:10FDFC000020042B0CD1074B0130E25A064BE25287
:10FE0C003633E218303BE2500433E0500433E05414
:0CFE1C0010BDC0462E030000FA020000DA
:10FE2800036810B5DB6F04009847C32304229B00C6
:10FE3800E254143BE25C044B2000E15A23681B6F38
:0CFE48009847012010BDC046FA020000DF
:10FE5400036870B55B6F04000D009847C3239B00D3
:10FE6400E35C042B05D0EB220A490B48520001F055
:10FE74007FFDC423C9229B00E554084B9200A35084
:10FE8400CA2300229B00E250236820009B6F9847FE
:10FE940070BDC046493A02102C3B0210B901011052
:10FEA400036810B5DB6F04009847C7239B00E35C2D
:10FEB400042B04D000201B4BE35A83422FD11A4B4E
:10FEC400E35C012B2CD0022B04D00020002B26D184
:10FED400012319E0134B0020E15A8F230A009A43AF
:10FEE40082421CD10F220B00134011420CD01E235E
:10FEF4004A001A40C9110A43023A063B5343E31825
:10FF040030331B789B07DB0F084A01201380C02382
:10FF14009B00E25002220433E2500433E05410BD4B
:10FF24000023F1E7FA020000F6020000C8AA00204C
:10FF340030B5036891B0DB6F04009847BB23C82237
:10FF44009B00E058920003686946A258DB6B98470F
:10FF5400BD239B00E5182A0069462000FFF7DDFD5C
:10FF6400C02200239200A3500432A3500432A350B1
:10FF7400C32301229B00E2542368290020005B6E06
:06FF8400984711B030BDEA
:10FF8C00036813B5DB6F04009847C7239B00E35C41
:10FF9C00012B06D800220A4913000A48009201F0EE
:10FFAC00F9FECB2201239200A354203AA25C002A32
:10FFBC0003D12000FFF7B8FF13BD034AA354FBE79E
:0CFFCC008E3A02100E0115802D0300007B
:10FFD800F8B51D00036804005B6F0F001600984712
:10FFE800C3239B00E35C012B04D00C490C480D4A49
:08FFF80001F0BCFCC423C92286
:020000041001E9
:100000009B00E7540433E6500433E550084B92005C
:10001000A350CA2300229B00E250236820009B6F5C
:100020009847F8BD493A0210543B0210BA0200004A
:04003000490A011068
:10003400036870B5DB6F04009847BF239B00E35A45
:10004400002B43D0C2229200A15C143AA25C012A84
:1000540022D1012906D0BB239B00E0580368DB6C46
:10006400984770BDC1229200A058984201D9180047
:10007400A350834209D9C8239B00E158F0F782FAC0
:10008400002902D10122194BE2540222184B20000C
:10009400E254FFF7FBFDE4E7BB229200002901D004
:1000A400A058DBE7C121890061589942F8D10120A9
:1000B4000F4BE0541533A058E2588A4200D90A0085
:1000C400C021036889001B6C61580DE0BB23C12269
:1000D4009B009200E058A15803680029BFD1032572
:1000E400034A9B6CA5540A009847BAE70903000029
:0400F4000B030000FA
:1000F800036810B5DB6F040098470022024BE254F6
:10010800024B0332E25410BD2D0300000B03000024
:10011800036810B5DB6F04009847C423C32200218D
:1001280092009B00E35CA154134AA15C002903D010
:100138002000FFF7DDFF10BD002B06D1BB239B007D
:10014800E0580368DB6C9847F5E70C4BE25C012A42
:1001580008D10232E2541F3BE05803689B6C0A0046
:100168009847E8E7022AE6D10132E254BB239B0014
:10017800E05803681B6CF2E72D0300000B03000036
:10018800036810B5DB6F04009847CB2300229B005F
:10019800E254203BE35C934203D12000FFF7A8FF21
:1001A80010BD0122014BE254FAE7C0462D030000BE
:1001B800036810B5DB6F04009847C423C3220021ED
:1001C80092009B00E35CA1540E4AA25C8A4203D0D1
:1001D8002000FFF78DFF10BD002B0BD00A4B20002D
:1001E800E25A0A4BE252363BE25A3833E254FFF7FE
:1001F8001DFFF0E7BB239B00E0580368DB6C9847C2
:10020800E9E7C0462D030000FA0200002E030000B3
:1002180070B5BC2504000368AD005B6F9847635D4B
:10022800002B10D1BB26B600A059210003689B689B
:100238009847A059402103689B6B9847C8239B00A7
:10024800E05001236355236820009B6F984770BDD9
:10025800036870B55B6F05009847C7239B00EC5C8B
:100268002B68E4B228009B6F043C984763425C41CA
:04027800E0B270BDC3
:10027C0070B5040003680B4D5B6F98472000FFF7C7
:10028C00C5FF635D002B07D1BB239B00E0580368BF
:10029C005B69984701236355236820009B6F98473F
:0802AC0070BDC046F102000024
:1002B400F0B50D0089B00693036802925B6F0400E9
:1002C40098478F232A009A4301D12B0706D1002295
:1002D400284913002848009201F060FD274BE65C92
:1002E400002E06D1236820009B6F9847300009B088
:1002F400F0BD1E226B001340EA0913431822023B8F
:100304005A43A3180393303304931B7801270592AF
:100314001A003A4007923B4205D08E2218491948E8
:10032400D20001F025FB8023029ADB009A4203D914
:1003340013491548154AF4E7BB239B00E0582900EC
:100344000368029A1E6D069BB047061ECAD0059824
:100354000E991C302018FEF75FFD049B079A1B784A
:100364001F43049B1F70039B31331A70039B029A33
:100374009A85B7E7773B021004011580F20200006A
:10038400493A0210963B0210B83B02107104000077
:10039400BB239B0010B5C05803685B6B984710BD26
:1003A40070B50D00036804005B6F98472B0708D1F4
:1003B400C8239B00E558236820009B6F98472800BA
:1003C40070BD1E2369001940ED0929430239063B1B
:0803D4004B43E3189D8DEEE799
:1003DC00F7B50E00036804005B6F984737008F2356
:1003EC009F4301D1330706D1002217491300174848
:1003FC00009201F0CFFC1E22182573001340F20965
:10040C001343023B5D4365192B0030331B78DB072C
:10041C0009D42000FFF71AFF002810D00C490D4812
:10042C000D4A01F0A1FA31352B78002B07D0BB23F4
:10043C009B00E05831000368DB6E98472F702368EF
:10044C0020009B6F9847F7BD773B02100401158085
:0C045C00493A0210D03B02108C05000051
:1004680073B50D00036804005B6F98478F232A005B
:100478009A4301D12B0706D100221A4913001A48C2
:10048800009201F089FC1E2218266B001340EA092D
:100498001343023B5E43A619320030321178CB0772
:1004A80009D42000FFF7D4FE002816D00F491048C1
:1004B800104A01F05BFA02230B431370BB239B0025
:1004C800E0582900036831369B6D98473378002B34
:1004D80003D029002000FFF77DFF236820009B6FD1
:1004E800984773BD773B021004011580493A021002
:0804F800D03B0210CC0400000F
:10050000036810B5DB6F04009847C7239B00E35CCA
:10051000042B04D000200E4BE35A834217D10D4B1D
:100520000020E35C022B12D1094BE15A8F230A0011
:100530009A4382420BD10B0709D0BE239B00E35A9A
:10054000834204D12000C9B2FFF78EFF012010BD05
:08055000FA020000F6020000AF
:10055800F7B50E00036804005B6F98478F233200DD
:100568009A4301D1330706D100221D4913001D48C3
:10057800009201F011FC1E23182577001F40F30993
:100588001F432B00023F7B43E3181A0030321278D6
:10059800D20709D42000FFF75BFE00281AD01249C1
:1005A8001248134A01F0E2F931331B78002B03D0CB
:1005B80031002000FFF70EFF02227D436519303518
:1005C8002B78310093432B70BB239B00E0580368C2
:1005D800DB6D9847236820009B6F9847F7BDC0469E
:1005E800773B021004011580493A0210D03B0210F3
:0405F800F10400000A
:1005FC00036810B5DB6F04009847C7239B00E35CCE
:10060C00042B04D000200E4BE35A834217D10D4B20
:10061C000020E35C022B12D1094BE15A8F230A0014
:10062C009A4382420BD10B0709D0BE239B00E35A9D
:10063C00834204D12000C9B2FFF788FF012010BD0E
:08064C00FA020000F6020000B2
:10065400F0B50E001F00036885B05B6F03920400C1
:1006640098478F2332009A4301D1330706D10022E1
:10067400130021492148009201F090FB1E23182504
:1006840071001940F309194302394D4365192B00D0
:1006940030331B78DB0709D42000FFF7DBFD00288B
:1006A40010D017491748184A01F062F9AB8DBB42C4
:1006B40004D91300154916480092DDE731352A782C
:1006C400002A07D0236820009B6F9847002630003B
:1006D40005B0F0BDBB229200A05831000268176E2D
:1006E400039AB847061E02D02B7801332B70236877
:1006F40020009B6F9847EAE7773B021004011580BE
:10070400493A0210D03B0210AF050000DE3B021054
:040714000501158046
:1007180037B50D00036804005B6F98478F232A00E4
:100728009A4301D12B0706D1002215491300154819
:10073800009201F031FB1E236A001A40EB091A43AC
:100748001823023A5343E31830331B78DB0709D4E4
:100758002000FFF77DFD051E0CD00B490B480C4A05
:1007680001F004F9BB239B00E058290003685B6E85
:1007780098470500236820009B6F984728003EBDD6
:10078800773B021004011580493A0210D03B021051
:04079800E90500006F
:10079C00F0B50E0085B00293036803925B6F040002
:1007AC0098478F2332009A4301D1330706D1002298
:1007BC00130026492648009201F0ECFA1E23182556
:1007CC0071001940F309194302394D4365192B0087
:1007DC0030331B78DB0709D42000FFF737FD0028E6
:1007EC0012D01C491C481D4A01F0BEF8AB8D029971
:1007FC008B4204D213001A491A480092DCE72F00EE
:10080C0031373B78002B07D0236820009B6F98472B
:10081C000026300005B0F0BDBB239B00E058310032
:10082C000368039A9B6E9C46029B6646B047061E65
:10083C0009D0029BEB853B7801333B702368200089
:10084C009B6F9847E5E7E885F8E7C0462F3C021018
:10085C0004011580493A0210D03B02100A06000030
:08086C004D3C0210050115804E
:1008740037B50D00036804005B6F98478F232A0087
:100884009A4301D12B0706D10022124913001248C2
:10089400009201F083FA1E226B001340ED091D4300
:1008A4001823023D6B43E3181A0030321278D20742
:1008B40009D42000FFF7CEFC051E05D007490848DF
:1008C400084A01F055F8DD8D236820009B6F984796
:1008D40028003EBD773B021004011580493A0210FE
:0808E400D03B021049060000A0
:1008EC00036870B5DB6F04000D009847C7218900C1
:1008FC00625C6554D3B2AA4208D0032B07D9032DEE
:10090C000DD92368290020001B6E984770BD012B60
:10091C00F7D9012DF5D82000FFF730FCF1E7B42210
:10092C002000920000211C3006F088FE0023024AB1
:10093C00A354024AA354ECE71D030000F20200008A
:10094C00036870B5DB6F04009847BB23BE259B0082
:10095C00E058AD000368615DDB6A9847635B022178
:10096C00002B00D003212000FFF7BAFF012070BD3F
:10097C00036810B5DB6F04009847BE239B00E15C55
:10098C000C4BE15400290AD1313BE05803681B6A37
:10099C00984703212000FFF7A3FF012010BD01227F
:1009AC00054B2000E2541A330232E2542368DB6E0A
:0C09BC009847F2E71D030000F202000063
:1009C800036810B50400DB6F984700201A4BE35CFE
:1009D80083420ED1194BE05C0B282BD8EFF740FD72
:1009E800060A2A0E2A12162A1A1E22262000FFF7A5
:1009F80055FA10BD2000FFF7FDFDFAE72000FFF7CC
:100A08007BFDF6E72000FFF79DFFF2E72000FEF7E9
:100A1800DDFFEEE72000FFF7D3F9EAE72000FFF754
:100A2800A9FFE6E72000FFF7DDF9E2E72000FFF77E
:100A3800F7F9DEE70020DCE7F5020000F702000026
:100A4800036870B5DB6F04009847C5229200A1586F
:100A5800C4230432C325A05800229B00AD00E35CE8
:100A680062551B4AA25C002A10D0012B0AD8022327
:100A78006355BD239B00E1182368012220009B6E6B
:100A8800984770BD2000FFF733FBFAE7042B12D11B
:100A98002000FFF795FF002806D1BB239B00E058F4
:100AA8000368DB6C9847ECE7635D002BE9D1200015
:100AB800FFF7BCFAE5E7032BEFD00125054AA5545B
:100AC800063AA050043AA1500832A354EFE7C046B2
:080AD8002D0300000A030000D9
:100AE00010B504000368DB6F984702212000FFF770
:100AF000FDFE0022044B2000E254FFF745FB236873
:0C0B00002000DB6D984710BD1E030000B4
:100B0C0070B504000368104D5B6F9847635D002B54
:100B1C0007D0BB239B00E05803689B6998470023D0
:100B2C006355C7239B00E35C012B03D901212000F3
:100B3C00FFF7D6FE0023054A2000A354044AA35411
:100B4C0023689B6F984770BDF10200001D030000E5
:040B5C001E03000074
:100B600070B5BC2504000368AD005B6F9847635DFA
:100B7000002B0AD02000FFF7C9FFBB239B00E058E1
:100B80000368DB68984700236355236820009B6F48
:040B9000984770BD55
:100B9400036870B5DB6F0D0004009847002D08D181
:100BA400C7239B00E35C002B03D029002000FFF740
:040BB4009BFE70BD77
:100BB800F8B503680400DB6F9847C4231A4F9B00FD
:100BC800E65CE35D002B01D1002E0FD12000FFF77A
:100BD8003FFB051E0AD10100B422200092001C3000
:100BE80006F02EFD114BE554114BE554C3230022AA
:100BF8009B00E254E35D934203D02000FFF778FAAC
:100C0800F8BDBB239B00E0580368002E09D0DB69C0
:100C1800984720000421FFF765FE2000FFF706FA39
:100C2800EEE7DB6C9847EBE72D0300001D0300009F
:040C3800F2020000C4
:100C3C00F0B5060085B002930AAB1B881C360393F3
:100C4C00204B04000360BB2335009B0000910192F4
:100C5C00C71828001835FAF7ADFEBD42F9D1B422F9
:100C6C00019B0021A380029B3000E380039B920038
:100C7C00238106F0E3FCBD239B00E0182822002111
:100C8C0006F0DCFCBB23009A9B00E250BC22002344
:100C9C00012120009200A3520B4AA3544232A350CC
:100CAC00143AA3500432A3500432A3500432A3507C
:100CBC000432A354143AA154044AA354044AA3542E
:100CCC0005B0F0BD843C0210F20200001D030000D0
:040CDC001E030000F3
:100CE0000E4B70B50360BC239B00C35C0400002B5B
:100CF00004D00B490B480C4A00F03CFEFFF730FFD4
:100D0000BB2326009B00E5181C36B54204D0183DD5
:100D10002800F9F7D0FCF8E7200070BD843C0210F1
:0C0D2000493A02106E3C0210620500000F
:100D2C0037B50D0003680400DB6F98478F232A004A
:100D3C009A4301D12B0706D1002210491300104809
:100D4C00009201F027F81E226B001340ED091D43A1
:100D5C001823023D6B43E2183132117800290BD075
:100D6C001C330139E41820001170FBF774F80028CB
:100D7C0002D02000FDF7BEFD37BDC046773B021008
:040D8C0004011580C9
:100D900010B5EFF3108072B6054A1378002B05D119
:100DA00001210C00034B84431C70117010BDC04620
:080DB00057AB00204EAB002000
:100DB80010B5EFF310820123934304D0362206497D
:100DC800064800F0D3FD064A1370064B1B78002B2B
:100DD80000D062B610BDC046693D0210853D0210C4
:080DE80057AB00204EAB0020C8
:0C0DF000014B18787047C04657AB00203C
:100DFC0070B50D000400160002F05EF9013507D045
:100E0C000021200002F07AF93100200002F05CF998
:020E1C0070BDA7
:100E1E00F8B50D00040016001F0002F04CF9013564
:100E2E000BD03900200002F030F90121200002F031
:0C0E3E0064F93100200002F046F9F8BD14
:0A0E4A0010B50022FFF7D5FF10BD20
:0C0E540010B513000022FFF7E0FF10BDF6
:0A0E600010B50022FFF7F6FF10BDE9
:100E6A0070B50C00050011001A00002909D12100F3
:100E7A00FFF7BFFF013403D02800049902F007F9F5
:0C0E8A0070BD2100049BFFF7C5FFF9E7D5
:100E960000228B5E5A1C01D1180002E0834201D168
:080EA600486870470C31F3E7C6
:100EB00013B50400431C0AD0FFF7EDFF431C06D115
:100EC0000023220002490348009300F069FF16BD89
:080ED0009F3D0210300101807A
:100ED80000228B5E5A1C01D1180002E0834201D126
:080EE800886870470C31F3E744
:100EF00013B50400431C0AD0FFF7EEFF431C06D1D4
:100F00000023220002490348009300F049FF16BD68
:080F1000BF3D02103001018019
:100F1800F7B54668330032331C78002C32D10368A9
:100F28005B689847326A030082422BD0821A306984
:100F3800336210403322B256002A24DB2100EFF737
:100F48001BFC3427F75704000D00002F14D0002194
:100F5800706A24184D41009401958F421BDB3A00BA
:100F680020002900EFF7FCFB3A0004000D00EFF722
:100F780003FC009B181A7062B26AF36A12196B417B
:100F8800B262F362F7BDB1680200230008002100D5
:100F9800EFF7D8FCD5E7F7680B00009801993A00FD
:100FA800EFF7B0FC4743009B0400DF1B0D0077629E
:020FB800E2E76E
:100FBA000300824206D901208A4202D99942894114
:100FCA004842704700208B42FBD991424041F8E7E2
:100FDC00F0B545683E4B2A6B060085B01A426BD1C2
:100FEC00FFF794FF6B68002B00D167E01A685B6811
:100FFC00E96A994207D302D1A96A914203D33368B3
:10100C005B69984758E07468A06AE16A121A8B41D0
:10101C001900E369100067698B4224D302D1A369DC
:10102C00834220D33422A256002A29DBEFF7A2FBFD
:10103C00230033331B785BB29C46002B10D0A36883
:10104C000393039B013B009300230193009A019BA4
:10105C00801859416346002B1BDB6246EFF77EFB81
:10106C00874200D90700236AFB1827691F402B6AA7
:10107C00BB4213D1CA2217491748FF3200F074FC47
:10108C00E36802009C460B0060460021EFF758FC19
:10109C00CEE7039A019BEFF733FCE1E733683800A6
:1010AC001B69984733685B6898473A000100286AC7
:1010BC00FFF77DFF0028A2D105B0F0BD2B6A6A694D
:1010CC0028699B18184033681B699847F4E7C04699
:0C10DC0000FFFF00F23D0210043E021075
:1010E8004368F0B51A0030321278040085B0002A3F
:1010F80000D083E032331B78002B7FD103681B6854
:1011080098472368DB69984706680700002E06D1D0
:10111800330032003B493C48009600F03DFE300069
:101128003A490391EFF72CFA03980029F9D1010005
:101138003648EFF79FF91F23012265680290A860DF
:10114800013B04D31100029899408842F8D12A0043
:101158003332137003993000EFF78CF980210300C4
:101168001F22E8600906884206D00121013A03D30C
:10117800080090408342F9D1290034310A70786818
:10118800011F1C2905D9002221491300214800927A
:10119800C3E70122202833D08240013A07200027E4
:1011A80088401E002A613B00029A6861C117EFF768
:1011B800C9FB02000B0001204042C1178019794188
:1011C8008018594132003B00EFF79CFB2368A86167
:1011D800E9615B682F606F609847002128620122EF
:1011E800002063689862D9625F621A8632332000F1
:1011F8001F70FFF78DFE2000FFF7ECFE05B0F0BD75
:101208005242CBE7283E02100E01048040420F00F4
:08121800413E021005010480B3
:1012200070B5050000F054FC2B686C68DB689847CB
:10123000230032331B78002B02D000F05FFC70BD1E
:1012400026000123313633706368002B16D0280046
:10125000FFF762FE6368E26A596891420ED803D1D3
:101260001968A26A914209D86A68DB6852686360AB
:101270002368002BE8D090689847E5E70023280012
:081280003370FFF7ABFED8E765
:1012880070B50400FFF72CFF00F01EFC2000FFF7EC
:101298003FFE63689C6ADD6A00F02CFC2900200090
:0212A80070BD17
:0812AA0010B5FFF7ECFF10BDC9
:1012B40010B50022024B1A7003F06FFA10BDC0463D
:0412C4004BAB002010
:1012C80010B503F01FFA0122014B1A7010BDC04679
:0412D8004BAB0020FC
:0812DC0000487047803E02103B
:1012E400034B10B51B68002B01D00248984710BD72
:0812F400D0040020803E02102E
:1012FC0010B50C23CA5E0423C95E02F0D7FF10BDE3
:0C130C0010B5040000F0DEFB200010BD56
:0C13180010B5040000F0EEFB200010BD3A
:04132400007B704793
:101328000E4B70B5036000230D4E4360816002735D
:10133800040030000D00FDF709FB01F047FA002D0D
:101348000AD0084B1A681C6062603000FDF7FEFA8C
:1013580001F058FA200070BD6560F6E7BC3E021047
:081368001C9C0020189C0020D1
:1013700070B50400144B154D03602800FDF7EAFA20
:1013800001F028FAA368002B05D0114962680B68A8
:10139000A34213D10A600F4B1A68A24201D1002266
:1013A0001A602800FDF7D6FA01F030FA237B002BF3
:1013B00002D1201F01F05AF8200070BD19005B68AF
:1013C000A342FBD14A60E6E7BC3E02101C9C002011
:0813D000189C0020449C002041
:1013D80010B50400FFF7C8FF2000102101F02CF819
:0413E800200010BD14
:1013EC00F7B51A4E019030000D00FDF7ADFA01F083
:1013FC00EBF9174B1C68002C11D1072D1ED12A00BC
:10140C001448019906F062F8002817D13000FDF756
:10141C009BFA01F0F5F9104B1C682000FEBDA76883
:10142C00002F11D0380006F009FCA8420CD12A007C
:10143C003800019906F04AF8002805D13000FDF774
:10144C0083FA01F0DDF9E8E76468D4E71C9C00201E
:0C145C00189C0020AC3E0210449C0020B4
:0414680000207047A9
:10146C00036870B5012200211B6904009847051E12
:10147C000DDB2368022200211B692000984706001F
:10148C0023682900002220001B699847350028009A
:02149C0070BD21
:1014A00070B50E000024104904604460050030004F
:1014B00006F0FCFB3018030021001A782F2A08D10F
:1014C00001332B60002909D12A220849084800F07D
:1014D00051FA002AF5D001310133EEE7FFF786FF1C
:1014E0006860280070BDC046143F0210303F0210F3
:0414F0003D3F02106A
:0414F40000687047D5
:1014F800436810B5181E05D0FFF710FF01384342A6
:061508005841C0B210BD05
:10150E0010B50400FFF7F1FF0023984203D0636883
:0A151E00002B00D0043B180010BDA4
:10152800436810B5181E04D0FFF7F8FE434258412F
:04153800C0B210BD70
:10153C0010B50400FFF7F2FF0023984203D0636854
:0A154C00002B00D0043B180010BD76
:0A1556004068431E9841C0B2704780
:0415600000207047B0
:10156400F8B50E00036804001B6D8D18984733000E
:1015740022689D4207D019785F1C2000936C98471D
:10158400013006D13D00236820005B6D9847A81BFD
:06159400F8BD3B00ECE78E
:10159A00F8B50E00036804001B6D8F1835009847D4
:1015AA002368AF4205D1236820005B6D9847A81BCA
:1015BA00F8BDDB6C20009847431CF4D02870013535
:0215CA00EEE74A
:0415CC000020704744
:0215D000704762
:1015D40013B504000E4B002208C0FFF7A3FE0D4B09
:1015E400200023600C4B0D4963600023636100F00D
:1015F40099FF6061002806D10300020000900849A9
:10160400084800F0CBFB00F0D6FC200016BDC04615
:10161400CC3E0210C43F021024400210463F021088
:08162400493F02101901018089
:10162C0010B50400074B0360074B4360406904F09E
:10163C00A3FC064B201D2360054B6360FFF792FE55
:10164C00200010BDC43F021024400210643F021061
:04165C00B43F021085
:1016600030B5002585B01A4CAB0029001948E25866
:10167000013500F013FA0D2DF5D1A36C1648029335
:10168000636C0193236C0093E36BA26B616B00F0BE
:1016900005FA124B1248196800F000FAE36C1B07B8
:1016A00012D5104800F0FAF9236D0F48DB0700D47B
:1016B0000E4800F0F3F9E36C0D485B0700D40D48C9
:1016C00000F0ECF905B030BD0B4800F0E7F9EFE7AA
:1016D00070A700202C4002103A40021000ED00E0FC
:1016E0008940021097400210A6400210B340021039
:0C16F000D6400210E2400210C64002107A
:1016FC00F7B51B4F05000E003800012100F04CF926
:10170C000024A04216D1174800F0C2F9302D18D091
:10171C00402D1BD0202D1ED1134800F0B9F9134CCD
:10172C00134800F0B5F9FFF795FF124800F0B0F937
:10173C0000233B700023320020000F49009300F07F
:10174C0029FB0E4800F0A4F90D4CE9E70D4800F018
:10175C009FF90D4CE4E70D4800F09AF90C4CDFE7CB
:10176C0053AB0020EE400210174102103E01FF80E7
:10177C00444102104F4102106E41021026410210EA
